:020000040803EF
:10C00000C0E7002051C3030841190408950D040836
:10C01000E11604080DE50308895D0408000000002E
:10C02000000000000000000000000000B9C203088A
:10C03000ADF0030800000000FDC2030885470408B6
:10C040006BC30308412504086BC30308B12E040821
:10C050006BC303086BC3030881000408F1000408E4
:10C0600013010408330104085501040805E8030816
:10C0700079E80308EDE803086DE90308EDE9030832
:10C080006DEA0308EDEA03086BC303086BC30308FA
:10C090006BC303086BC303086BC303087501040873
:10C0A0006BC303086BC303086BC303086BC30308AC
:10C0B0006D48040891480408B94804086BC3030894
:10C0C0006BC303086BC303086BC303086BC303088C
:10C0D0006BC30308AD590408295A0408A55A04087B
:10C0E000A1000408AD2A04086BC303086BC303084E
:10C0F0006BC303086BC303086BC303086BC303085C
:10C100006BC303086BC30308E14804086BC303084F
:10C1100011550408915504080949040831490408D7
:10C120006DEB0308EDEB03086DEC0308F1EC03087D
:10C1300000F002F800F0B0F80AA090E8000C824489
:10C140008344AAF10107DA4501D100F0A5F8AFF266
:10C15000090EBAE80F0013F0010F18BFFB1A43F0E5
:10C1600001031847A80B0100C80B01000A444FF057
:10C17000000C10F8013B13F0070408BF10F8014B46
:10C180001D1108BF10F8015B641E05D010F8016B8B
:10C19000641E01F8016BF9D113F0080F1EBF10F8EF
:10C1A000014BAD1C0C1B09D16D1E58BF01F801CB12
:10C1B000FAD505E014F8016B01F8016B6D1EF9D595
:10C1C0009142D6D3704700000023002400250026AA
:10C1D000103A28BF78C1FBD8520728BF30C148BFEA
:10C1E0000B6070476E2900F0D781702900F0BD8286
:10C1F00066290FF0138065290FF0108067290FF072
:10C200000D8061290FF00C8003681B0A28BF41F0E4
:10C210008001692900F08481642900F081817529F9
:10C2200000F07E816F2900F04A82782900F089822F
:10C23000E92901F03F80E42901F03C80F52901F073
:10C240003980EF2900F04782F82900F088820368DE
:10C25000DB0928BF41F08001632900F0F6877329CC
:10C2600000F0FB87E32901F01980F32901F01E801B
:10C27000002070471FB501F0B7F80400002000212E
:10C280000EF0AAF9401C6060002000210EF0BAF9FF
:10C29000E0601FBD10B510BD01F074FB1146FFF743
:10C2A000E9FF0AF029FC01F0A0FB03B4FFF7F2FF5D
:10C2B00003BC0AF048F80000224B19680868B0E88F
:10C2C000F00F80F30988BFF36F8F4FF0000080F309
:10C2D00011884EF00D0E70470000000006480068FF
:10C2E000006880F3088862B661B6BFF34F8FBFF372
:10C2F0006F8F00DF00BF00BF08ED00E0EFF30980A3
:10C30000BFF36F8F0F4B1A6820E9F00F106008B56C
:10C310004FF0500080F31188BFF34F8FBFF36F8F42
:10C320000DF076FA4FF0000080F31188BDE8084068
:10C3300019680868B0E8F00F80F30988BFF36F8FC1
:10C34000704700BF74060020EFF3058070470000BF
:10C350000948804709480047FEE7FEE7FEE7FEE799
:10C36000FEE7FEE7FEE7FEE7FEE7FEE704480549D5
:10C37000054A064B70470000FD47040831C1030819
:10C38000C0B70020C0E70020C0C70020C0C7002001
:10C39000704710B5044600F0A9FC0068005DC006B7
:10C3A00002D504F1200010BD204610BD7CB51D460D
:10C3B00016460C00009001D02044401E074B7B44E1
:10C3C0002A4669460190304600F015FF05461CB12B
:10C3D0000020694600F022FF28467CBD650E000063
:10C3E0000FB4044910B503AA029800F03BFF10BC3B
:10C3F0005DF814FBC40500200FB41CB5084B06AA59
:10C400007B4469460090059800F0F5FE0446002044
:10C41000694600F003FF20461CBC5DF814FB0000D9
:10C42000190E00000FB47CB50C0009AA009001D0D1
:10C430002044401E084B7B4469460190089800F058
:10C44000DAFE05461CB10020694600F0E7FE2846EA
:10C450007CBC5DF814FB0000ED0D000070B50446D7
:10C4600085690068C10601D5302600E02026C00796
:10C4700007D070BDD4E9012130469047206A401CA6
:10C4800020626D1EF6D570BD70B5044685690078D2
:10C49000C00707D170BDD4E9012120209047206A50
:10C4A000401C20626D1EF6D570BD09684A0501D595
:10C4B00040B27047C905FCD500B2704709684A050B
:10C4C00001D5C0B27047C905FCD580B2704770B5C0
:10C4D0000C460546012A05D02878800600D5EA6971
:10C4E000002302E0012305E05B1C934202D2E05CE2
:10C4F0000028F9D1A869E618C01AA861286A18446A
:10C5000028622846FFF7AAFF04E0D5E9012114F8C4
:10C51000010B9047B442F8D32846FFF7B5FF70BD32
:10C520002DE9F0410646002410687529314616A50C
:10C5300010D0FFF7BAFF002802DA404213A507E047
:10C5400031688A0701D512A502E0490704D511A573
:10C55000012401E0FFF7B2FF00210A2206F12407BF
:10C5600009E0B0FBF2FCB0FBF2F302FB1C00303040
:10C5700078541846491C0028F3D123462A463046F1
:10C58000BDE8F04100F0C9BB000000002D00000034
:10C590002B0000002000000011680268006A5305AB
:10C5A00001D508700AE0D30501D5088006E013061E
:10C5B00003D5C217C1E9000200E0086001207047FE
:10C5C0002DE9FF5F15468A460446DFF8AC80F84443
:10C5D0000027D8E900103E46CDE9001010E03AF8F7
:10C5E00016106A4602A800F0DBFE411C07D0217835
:10C5F000890603D5E269391891420DD80744761CA3
:10C600002078800602D5E069B84205DDAE42E6DB5F
:10C610003AF816000028E2D1A069C01BA0612046AC
:10C62000FFF71CFFD8E90010CDE90010002017E04B
:10C630003AF818106A4602A800F0B2FEB0F1FF3FC7
:10C6400081460BD000250DF1080B05E0D4E901214E
:10C650001BF8050090476D1C4D45F7D308F101000C
:10C66000B0428046E4DB206A384420622046FFF76F
:10C670000BFFBDE8FF9F00007200010030B40021F5
:10C6800000F1240408E002F00705D208303542EA40
:10C690004372DB086554491C52EA0305F3D1046870
:10C6A000002310A2250707D5A40600D421B1C46930
:10C6B00001230DA2641EC46130BC00F02EBB10B576
:10C6C000044621461068FFF7F9FE02462046BDE801
:10C6D00010400023D2E7D21D22F00701D1E9002348
:10C6E000CCE700000000000030000000F0B40D4670
:10C6F0000188090502D5214C7C4402E01F4C7C4492
:10C700000E34002100F1240608E002F00F071209A0
:10C71000E75D42EA03721B097754491C52EA03079A
:10C72000F3D102780023120704D5702D06D009B189
:10C73000022311342246F0BC00F0EFBA012310347A
:10C74000F8E770B504460D4621461068FFF7B6FEBF
:10C75000024629462046BDE870400023C6E7D21DA8
:10C7600022F00703D3E90023C0E70368126843F00F
:10C77000200303600823C3610023B7E750FF0000D4
:10C780002DE9F05F894604464FF0000ADFF874B1E6
:10C79000FB44C0F820A02046E1688847002874D0F8
:10C7A000252806D0D4E901219047206A401C206248
:10C7B000F1E700265F462046E168884720280546C5
:10C7C00007DB312D05D2781910F8200C08B106438B
:10C7D000F1E7B00701D526F00406C4F81CA0002735
:10C7E000C4F818A02A2D09D0284609F0A5FD38B3B1
:10C7F00004EB8708303DC8F8185019E059F8041BBD
:10C80000204604EB87029161E1688847012F0546C5
:10C8100018D1E069002820DA26F020061DE0D8F8BB
:10C82000180000EB800005EB40003038C8F8180015
:10C830002046E1688847054609F07EFD0028EED1D4
:10C84000012F0AD02E2D08D12046E16888477F1C91
:10C850000546022F46F02006C4DBA069002803DA53
:10C86000404246F00106A061F00701D026F0100614
:10C870006C2D0BD0682D09D04C2D39D06A2D35D0B8
:10C88000742D35D07A2D33D016E038E0E1682F468C
:10C8900020468847B842054609D16C2F26D04FF470
:10C8A0008060E168064320468847054604E06C2F17
:10C8B0001AD04FF4807006430DB3A5F1410019283A
:10C8C00002D8203546F400664A46294620462660AE
:10C8D0004E46FFF787FC80B101280BD0F61D26F0ED
:10C8E000070000F1080956E74020E4E78020D8E778
:10C8F0000020D6E706F104094DE7284652E7206AF2
:10C90000BDE8F09FE0FE000070B5064600F0F6F9C5
:10C910000468054630460A22002100F009FD2C601B
:10C9200070BD401ECAB210F8011F8A4202D0002911
:10C93000F9D10020704710B5431E13F8014F002CA9
:10C94000FBD105E011F8014B002C03F8014B03D09B
:10C95000521EF7D20021197010BD40EA010310B534
:10C960009B070FD1042A0DD310C808C9121F9C427F
:10C97000F8D020BA19BA884201D9012010BD4FF071
:10C98000FF3010BD1AB1D30703D0521C07E00020BE
:10C9900010BD10F8013B11F8014B1B1B07D110F81B
:10C9A000013B11F8014B1B1B01D1921EF1D118461E
:10C9B00010BD40EA0103024630B59B0710D14FF08D
:10C9C000013400E008C208C91D1B9D4315EAC41FBD
:10C9D000F8D013F0FF0102F8011B0DD01B0AF8E795
:10C9E00011F8013B002B02F8013B05D011F8013B87
:10C9F000002B02F8013BF3D130BD0022CBB210F87E
:10CA0000011B994200D1421E0029F8D110467047FF
:10CA100010B5431C02E010F8011B71B18107FAD177
:10CA20004FF0013202C88C1A8C4314EAC211F9D0BB
:10CA3000C01A0A0603D0C01E10BDC01A10BD0A04D9
:10CA400001D0801E10BD0902FCD0401E10BD40EA7E
:10CA5000010370B59B072ED14FF00136042A2AD36B
:10CA600008C810C99D1B9D43121F15EAC61517D093
:10CA7000D8B2E1B2401A50EA056110D198B2A1B221
:10CA8000401A50EA05410AD123F07F4024F07F414B
:10CA9000401A50EA052102D1180EA0EB146070BDB7
:10CAA000A342DBD018BA21BA884201D9012070BD57
:10CAB0004FF0FF3070BD0AB9002070BD10F8013B87
:10CAC00011F8014B63B1A3420AD1521E08D010F8ED
:10CAD000013B11F8014B1BB1A34201D1521EEDD114
:10CAE000181B70BD421E12F8013F002BFBD111F83C
:10CAF000013B002B02F8013BF9D17047032A40F2B9
:10CB0000308010F0030C00F0158011F8013BBCF1EF
:10CB1000020F624498BF11F801CB00F8013B38BF07
:10CB200011F8013BA2F1040298BF00F801CB38BF15
:10CB300000F8013B11F0030300F02580083AC0F033
:10CB4000088051F8043B083A51F804CBA0E80810DB
:10CB5000F5E7121D5CBF51F8043B40F8043BAFF30E
:10CB60000080D20724BF11F8013B11F801CB48BF68
:10CB700011F8012B24BF00F8013B00F801CB48BF9E
:10CB800000F8012B704710B5203AC0F00B80B1E8D7
:10CB90001850203AA0E81850B1E81850A0E81850F2
:10CBA000BFF4F5AF5FEA027C24BFB1E81850A0E8FB
:10CBB000185044BF18C918C0BDE810405FEA827C15
:10CBC00024BF51F8043B40F8043B08BF7047D2072C
:10CBD00028BF31F8023B48BF11F8012B28BF20F8CD
:10CBE000023B48BF00F8012B704702F0FF0343EA05
:10CBF000032242EA024200F002B84FF00002042988
:10CC0000C0F0128010F0030C00F01B80CCF1040C7B
:10CC1000BCF1020F18BF00F8012BA8BF20F8022BAF
:10CC2000A1EB0C0100F00DB85FEAC17C24BF00F855
:10CC3000012B00F8012B48BF00F8012B70474FF083
:10CC4000000200B5134694469646203922BFA0E85C
:10CC50000C50A0E80C50B1F12001BFF4F7AF090768
:10CC600028BFA0E80C5048BF0CC05DF804EB890059
:10CC700028BF40F8042B08BF704748BF20F8022B9C
:10CC800011F0804F18BF00F8012B704710B5044613
:10CC900010F0030F08BF11F0030F40F015804FF0A4
:10CCA000013E121FC0F20E8051F8043BA3EB0E0CA4
:10CCB0002CEA030C1CEACE1C08BF40F8043BF0D061
:10CCC000A1F1040102F10402521E08DB11F8013B3C
:10CCD000002B00F8013BF7D11146FFF78EFF2046ED
:10CCE00010BD7047704770477047000010B500F0E6
:10CCF0007BFB001D10BD00BFE1D80000004870475D
:10CD00005CB7002010B5FFF7F9FF006810BD10B543
:10CD10000446FFF7F3FF046010BD2DE9F0470D4610
:10CD200099469246044600F124080168880604D515
:10CD3000E06921F01001216000E00120A84201DD3E
:10CD4000471B00E00027A1697A1902EB0900081AC5
:10CD5000A0612078C00602D42046FFF77FFB0026A2
:10CD600008E0D4E901211AF806009047206A401C27
:10CD7000761C20624E45F4DB2078C0060AD520469A
:10CD8000FFF76CFB06E0D4E9012130209047206AD0
:10CD9000401C2062381EA7F10107F4DC07E0D4E94B
:10CDA000012118F805009047206A401C2062281EC7
:10CDB000A5F10105F3DC2046FFF766FB20780006AD
:10CDC00002D50220BDE8F0870120FBE770472DE97E
:10CDD000FF4F0C461E464FF0FF378BB0D2E90001E3
:10CDE000DDF860800A908A46C1F30A5505B93D46D0
:10CDF000002108464FF00000BAF1000F00F4400097
:10CE000005DA00EB80004FF4400101EA50004FEAE0
:10CE10009059B9F1010F00DDB9460A9850EA4A006D
:10CE20000ED044F61050A5F2FF3545432F14B8F14B
:10CE3000000F1ED07542291E1EDDC9F100021CE044
:10CE4000B8F1010F4FF0000001D0302103E0F243B0
:10CE500005E02154401CB042FBDB3046002200219B
:10CE600021540B99C1F80880C1E900200FB0BDE83A
:10CE7000F08FBD1B6D1CDEE74A4600DA694206A84A
:10CE800000F00AFD06AB93E8070003AB83E8070058
:10CE900050460A9900F0F2FD8DE80700A0F5005019
:10CEA0001F3800900398002D0ADD42F21F014A4608
:10CEB0000844002303A90390684601F05BF809E0E9
:10CEC000A0F500504A461F38002303A90390684686
:10CED00001F065F88DE807000004000C03D04FF066
:10CEE000FF30410800E01046B8F1000F03D00022E7
:10CEF000009215461EE0751E05D400F079FA303216
:10CF000062556D1EF9D5B3460122084302D00022B6
:10CF10007F1C04E02078302801D100227F1E002AE7
:10CF2000099784D01DE0112D07DA00F061FA303244
:10CF300062556D1C50EA0102F5D1084302D00098F9
:10CF4000C8B10EE00021681E05E0235C625C6354FA
:10CF50002254401E491C8142F7DBAB46A81B401EF1
:10CF60000990002004F80B000B98099AC0F808807B
:10CF7000C0E9002B7AE711264FF0000857E72DE9AA
:10CF8000F04F88460446D21D22F0070191B0D1E946
:10CF90000001CDE90A0109F043F902460B98C00FE0
:10CFA00001D02D2007E02068810701D52B2002E069
:10CFB000202101EAC000032A099001D0072A05DBDD
:10CFC00003464146204600F0D7FB0BE1207880065F
:10CFD00001D5E06900E00620B8F1650F814606D072
:10CFE000B8F1660F18D0B8F1670F70D131E00020AA
:10CFF000B9F1110F009001DB112301E009F10103E8
:10D000000AAA01A90CA8FFF7E2FEDDE90C700026D0
:10D0100009F10105834647E001204B4600904FF09F
:10D0200000470AAA01A90CA8FFF7D1FEDDE90DB05F
:10D030000C995D46002610B909F101000D18B9EBF5
:10D04000050003D4C0F1FF3609F10105A5EB090085
:10D050002BE0B9F1010F01DA4FF001090020B9F11D
:10D06000110F0090484601DD112300E003460AAA93
:10D0700001A90CA8FFF7ABFEDDE90C704D460026B8
:10D080008346207800070AD4AB4500DA5D4601A844
:10D09000012D04DD411911F8011C302907D04F453D
:10D0A00002DA17F1040F04DA012082460FE06D1E48
:10D0B000EEE7002F02DCED1B3E4403E0781CA842A3
:10D0C00000DD7D1CB81B00F1010A4FF000472078FD
:10D0D000000703D4AA4501DB4FF0FF3A0021B7F166
:10D0E000004F0DF143088DF8431024D002202B236C
:10D0F000002F01DA7F422D230A21021EA0F1010038
:10D1000000DC5FB197FBF1FC97FBF1F201FB1C7CAB
:10D1100017460CF1300C08F801CDEEE7A8F101003C
:10D1200003702188090501D5452100E06521A0F1A2
:10D13000010800F8011C09980FA9A1EB0807FF1DC1
:10D1400000B10120411901EBEA70A1693844081AC5
:10D15000401EA0612078C00602D42046FFF77EF969
:10D16000099828B1D4E901219047206A401C206227
:10D170002078C00622D52046FFF770F91EE0002E69
:10D1800004DBB34502DD01A8805D00E03020D4E976
:10D1900001219047206A401C2062761CAAF1010000
:10D1A0005FEA000A0AD100F01FF9C0680168405C1C
:10D1B000D4E901219047206A401C2062281EA5F175
:10D1C0000105DCDC07E0D4E9012118F8010B9047E8
:10D1D000206A401C2062381EA7F10107F3DC2046BC
:10D1E000FFF752F9032011B041E6000001694A1C23
:10D1F00002610878704700B58FB0CDE90131002198
:10D20000059105497944CDE9031011466846FFF7B9
:10D21000B7FA0FB000BD0000E5FFFFFF0A6802F893
:10D22000010B0A607047D1E900239A4202D2531CD5
:10D230000B601070704710B5436913B1AFF30080F5
:10D2400001E0FFF744F9012010BD127800F124013C
:10D250000A7000224A700122EDE711684FF0FF3298
:10D26000E9E70000074B70B50D467B44FFF7C3FFAD
:10D270000446284600F082FB10B14FF0FF3070BD2D
:10D28000204670BDFB93000010B5436913B1AFF3A6
:10D29000008001E0FFF794F9012010BD128800F131
:10D2A000240182840022C2840122EDE711684FF03C
:10D2B000FF32E9E72DE9F0418046D21D22F0070256
:10D2C0000025D2E90002F52915A614D0011E72F13D
:10D2D000000106DA0023D0EB030063EB020211A683
:10D2E00008E0D8F800108B0701D50FA602E0490727
:10D2F00001D50EA601251146002408F1240704E0FB
:10D3000000F076F830323A55641C50EA0102F7D149
:10D310002B46324621464046BDE8F041FFF7FDBCB2
:10D32000000000002D0000002B0000002000000085
:10D330002DE9F04791460F4680460446002614F832
:10D34000015B2DB1FFF7D2FC0068405DC007F6D14C
:10D350002B2D02D02D2D18D0641E4A46394620466A
:10D3600000F04AFA27B13968A14201D1C7F800801C
:10D370004FF0020471050BD54042002803DDFFF792
:10D38000BDFC0460A007BDE8F08746F48066E4E7D2
:10D390000028F8DAFFF7B2FC04606FF00040F2E713
:10D3A00070B516460C460546FFF7A0FC036893F8D7
:10D3B0000101012806D0FF2C0FD8185D68B10120AB
:10D3C0002C7070BDD3F807013246214603F20713D3
:10D3D00003442846BDE8704018474FF0FF3070BD49
:10D3E000004870475CB70020004870477CB70020B9
:10D3F00030B5B0F10A024FEA900E71F100034EEA27
:10D40000817EB0EB0E0061EB91014FEA101E4EEAF7
:10D41000017E10EB0E0041EB11114FEA102E4EEA87
:10D42000016E10EB0E0041EB11214FEA104E4EEA57
:10D43000014E10EB0E0041EB1141401841F100018B
:10D440004FEAD00040EA41704FEAD10110EB80056D
:10D450004FEA810444EA907444EB01046D1944EBF3
:10D460000404521BA3414FF0000348BF0A3200D509
:10D4700030BD401C41F1000130BD00002DE9F04FEE
:10D4800004460D46D21D22F0070089B0D0E900976E
:10D490004846394608F0C4FE0246F80F01D02D2355
:10D4A00007E02068810701D52B2302E0202101EA53
:10D4B000C0038DF820300BB1012000E00020032ACA
:10D4C000824601D0072A04DB2946204600F054F9A1
:10D4D0003FE12078800601D40D2500E0E569C7F31F
:10D4E0000A560D2D49DA00214FEA175B08464FF026
:10D4F0000000002F00F4400007DA00EB80004FF43A
:10D50000400100EBD07001EA60008115012901DDC6
:10D510004FF0FF3100224FEA850CBCF1180F06D303
:10D520001346ACF118004FF08052C24003E04FF4B4
:10D53000801323FA0CF30CF10C0CBCF1200F04D374
:10D54000ACF1200C09FA0CF001E007FA0CF000290C
:10D550004FF0004801DD18B90FE00ED140450CD363
:10D5600019EB02095F4121B9404502D19F4329EAE5
:10D570000209BBEB175F00D0761C2088000502D59E
:10D580007B48784402E07A487844193808AA302366
:10D5900002F80A30037C0AF10101002E0AF1020AA6
:10D5A00053546A4602DC4FF0300101E04FF0310184
:10D5B0004FF001088DF8001002D0A6F2FF3603E00C
:10D5C00059EA470100D06B4E002D02DC2178090793
:10D5D00004D54FF002082E218DF80110C446002119
:10D5E0000BE0C7F303433F01C35C491C6D1E02F807
:10D5F0000830052908F1010801DA002DF1DC0021CD
:10D600000CE000EB1973491C1B786D1E082902F809
:10D6100008304FEA091908F1010801DA002DF0DCA1
:10D6200021688B0602D516E0A8F10108E04505DD6A
:10D6300002EB080313F8013C302BF5D0B8F1000FD2
:10D6400009DD02EB080313F8013C2E2B03D1090777
:10D6500001D4A8F10108002D05DD3E2102F80810D3
:10D660006D1E08F10108407C002E02F8080008F148
:10D67000010804DA2D20764202F8080002E02B208F
:10D6800002F808000A214FF47A70864208F1010876
:10D690000BDB96FBF0F3303302F8083096FBF0F327
:10D6A00008F1010800FB136601E0642E0CDB642026
:10D6B00096FBF0F3303302F8083096FBF0F308F1F4
:10D6C000010800FB136601E00A2E06DB96FBF1F071
:10D6D000303002F8080008F1010896FBF1F001FB78
:10D6E0001060303002F80800A16908F1010808EB69
:10D6F000050202EB0A00081AA0612078C00602D4D5
:10D700002046FEF7ABFE216A08AE01EB0A0020625C
:10D7100004E0D4E9012116F8010B9047BAF1010A9F
:10D72000F7D22078C00602D52046FEF797FE6E4657
:10D7300009E016F8010B3E280FD0D4E901219047EB
:10D74000206A401C2062B8F10108F2D22046FEF7A0
:10D750009BFE09B00320BDE8F08F206A28442062B8
:10D7600003E0D4E90121302090476D1EEBD3F8E7A8
:10D77000DDF1000002FCFFFF2DE9F0411F460446E9
:10D7800003260168072A01F4006004DB08B116A52E
:10D7900005E016A503E008B115A500E015A521F0E8
:10D7A00010002060A069C01EA0610FB1401EA061E2
:10D7B0002046FEF753FE4FB1D4E901213846904789
:10D7C000206A401C2062C01C206206E0206AFAE742
:10D7D000D4E9012115F8010B9047761EF8D22046B6
:10D7E000FEF752FEBDE8F0814E414E006E616E00C4
:10D7F000494E4600696E66002DE9F05F8246154687
:10D800008B4600270AF10104B9460078302801D080
:10D810009DB113E014F8010B0127782803D0582894
:10D8200001D045B10AE00DB1102D07D1002714F841
:10D83000010B102502E0082500E00A250026B0466D
:10D840000EE005FB080005FB06F101271FFA80F832
:10D8500001EB1046B6F5803F00D3B94614F8010B32
:10D86000294600F0B4F80028EBDABBF1000F05D030
:10D870000FB1641E00E05446CBF80040B9F1000F30
:10D8800006D0FFF73BFA02210160C81EBDE8F09FF9
:10D8900048EA0640FAE700002DE9F04781461646BF
:10D8A0008AB0354878440DC88DE80D003248784478
:10D8B000801C03AC0DC884E80D0041F69B30084481
:10D8C000372190FBF1F290FBF1F5A5F1800501FB0A
:10D8D00012041B3C02D56442012000E00020DFF866
:10D8E00098A080460027FA44AAF1BE0A0EE0E0079D
:10D8F0000AD03246684607EB470101230AEB810153
:10D9000000F04DFB8DE8070064107F1C002CEED169
:10D91000194F7F44AE3F19E0E80715D007EB04101C
:10D920000DF1180A90E80E008AE80E00C068F04277
:10D9300001D1981908903246012306A903A800F0E6
:10D940002EFB03AB83E807006D10641C002DE3D1B0
:10D950004FF0010332466946B8F1000F03A802D028
:10D9600000F008FB01E000F01AFBC9E90001C9F86A
:10D9700008200AB0BDE8F0874CEF0000007B00F003
:10D98000800070477546FFF72BFDAE4605006946DF
:10D99000534620F00700854618B020B5FEF7E6FC98
:10D9A000BDE820404FF000064FF000074FF00008A0
:10D9B0004FF0000B21F00701AC46ACE8C009ACE821
:10D9C000C009ACE8C009ACE8C0098D4670473A28E8
:10D9D00000D2303820F02002412A01D3A2F13700D2
:10D9E000884201D34FF0FF30704710B50446AFF3C3
:10D9F00000802046BDE81040FEF757BC4FF0013CC8
:10DA000050F8042B51F8043B9A4221D1A2EB0C03AD
:10DA1000934313EACC1317D150F8042B51F8043B6D
:10DA20009A4215D1A2EB0C03934313EACC130BD10A
:10DA300050F8042B51F8043B9A4209D1A2EB0C0395
:10DA4000934313EACC13DBD04FF00000704700BFC4
:10DA5000D01A01BAB1FA81F101F0180122FA01F0ED
:10DA6000CB40C1F12001DBB2C0B2C01A2CFA01F3E5
:10DA7000D11A914311EAC311E6D170475FEA400C15
:10DA800008BF91F0000F4FEA8C234FEAC12243EA0E
:10DA900051514FEA1C5018BF00F5F0404FEA3000DA
:10DAA00018BF41F000415FEA6C5C00F02980BCF1D6
:10DAB000FF3F08BF40F080407047130C06BF1204C0
:10DAC0004FF0100C4FF0000C130E04BF12020CF1BB
:10DAD000080C130F04BF12010CF1040C930F04BFC8
:10DAE00092000CF1020CD30F04BF52000CF1010C98
:10DAF00011464FF00002A0F11F00A0EB0C00704790
:10DB000011F0004F08BF704731F000413FF4D5AF2E
:10DB10000B0C06BF09044FF0100C4FF0000C0B0E5D
:10DB200004BF09020CF1080C0B0F04BF09010CF132
:10DB3000040C8B0F04BF89000CF1020CCB0F04BF47
:10DB400049000CF1010CCCF12003A0EB0C0022FAEF
:10DB500003F302FA0CF241EA030100F101007047FD
:10DB600020F07F4C80EA030023F07F47ACEB0703F3
:10DB700003F57C5300F0004003F1FF032DE98049D9
:10DB80004FEA154B09B44FEA144325EA0B4E24EA39
:10DB900003480FF2042606EB132749083E785FEA94
:10DBA000320203FB0667C7F5000707FB06F64FEADC
:10DBB00054374FEAD64606F1020607FB066CCCF155
:10DBC000005C4FEA1C472CEA074C07FB06F40CFBF1
:10DBD00006F504EB15464FEA961634BF00204FF0C9
:10DBE00000404FEAD13706FB07FC4FEA1C4C0CFB08
:10DBF0000BF7D21B03FB0CF761EB07010CFB0EF7D5
:10DC0000B0EB074072EB17420CFB08F734BFA2EBF6
:10DC10000742B2EB074261EB17414FEA0C444FEA6F
:10DC2000910706FB07FC4FEA1C4C0CFB0BF7B0EB13
:10DC3000C74072EB573203FB0CF734BFA2EBC7426D
:10DC4000B2EBC74261EB57310CFB0EF7B0EBC700EC
:10DC500072EB57720CFB08F734BFA2EBC702B2EBB2
:10DC6000C70261EB5771039F4FEA816141EA92114C
:10DC700004EBCC044FEAD1374FEA826206FB07FC83
:10DC800042EA90124FEA80604FEA1C4C0CFB0BF703
:10DC9000D21B03FB0CF761EB07010CFB0EF7B0EB9B
:10DCA000074072EB17420CFB08F734BFA2EB0742A8
:10DCB000B2EB074261EB17414FEA8C554FEA9107EF
:10DCC00004EB9C2406FB07FC4FEA1C4C0CFB0BF7F7
:10DCD000B0EBC74072EB573203FB0CF734BFA2EB3B
:10DCE000C742B2EBC74261EB57310CFB0EF7B0EB0A
:10DCF000C70072EB57720CFB08F734BFA2EBC702E8
:10DD0000B2EBC70261EB577115EB4C254FEA81610D
:10DD100041EA92114FEA82624FEAD13742EA901209
:10DD200006FB07FC44F100044FEA80604FEA1C4CFC
:10DD30000CFB0BF7D21B03FB0CF761EB07010CFB91
:10DD40000EF7B0EB074072EB17420CFB08F734BF3D
:10DD5000A2EB0742B2EB074261EB174115EB1C1532
:10DD60004FEA813141EA92414FEA823242EA9042DF
:10DD70004FEA80304FEA0C7644F1000448EA03434E
:10DD80004EEA0B484FF0000EB2EB080C71EB0307A4
:10DD900024BF624639464EEB0E0E4FF0000B0018C2
:10DDA000524149414BEB0B0BB2EB080C71EB0307F3
:10DDB0007BF1000B24BF624639464EEB0E0E4FF04E
:10DDC000000B0018524149414BEB0B0BB2EB080C16
:10DDD00071EB03077BF1000B24BF624639464EEB23
:10DDE0000E0E51EA020718BF46F0010616EB0E763A
:10DDF00055F1000254F1000103D5BDE88901BDE8E9
:10DE00000088BDE88901BDE80048B619524141EBE0
:10DE10000101A3F10103704780807F7E7D7C7B7AC6
:10DE20007978777676757473727171706F6E6E6DC6
:10DE30006C6C6B6A6A69686867666665646463636C
:10DE400062616160605F5F5E5E5D5D5C5C5B5B5AF2
:10DE50005A5959585857575656555555545453535F
:10DE600052525251515050504F4F4F4E4E4D4D4DBA
:10DE70004C4C4C4B4B4B4A4A4A4949494848484705
:10DE80004747474646464545454444444443434343
:10DE90004342424242414141002B9C4630D47700EC
:10DEA0002BD01CB54FEA370703B44FF010004FF0EA
:10DEB0001001BAF1000F06D0BCF1000FDCBF40F03A
:10DEC000080040F008014FF000000FBCBDE8104012
:10DED0000BF1010BBBF1010F08BF5FEA170722BF6F
:10DEE00012F1010211F101014FF0004143F1000371
:10DEF00000F0004043EA00007047F9D35708D0E72C
:10DF000046EA064613F1400F4FEA16461FDD13F1AD
:10DF1000200FDFBF16430A46002120335B42BED0EC
:10DF2000C3F1200746EA064602FA07F74FEA16460B
:10DF300046EA0706C3F1200722FA03F201FA07F7BF
:10DF400021FA03F14FF0000342EA0702A7E746EA8D
:10DF5000020646EA06464FEA164646EA0106BCBFF6
:10DF600046EA0646360C4FF000034FF000024FF031
:10DF7000000194E72DE9804C9A46934670B491E8ED
:10DF8000380007C831EA400C48BF34EA430C03D5D7
:10DF9000FFF7E6FDFFF780FFF0BCBDE8008C2DE940
:10DFA000804C9A46934670B491E8380007C810F048
:10DFB000804F08BF13F0804F03D100F005F8FFF742
:10DFC0006BFFF0BCBDE8008C20F07F4780EA0300C7
:10DFD00023F07F4C07EB0C03A3F57C5300F00040CB
:10DFE000A3F1FE0392F0000F00F0B38095F0000F54
:10DFF00000F077802DE901494FEA11404FEA1446BD
:10E0000021EA004800FB06FC24EA064708FB06F666
:10E0100007FB08F800FB07F718EB06484CEB164C1B
:10E020004FEA124B18EB07484FEA15464CEB1740E6
:10E0300022EA0B4E0BFB06FC25EA06470EFB06F612
:10E0400007FB0EFE0BFB07F71EEB064E4CEB164CC8
:10E050004FF000061EEB074E4CEB174B18EB0B086E
:10E0600040F1000018EB0E0B58EB000840F10000E7
:10E070008F1A4FF000013CBFC943661B14BFB5EBBC
:10E08000040C00213CBFC943F61B4FEA17444EEA7B
:10E090008E0E27EA04454FEA1C4704FB07622CEA70
:10E0A000074C05FB07F70CFB05F604FB0CFC16EB15
:10E0B000074642EB174216EB0C4642EB1C421BEBA9
:10E0C000060658EB0202414146EA9E0601D5BDE82C
:10E0D0000189B619524141EB0101A3F10103BDE8E9
:10E0E00001894FEA14454FEA114724EA054621EA1F
:10E0F000074C05FB07F406FB07F70CFB06F105FBD5
:10E100000CFC11EB074144EB17444FEA124711EBAB
:10E110000C4144EB1C4422EA074C05FB07F206FBCA
:10E1200007F70CFB06F605FB0CFC16EB074642EB6B
:10E13000174216EB0C4642EB1C456A1854F10001DD
:10E1400048BF7047B619524141EB0101A3F10103E9
:10E15000704795F0000F37D04FEA11424FEA14474D
:10E1600021EA024624EA074C02FB07F106FB07F707
:10E170000CFB06F402FB0CFC14EB074441EB1741CB
:10E180004FEA154714EB0C4441EB1C4125EA074CC0
:10E1900002FB07F506FB07F70CFB06F602FB0CFC7F
:10E1A00016EB074645EB174516EB0C4645EB1C42B4
:10E1B000121951F1000148BF7047B619524141EBA5
:10E1C0000101A3F1010370474FEA14454FEA1147DB
:10E1D00024EA054621EA074C05FB07F106FB07F791
:10E1E0000CFB06F24FF0000605FB0CFC12EB07429D
:10E1F00041EB174112EB0C4251EB1C4148BF7047F9
:10E20000921841EB0101A3F101037047002904D0EA
:10E21000816841F0010181607047816821F001014E
:10E220008160704710B5154988420AD14415012113
:10E23000204604F053FB2046BDE81040002104F0C6
:10E240004DBB0F4988420AD104150121204604F034
:10E2500045FB2046BDE81040002104F03FBB0949C2
:10E2600088420AD10121CC03204604F037FB204626
:10E27000BDE81040002104F031BB10BD0024014076
:10E2800000280140003C0140014600208968490700
:10E2900000D501207047014600208968090700D594
:10E2A0000120704710B542680E4B1A400C790B687C
:10E2B00042EA04221343436082680B4B1A40D1E9BF
:10E2C000024323434C7942EA440213438360C26A07
:10E2D00022F47002097C491EC9B242EA0151C162AE
:10E2E00010BD0000FFFEF0FFFDF7F1FF816841F077
:10E2F000080181607047816841F0040181607047C6
:10E300000649002804D0086840F4000008607047FF
:10E31000086820F4000008607047000008240140ED
:10E3200002460021082001F04DBD70B505460E469D
:10E33000284600F039FA2846FFF7F2FF0446032C7E
:10E3400003D13146284604F0D9F9204670BD0000BB
:10E350000FB4F8B507AD00954FF40074204608F0EF
:10E360000DFF064611A221463046FEF75BF8044633
:10E37000C4F5007130192B46069AFEF717F80028ED
:10E3800006DD204482B23146002007F043FA07E060
:10E39000502208A10EA0FEF723F811A0FEF720F8E6
:10E3A000304608F0E7FEF8BC5DF814FB4C6F67419F
:10E3B00070703A002E2E5C53595354454D5C53599E
:10E3C00053504F52545C737973706F72742E6300A4
:10E3D0004C6F674572723A2025732C25640000004B
:10E3E0000000000010B506F0B5FF03280FD10C485F
:10E3F00006F09AFF04460A49032C09D04A8A491CB0
:10E4000008A002F019F8C8200BF048F8204610BD0B
:10E410004A8A491C0AA0FFF79BFF204610BD000056
:10E42000AA01002054435020536572766572C1AC36
:10E43000BDD3CAA7B0DC3A25733A256420A3A10056
:10E4400054435020536572766572C1ACBDD3B3C9D5
:10E45000B9A63A25733A256420A3A10010B501207E
:10E4600004F04AFABDE81040002004F045BA00006C
:10E4700008B50349084400900098008808BD0000D2
:10E48000006C004008B5034A1044009000980160F9
:10E4900008BD0000006C004001490C204870704726
:10E4A0005C00002010220A21042002F053BC0A2143
:10E4B000042003F03DB8000010B506F07BF903F02E
:10E4C000CFF8002003F0B4F90F2004F01DFD04F094
:10E4D00079F80D49022005F00BF907F01FFD03F054
:10E4E000B1F8FFF7DFFF06F047FA03F0D3FC4FF473
:10E4F000E134204604F0A4FA204604F0B7FABDE85F
:10E50000104004F037B8000079360408FEE730B553
:10E5100000231AE0CD5C2C0905F00F053034392CAE
:10E5200003D9E41D00F8134001E000F81340303532
:10E53000ECB2392C04D900EB4305E41D6C7002E009
:10E5400000EB43056C705B1C9BB29342E2D330BD81
:10E55000810701D0002070476421B0FBF1F201FB7C
:10E56000120109B1012070474FF4C871B0FBF1F2FC
:10E5700001FB120008B100207047012070470246DD
:10E580000021012001F0D8BC2DE9F04105460F46DD
:10E59000032640F2492008F0F1FD04463B464FF4C3
:10E5A00000773AA2394604F12600FDF73BFF002828
:10E5B00001DDB8420BDD40F2A72235A139A001F000
:10E5C0003BFF204608F0D6FD0220BDE8F08128225E
:10E5D0002270642190FBF1F23032A27090FBF1F2D4
:10E5E00001FB12020A2192FBF1F23032E27090FB41
:10E5F000F1F201FB1200303020713149087860716E
:10E60000401CC0B20870392801D93020087004229B
:10E610002CA1A01DFEF73AFB012104F10A0002F033
:10E62000ABFA3B2184F82210B5F82310A4F823108C
:10E63000262184F82510687843280ED07221617055
:10E64000032222A12046FEF776F92046FFF780FE3E
:10E65000204608F08FFD3046B7E752216170032253
:10E660001AA12046FEF767F92046FEF7D1F982B2DB
:10E670002146174802F054FE0028E9D040F2C1229A
:10E6800003A114A001F0D8FEE2E70000257300000A
:10E6900055534552434D445C75736572636D642EEA
:10E6A0006300000025732C25643A75704461746121
:10E6B000427566207370696C6C6F766572A3A100F9
:10E6C000480000204D41433A000000002458290032
:10E6D0004E0C002025732C25643A7354637030511E
:10E6E00075657565207370696C6C6F766572A3A132
:10E6F0000000000010B5044694F8240030381128BA
:10E7000035D2DFE800F0090D1115191D2125292D3D
:10E710003434343434343100204604F0B7FE27E07A
:10E72000204602F0CFF923E0204602F0C9FC1FE0AA
:10E73000204605F051F81BE0204601F04FFF17E09E
:10E74000204602F0D3F813E0204602F04BF80FE029
:10E75000204601F0C7FF0BE0204606F0EDFA07E087
:10E76000204606F069FB03E007F008FC00E04E20BD
:10E770000C49502809D049280DD04E2811D149689C
:10E780002046BDE81040FFF7FFBE89682046BDE87F
:10E790001040FFF7F9BEC9682046BDE81040FFF7FA
:10E7A000F3BE10BD480000200246002101A307204F
:10E7B00001F008BB434D494F5400000070B50446BA
:10E7C000084611461D46049EFEF7ABF8024601209E
:10E7D00006E0231803F8011CB04204D8401C80B2A4
:10E7E000115CA942F5D170BD30B5054600205B1E15
:10E7F00004E02C54984204DA401C80B20C5C944231
:10E80000F7D130BD10B5022000F0C2FB012805D1C0
:10E81000022000F0D9FA022000F0E8FD082000F004
:10E82000B7FB01280FD1082000F0CEFAD52206A1AF
:10E830000AA0FDF7D5FD0DA0FDF7D2FDBDE8104003
:10E84000082000F0D3BD10BD2E2E5C535953544503
:10E850004D5C444D415C646D612E63004C6F6745B7
:10E8600072723A2025732C2564000000444D41311A
:10E870005F5445312100000010B5202000F088FBD6
:10E88000012805D1202000F09FFA202000F0AEFDE5
:10E89000802000F07DFB01280FD1802000F094FA49
:10E8A000EB2206A10AA0FDF79BFD0DA0FDF798FD48
:10E8B000BDE81040802000F099BD10BD2E2E5C53A5
:10E8C000595354454D5C444D415C646D612E630069
:10E8D0004C6F674572723A2025732C256400000046
:10E8E000444D41315F5445322100000010B54FF4D2
:10E8F0000074204600F04CFB012805D1204600F0B2
:10E9000063FA204600F072FD4FF40064204600F0E8
:10E910003FFB012810D1204600F056FA40F20112C8
:10E9200006A10BA0FDF75CFD0DA0FDF759FD2046EB
:10E93000BDE8104000F05ABD10BD00002E2E5C5303
:10E94000595354454D5C444D415C646D612E6300E8
:10E950004C6F674572723A2025732C2564000000C5
:10E96000444D41315F5445332100000010B54FF450
:10E970000054204600F00CFB012805D1204600F091
:10E9800023FA204600F032FD4FF40044204600F008
:10E99000FFFA012810D1204600F016FA40F21712B3
:10E9A00006A10BA0FDF71CFD0DA0FDF719FD2046EB
:10E9B000BDE8104000F01ABD10BD00002E2E5C53C3
:10E9C000595354454D5C444D415C646D612E630068
:10E9D0004C6F674572723A2025732C256400000045
:10E9E000444D41315F5445342100000010B54FF4CF
:10E9F0000034204600F0CCFA012805D1204600F072
:10EA0000E3F9204600F0F2FC4FF40024204600F029
:10EA1000BFFA012810D1204600F0D6F940F22D129D
:10EA200006A10BA0FDF7DCFC0DA0FDF7D9FC2046EC
:10EA3000BDE8104000F0DABC10BD00002E2E5C5383
:10EA4000595354454D5C444D415C646D612E6300E7
:10EA50004C6F674572723A2025732C2564000000C4
:10EA6000444D41315F5445352100000010B54FF44D
:10EA70000014204600F08CFA012805D1204600F051
:10EA8000A3F9204600F0B2FC4FF40004204600F049
:10EA90007FFA012810D1204600F096F940F2431287
:10EAA00006A10BA0FDF79CFC0DA0FDF799FC2046EC
:10EAB000BDE8104000F09ABC10BD00002E2E5C5343
:10EAC000595354454D5C444D415C646D612E630067
:10EAD0004C6F674572723A2025732C256400000044
:10EAE000444D41315F5445362100000010B54FF0D0
:10EAF0000074204600F04CFA012805D1204600F0B1
:10EB000063F9204600F072FC4FF00064204600F0EC
:10EB10003FFA012810D1204600F056F940F2591270
:10EB200006A10BA0FDF75CFC0DA0FDF759FC2046EB
:10EB3000BDE8104000F05ABC10BD00002E2E5C5302
:10EB4000595354454D5C444D415C646D612E6300E6
:10EB50004C6F674572723A2025732C2564000000C3
:10EB6000444D41315F5445372100000010B5124C2F
:10EB7000204600F00DFA012805D1204600F024F9C6
:10EB8000204600F033FC0C4CA41D204600F000FA97
:10EB9000012810D1204600F017F940F26F1207A1AA
:10EBA0000BA0FDF71DFC0EA0FDF71AFC2046BDE8EA
:10EBB000104000F01BBC10BD020000102E2E5C5354
:10EBC000595354454D5C444D415C646D612E630066
:10EBD0004C6F674572723A2025732C256400000043
:10EBE000444D41325F5445322100000010B5124CB3
:10EBF000204600F0CDF9012805D1204600F0E4F8C8
:10EC0000204600F0F3FB0C4C6034204600F0C0F9C5
:10EC1000012810D1204600F0D7F840F2851207A154
:10EC20000BA0FDF7DDFB0EA0FDF7DAFB2046BDE8EB
:10EC3000104000F0DBBB10BD200000102E2E5C53F6
:10EC4000595354454D5C444D415C646D612E6300E5
:10EC50004C6F674572723A2025732C2564000000C2
:10EC6000444D41325F5445322100000010B5124C32
:10EC7000204600F08DF9012805D1204600F0A4F8C7
:10EC8000204600F0B3FB0D4C204600F081F901282E
:10EC900010D1204600F098F840F29B1208A10DA078
:10ECA000FDF79EFB0FA0FDF79BFB2046BDE8104043
:10ECB00000F09CBB10BD0000000200100008001016
:10ECC0002E2E5C53595354454D5C444D415C646D4C
:10ECD000612E63004C6F674572723A2025732C25B4
:10ECE00064000000444D41325F5445332100000070
:10ECF00010B5224C204600F04BF9012805D12046E2
:10ED000000F062F8204600F071FB1D4C204600F038
:10ED10003FF901280ED1204600F056F840F2B1121A
:10ED200018A11DA0FDF75CFB1FA0FDF759FB2046B5
:10ED300000F05CFB1F4C204600F02AF9012805D1A9
:10ED4000204600F041F8204600F050FB1A4C2046C7
:10ED500000F01EF9012810D1204600F035F84FF4DC
:10ED6000DF7208A10CA0FDF73BFB14A0FDF738FBF8
:10ED70002046BDE8104000F039BB10BD0020001057
:10ED8000008000102E2E5C53595354454D5C444D69
:10ED9000415C646D612E63004C6F674572723A206E
:10EDA00025732C2564000000444D41325F544534E6
:10EDB000210000000000021000000810444D413204
:10EDC0005F54453521000000C10002D502490860AA
:10EDD0007047024948607047040402400000024046
:10EDE000002904D0016841F0010101607047016809
:10EDF0004FF6FE7211400160704700002DE9F047A8
:10EE00008CB00446DDE914980D4617469A46072C47
:10EE100004D20121084603F037FD03E0012102205E
:10EE200003F032FD184E56F8240000F031F8019539
:10EE30000297CDF80CA0002504950595802006903A
:10EE400007950895CDF8249040010A900B9556F847
:10EE5000240001A900F0B8F80C4810F824008DF83F
:10EE600000008DF801808DF8025001208DF803001C
:10EE7000684602F067FD56F824000122022100F0E6
:10EE800099F80CB0BDE8F087C805002058C5040803
:10EE900001684FF6FE72114001600021016041607F
:10EEA0008160C1603649364A0839904204D14868C9
:10EEB00040F00F0048607047314A1432904204D14C
:10EEC000486840F0F000486070472D4A2832904270
:10EED00004D1486840F4706048607047284A3C326A
:10EEE000904204D1486840F4704048607047244A1A
:10EEF0005032904204D1486840F470204860704716
:10EF00001F4A6432904204D1486840F4700048605F
:10EF100070471B4A7832904204D1486840F07060D4
:10EF200048607047174A111F904204D1086840F0AA
:10EF30000F0008607047134A1432904204D10868E9
:10EF400040F0F000086070470E4A2832904204D129
:10EF5000086840F47060086070470A4A3C3290428A
:10EF600004D1086840F4704008607047054A503288
:10EF70009042FAD1086840F47020086070470000A1
:10EF80000800024008040240406880B27047000058
:10EF900002460020D10002D50449096801E0044975
:10EFA0000968114200D001207047000000040240AF
:10EFB00000000240002A03D002680A430260704742
:10EFC00002688A430260704730B5026847F6F07302
:10EFD0009A430C6A8B682343D1E904452C432343AD
:10EFE0008C692343CC6923434C6A23438C6A2343B3
:10EFF00013430360CA6842600A6882604968C1605E
:10F0000030BD416070470921042002F091BA0246E8
:10F010000021092000F0D6BE0FB4F8B507AD009569
:10F020004FF40074204608F0A9F8064611A22146C4
:10F030003046FDF7F7F90446C4F5007130192B4648
:10F04000069AFDF7B3F9002806DD204482B2314666
:10F05000002006F0DFFB07E06E2208A10EA0FDF7FE
:10F06000BFF911A0FDF7BCF9304608F083F8F8BCF1
:10F070005DF814FB4C6F674465623A002E2E5C53BA
:10F08000595354454D5C535953504F52545C737906
:10F0900073706F72742E63004C6F674572723A2002
:10F0A00025732C256400000000000000704700005C
:10F0B00070B504460AF0FAFF01280CD0094D6888A3
:10F0C000844203D3B4FBF0F00AF0E8F96888B4FB9B
:10F0D000F0F100FB11444FF47A706043BDE87040DA
:10F0E00000F002B82006002070B5054611488542A0
:10F0F00008D90546612210A116A0FDF771F919A0E3
:10F10000FDF76EF900214FF0E0267469164800788B
:10F110004543B369B2699A42FCD003D2A3EB020023
:10F12000014403E0A4EB0200184401441346A94241
:10F13000F0D370BDE3388E032E2E5C5359535445E3
:10F140004D5C5359535449434B5C737973746963F1
:10F150006B2E63004C6F674572723A2025732C2525
:10F1600064000000000000002006002070B5054685
:10F170000C467B2003F024FC012804D122461EA16A
:10F180002846FDF783FD7C2003F01AFC012804D1FA
:10F1900022461CA12846FDF779FD7D2003F010FCD6
:10F1A000012804D122461AA12846FDF76FFD7E20D2
:10F1B00003F006FC012804D1224619A12846FDF7D8
:10F1C00065FD7C2003F0FCFB88B97D2003F0F8FB93
:10F1D00068B97E2003F0F4FB48B97A2003F0F0FB15
:10F1E000012804D1224612A12846FDF74FFDBDE8B3
:10F1F000704003F087BB0000D6D8C9CFB5E7C6F48E
:10F20000B6AF0000C8EDB8B4CEBBC6F4B6AF0000D0
:10F21000B6C0C1A2BFB4C3C5B9B7C6F4B6AF00008B
:10F22000B4B0BFDABFB4C3C5B9B7C6F4B6AF000057
:10F23000D3B2B8B4CEBBC6F4B6AF00001CB504461A
:10F240001021002200910CA31146402002F0F0FE94
:10F250000C490022CDE9002110232022002140206A
:10F2600002F0EEFD0C2100220091234611465A20A7
:10F2700002F0DEFE1CBD00002020202020202020E7
:10F280000000000054B304081CB5044610210022FD
:10F2900000910CA31146104602F0CAFE0C49002250
:10F2A000CDE90021002110232022084602F0C8FDEC
:10F2B0000C2100220091234611461A2002F0B8FECC
:10F2C0001CBD000020202020202020200000000065
:10F2D00014B3040808B504A00023009003220C21F5
:10F2E000184602F061FF08BD4D454E5520202020F4
:10F2F0002020202020202020204241434B000000DD
:10F3000038B50C4C2078C1074FF010000AD000909F
:10F3100009A300220221382002F08AFE2068401C46
:10F32000206038BD009005A300220221382002F0A1
:10F330007FFEF3E7A40100203A0000002000000057
:10F3400010B5102007F01AFF04460E4B0EA2102134
:10F350002046FDF767F82046FFF770FF1021204692
:10F36000FDF74BFC074B0AA25B1D10212046FDF761
:10F3700059F82046FFF788FF2046BDE8104007F007
:10F38000F9BE0000911C002025736D56000000009E
:10F39000435351257300000038B51E2007F0EEFEE0
:10F3A0000446052210492046FDF770FC0122002387
:10F3B00010211046009402F0F7FE1E212046FDF7B2
:10F3C0001CFC09490A220B392046FDF75FFC00238B
:10F3D00002220C210120009402F0E6FE2046BDE846
:10F3E000384007F0C7BE0000EF5B002030B46A4928
:10F3F000B0F1007F01F1300271D036DCB0F5005F72
:10F400006ED018DC80287AD00ADC02286DD008285B
:10F4100070D0202868D14868002865D030BC0047EB
:10F42000B0F5007F71D0B0F5006F5DD19068002815
:10F430005AD030BC0047B0F5002F77D00ADCB0F5C9
:10F44000004F6ED0B0F5003F4ED1086900284BD078
:10F4500030BC0047B0F5001F6DD0B0F5000F43D1B0
:10F460005069002840D030BC00474C4C031BA042E0
:10F470007CD01ADC4A4CA0EB0403A0426CD00BDC1D
:10F48000B0F1006F61D0A0F18050801E2CD1C8690E
:10F4900000287FD030BC0047182B62D0782B79D160
:10F4A000106A002876D030BC0047B3F5FC4F67D017
:10F4B0000ADCB3F5C06F5ED0B3F5F05F6AD1886A3D
:10F4C000002867D030BC0047B3F5FF3F5DD035481A
:10F4D000C3425FD1D06A00285CD030BC00472FE027
:10F4E00018E00CE001E005E054E00868002851D085
:10F4F00030BC0047106800284CD030BC0047506832
:10F50000002847D030BC0047FFE78868002841D07A
:10F5100030BC0047C86800283CD030BC004705E03C
:10F52000FFE7D068002835D030BC004710690028BC
:10F5300030D030BC0047486900282BD030BC004791
:10F540008869002826D030BC00479069002821D067
:10F5500030BC00470AE0FFE7D06900281AD030BC71
:10F560000047086A002815D030BC0047486A0028C8
:10F5700010D030BC0047506A00280BD030BC004788
:10F58000906A002806D030BC0047C86A002801D025
:10F5900030BC004730BC7047445B002000020010C4
:10F5A000080000100002F8FF10B5144600290BD027
:10F5B000012919D04E2215A119A0FCF711FF1CA09A
:10F5C000FCF70EFF204610BD224951F8202042B121
:10F5D00043220EA112A0FCF703FF1FA0FCF700FFBF
:10F5E000F0E741F82040EDE71A49303151F820208A
:10F5F00042B14A2205A10AA0FCF7F2FE1DA0FCF7C9
:10F60000EFFEDFE741F82040DCE700002E2E5C53E0
:10F61000595354454D5C444D415C646D612E63000B
:10F620004C6F674572723A2025732C2564000000E8
:10F63000446D6154652043616C6C6261636B202290
:10F64000654972715479706522206572726F7221FA
:10F6500000000000445B0020446D6154632043615E
:10F660006C6C6261636B2072657065617420726599
:10F6700067210000446D6154652043616C6C6261D8
:10F68000636B20726570656174207265672100008C
:10F6900010B50021084600F0C9FA0446032C02D038
:10F6A00005A000F0C9FE4FF47A70FFF701FD00F0ED
:10F6B000FBF8204610BD00004543323020C8EDB9AC
:10F6C000D8BBFACAA7B0DCA3ACBCB4BDABB6CFB54F
:10F6D000E7B9D8BBFAA3A10010B50021022000F0C1
:10F6E000A5FA032809D00021032000F09FFA002189
:10F6F000BDE81040022000F099BA10BD10B51022EC
:10F700000F21042001F026FB00F0CEF810220B217F
:10F71000042001F01FFB02490020086010BD00001A
:10F72000AC0123420021012000F080BA70B500F046
:10F7300089FCFFF7E3FF00F0C3F9FFF7F3FFFFF7E2
:10F74000CBFF0446094800F07BF9084A142108A0C1
:10F75000FEF7FEFD05481530054600F08DF92946F7
:10F7600008A0FEF7F5FD204670BD00007C1C0020BF
:10F770004543323020C8EDBCFEB0E6B1BEA3BA2589
:10F780002E2A73004543323020B9A9B5E7B5E7D139
:10F79000B9A3BA2573206D56000000002DE9F04191
:10F7A00005460E461F48044600F02EF903280AD0ED
:10F7B0001DA231462846FCF735FE1EA000F03CFE97
:10F7C0000220BDE8F081224619211EA0FEF7C0FDEF
:10F7D00000F07AF80446032C09D01FA231462846CF
:10F7E000FCF720FE1FA000F027FE0220E9E700F052
:10F7F00099F800F0E3F8014620A0FEF7A9FD0948BA
:10F80000001F074600F0BEF83B4620A231462846BE
:10F81000FCF708FE3A4603211FA0FEF799FD20469B
:10F82000CFE700009A1C0020C7EBB2E5C8EB5349B4
:10F830004DBFA800CEB4BCECB2E2B5BD53494DBF3C
:10F84000A800000053696DBFA84943434944A3BAC7
:10F85000252E2A730000000053494DBFA8C7B7B733
:10F86000D100000053494DC7B7B7D1CEDEB7A8D7F6
:10F87000A2B2E1C9CFCDF8C2E7000000CDF8C2E7DF
:10F88000D0C5CFA2A3BA257300000000D0C5BAC569
:10F89000D6CAC1BF3A2573004C544520435351A3E7
:10F8A000BA252E2A7300000003490020086040F6A4
:10F8B000B830FFF7FDBB0000BC0123420149012025
:10F8C00008607047BC0123422DE9F04104252D2436
:10F8D0000021012000F076FA104F114E4FF4FA6823
:10F8E00015E04046FFF7E4FB0021022000F06AFA31
:10F8F0000546032D0BD1B86C002807DDB86C805D80
:10F90000312807D0B86C805D352803D00225641EED
:10F91000601CE6D12846BDE8F08100009C02002072
:10F92000BD1C00202DE9F04104251E2400210320E8
:10F9300000F048FA114F124E4FF4FA6818E04046B2
:10F94000FFF7B6FB0021042000F03CFA0546032D2A
:10F950000ED1D7F88000002809DDD7F88000805D3F
:10F96000312808D0D7F88000805D352803D00225E3
:10F97000641E601CE3D12846BDE8F0819C02002093
:10F98000BE1C002070B5054600202860002106201E
:10F9900000F018FA0446032C09D10648D0F8B81034
:10F9A0000548192301442C222846FEF71DFF204656
:10F9B00070BD00009C020020BA1C002010B5002180
:10F9C000052000F0FFF9032801D008A010BD0C4C61
:10F9D00020680C4908440D21FCF7A3FF00210170A9
:10F9E000216808480A30084410BD0000BBF1C8A1D6
:10F9F000CDF8C2E7D0C5CFA2CAA7B0DC2100000075
:10FA000038030020B41C002070B505461921284693
:10FA1000FDF7F3F80021084600F0D4F90446032C62
:10FA200008D1054801690548192301440D222846DB
:10FA3000FEF7DAFE204670BD9C020020BC1C0020B0
:10FA400070B5054615212846FDF7D7F80021052099
:10FA500000F0ECF80446032C09D10D210548FCF711
:10FA600060FF811C14230D222846FEF7BDFE2046B0
:10FA700070BD0000B41C002070B50446002020605A
:10FA800020710021062000F0D1F80546032D05D095
:10FA900008A12046FCF78DFF284670BD2C210748A1
:10FAA000FCF7ABFF411C04230D222046FEF79CFE11
:10FAB000F2E700003335303000000000B41C0020B5
:10FAC00070B500240425FFF7F9FE00F0E3FB4FF4C6
:10FAD0007A7610E0641CE4B23046FFF7E9FA08A138
:10FAE000084806F0FBFD002805DB214606A0FFF7CD
:10FAF00093FA032501E0142CECD3284670BD0000D6
:10FB000052445900B41C00204543323020537461E4
:10FB10007274205761697465643A2564205300004B
:10FB20000FB42DE9F84F81464FF004082F48C9EB78
:10FB3000C90100EB8104667E60680B904FF49675F6
:10FB4000284607F01BFB82460CAB00932946504623
:10FB50000B9AFCF72BFC0746002F01DDAF422EDD90
:10FB600023A000F069FC2DE000F094FB0025BAB260
:10FB70005146022005F04EFE16E03220FFF798FABB
:10FB8000E168274806F0AAFD20612069002802DB11
:10FB90004FF0030816E06169214806F09FFD002838
:10FBA00002DB4FF002080DE028466D1C2189EDB202
:10FBB000B0EB410FE1D34FF47A70FFF779FA761E7C
:10FBC000F6B2D1D2504607F0D5FA404603F0CCFE4B
:10FBD0000446484601F016F90146224611A0FFF7F7
:10FBE0001BFA4046BDE8F80F5DF814FB5C040020EA
:10FBF0004874747020636D645061636B20D2E7B306
:10FC0000F6A3A12D2DD4F6BCD3485454505F434DD8
:10FC1000445041434B5F4C454ECAFDD6B5A1A300AD
:10FC2000B41C002025732025730000000FB42DE9BB
:10FC3000F84F82464FF004083F48CAEBCA0100EB78
:10FC40008104667E60680B904FF4A165284607F03A
:10FC500095FA83460CAB0093294658460B9AFCF75D
:10FC6000A5FB07464FF00009002F01DDAF423EDD46
:10FC7000B62232A13AA000F0DFFB584607F07AFA2C
:10FC80000220BDE8F80F5DF814FB00F003FB00252F
:10FC9000BAB25946022005F0BDFD16E06420FFF718
:10FCA00007FAE168354806F019FD2061206900284F
:10FCB00002DB4FF003081DE06169304806F00EFDDD
:10FCC000002802DB4FF0020814E028466D1C218951
:10FCD000EDB28842E2D3607E801B00EBC00101EBF5
:10FCE00000104FF4FA7101EB8000FFF7E1F9761E86
:10FCF000F6B2CAD2584607F03DFACDF80090B8F1F6
:10FD0000050F0ED2DFE808F0030507090B001CA45D
:10FD100008E01EA406E020A404E021A402E022A43E
:10FD200000E023A4504601F0E9FC0146224623A04E
:10FD3000FFF772F94046A4E7D80100202E2E5C4858
:10FD4000415244574152455C4C54455C4543323026
:10FD50005C656332306D6F64756C652E6300000006
:10FD600025732C25643A636D645061636B20737056
:10FD7000696C6C6F766572A3A1000000B41C002052
:10FD8000496E506172616D45727200004F7574501A
:10FD90006172616D4572720052554E4552520000BB
:10FDA00052554E4F4B00000054494D454F5554009D
:10FDB000CEB4D6AAB4EDCEF3000000002573202502
:10FDC000730000000FB42DE9F84F8146042738482E
:10FDD000C9EBC90100EB8104667E60680B9080204E
:10FDE00007F0CCF982460CAB0093802150460B9A69
:10FDF000FCF7DCFA8046B8F1000F02DDB8F1800FA5
:10FE00002FDD65222BA133A000F016FB02272BE08B
:10FE100000F040FA00251FFA88F25146022005F052
:10FE2000F9FC14E06420FFF743F9E168304806F07C
:10FE300055FC20612069002801DB032714E061697B
:10FE40002B4806F04BFC002801DB02270CE028467B
:10FE50006D1C2189EDB28842E4D34FF47A70FFF72C
:10FE600027F9761EF6B2D3D2504607F083F9002068
:10FE70000090052F0ED2DFE807F0030507090B00FD
:10FE80001CA408E01EA406E020A404E021A402E0D3
:10FE900022A400E023A4484601F09AFD0146224630
:10FEA00023A0FFF7B9F83846BDE8F80F5DF814FB5A
:10FEB0009C0200202E2E5C48415244574152455C22
:10FEC0004C54455C454332305C656332306E65743A
:10FED0002E63000025732C25643A636D64506163C2
:10FEE0006B207370696C6C6F766572A3A100000063
:10FEF000B41C0020496E506172616D457272000041
:10FF00004F7574506172616D4572720052554E4565
:10FF10005252000052554E4F4B00000054494D457F
:10FF20004F555400CEB4D6AAB4EDCEF30000000075
:10FF300025732025730000000FB42DE9F84F81468A
:10FF40004FF004082F48C9EBC90100EB8104667E1D
:10FF500060680B90802007F011F982460CAB00938B
:10FF6000802150460B9AFCF721FA0746002F01DD4D
:10FF7000802F2FDD24A000F05FFA4FF002082CE064
:10FF800000F088F90025BAB25146022005F042FC83
:10FF900016E06420FFF78CF8E168274806F09EFB26
:10FFA00020612069002802DB4FF0030815E0616939
:10FFB000214806F093FB002802DB4FF002080CE01A
:10FFC00028466D1C2189EDB28842E2D34FF47A7045
:10FFD000FFF76EF8761EF6B2D2D2504607F0CAF896
:10FFE000404603F08FFC0446484604F001FD0146FC
:10FFF000224612A0FFF710F84046BDE8F80F5DF862
:020000040804EE
:1000000014FB0000D003002054637020636D645023
:1000100061636B20D2E7B3F6A3A12D2DD4F6BCD338
:100020005443505F434D445041434B5F4C454ECA8F
:10003000FDD6B5A1A3000000B41C00202573202527
:100040007300000010B501230C224FF4E1310220AF
:1000500005F00EFB00F01EF900F024F9054801F050
:1000600055F9054801F052F9BDE810400349022056
:1000700005F02CBE341F00203A230020B5020408EE
:1000800010B5012000F0AAF828B1012000F09AF87C
:10009000012001F0F9F9BDE81040012000F098B806
:1000A00030B591B00A240E4D55F8240000F0A0F8A8
:1000B00088B155F8240000F085F8402101A8FCF72C
:1000C000BEFD234607A2402101A8FCF7ABF955F875
:1000D000240001F0D9F9641C0F2CE5DD11B030BD0E
:1000E000DCC5040845585449256420495251210073
:1000F00010B5022000F072F8012805D1022000F0AE
:1001000061F8022001F0C0F9BDE81040022000F0C3
:100110005FB810B5042000F061F828B1042000F0A9
:1001200051F8042001F0B0F9BDE81040042000F0BF
:100130004FB810B5082000F051F8012805D108206B
:1001400000F040F8082001F09FF9BDE810400820B9
:1001500000F03EB810B5102000F040F828B1102093
:1001600000F030F8102001F08FF9BDE810401020A9
:1001700000F02EB830B591B005240E4D55F824008E
:1001800000F036F888B155F8240000F01BF8402143
:1001900001A8FCF754FD234607A2402101A8FCF763
:1001A00041F955F8240001F06FF9641C092CE5DDD4
:1001B00011B030BDDCC504084558544925642049B8
:1001C00052512100014908607047000014040140A9
:1001D00001490860704700001404014001460020F6
:1001E000024A12680A4200D00120704714040140FC
:1001F00001460020054A12680A40044B14331B686C
:100200000B4202D0002A00D00120704700040140B8
:1002100030B51B4A83790168002B2AD013688B43C1
:100220001360111D0B680468A3430B60017911442E
:100230000B68046823430B60114C08342168036881
:1002400099432160231D19680568A9431960417904
:10025000102905D011440A68006802430A6030BDC5
:100260002168026811432160196800680143196020
:1002700030BD0079104402688A43026030BD00003E
:10028000000401400021016001710C224271817162
:10029000704700004FF4A0710148FCF7AEBC0000AD
:1002A000B41C00204FF4A0710148FCF7A6BC00006C
:1002B000F41D002070B505460C462848007800283B
:1002C00006D022462946BDE870402548FCF733BBDE
:1002D00024A1284606F002FA002821DB23A12846A3
:1002E00006F0FCF900280DDB22462946234801F0E0
:1002F00017F8002830D0BDE87040712220A129A055
:1003000000F09AB8224629462D4801F009F8002845
:1003100022D0BDE87040782219A12AA000F08CB844
:100320002F48FCF775FBC0F5A070A04205D92946FF
:10033000BDE870402A48FCF7D5BB842210A129A053
:1003400000F07AF8FFF7A6FF2946BDE870404FF4A9
:10035000A0722348FCF79ABC70BD0000D4010020B5
:10036000F41D00202B51495552433A002B51495559
:1003700052433A202272656376220000341F002027
:100380002E2E5C48415244574152455C4C54455CCA
:10039000454332305C656332306D6F64756C652E39
:1003A0006300000025732C25643A73546370517503
:1003B000657565207370696C6C6F766572A3A100BA
:1003C0003A23002025732C25643A735572635175C6
:1003D000657565207370696C6C6F766572A3A1009A
:1003E000B41C002025732C25643A656332304174B7
:1003F000427566207370696C6C6F7665722E200092
:1004000070B500F0CFF80024094D05EBC42000F0D2
:1004100063F8641CE4B2002CF7D006480021416068
:10042000C16002F06DFFBDE8704000F099B80000B7
:1004300000F80708681C00200FB4F8B507AD009558
:100440004FF40074204606F099FE064611A221469C
:100450003046FBF7E7FF0446C4F5007130192B4620
:10046000069AFBF7A3FF002806DD204482B231463E
:10047000002005F0CFF907E08B2208A10EA0FBF7C2
:10048000AFFF11A0FBF7ACFF304606F073FEF8BCDF
:100490005DF814FB4C6F674572723A002E2E5C5368
:1004A000595354454D5C535953504F52545C7379D2
:1004B00073706F72742E63004C6F674572723A20CE
:1004C00025732C2564000000000000000149C8606D
:1004D000704700000020024070B505464FF43026FA
:1004E000304600F06BF8042811D1094C206940F027
:1004F000020020616561206940F0400020613046C3
:1005000000F05CF8216941F6FD721140216170BD77
:100510000020024004200849CA68D20701D0012007
:100520007047CA68520701D502207047C968C906DA
:10053000FBD5032070470000002002400146002048
:10054000064A012904D0D2680A4200D0012070472F
:10055000D169C907FBD0012070470000002002408C
:100560000248016941F080010161704700200240AA
:10057000F0B506460D464FF40057384600F01EF819
:1005800004280CD1064C206940F001002061358020
:10059000384600F013F82169BA1E11402161F0BD00
:1005A000002002400348024941600349416070470E
:1005B0002301674500200240AB89EFCD00B503461B
:1005C000FFF7A8FF02E0FFF7A5FF5B1E012801D19E
:1005D000002BF8D1002B00D1052000BD2DE9F047FC
:1005E00007463C46A0782179303800EBC00202EB88
:1005F000001001EB8001E0786FF02F02303800EB43
:10060000800002EB40000D18DFF8A4A0F822274973
:10061000504602F04CFE4FF48076304606F0AEFDB8
:100620008046224B23A21033994631464046FBF7C1
:10063000F9FE064694F82300312804D1611991F897
:100640002610242902D030281DD021E04021484620
:10065000FCF7D3FA2A4604F126014846FCF716FBBC
:10066000F8221249504605F033FDC6F5807108EBBB
:1006700006004B4615A2FBF7D5FE532441463846EB
:10068000FDF782FF05E0601990F82600242806D0C7
:100690004924404606F06EFD2046BDE8F08753240D
:1006A00041463846FDF770FFF3E70000560B002087
:1006B000008801082A4745542A20467470466F6C0A
:1006C0006465723A5B25735D210000002A5345542E
:1006D0002A20467470466F6C6465723A5B25735DC0
:1006E000210000002DE9F04707463C46A07821791B
:1006F000303800EBC00202EB001001EB8001E07823
:100700006FF02F02303800EB800002EB40000D1834
:10071000DFF8A4A0F8222749504602F0C8FD4FF4A4
:100720008076304606F02AFD8046224B23A2D03345
:10073000994631464046FBF775FE064694F823007D
:10074000312804D1611991F82610242902D03028CB
:100750001DD021E010214846FCF74FFA2A4604F14B
:1007600026014846FCF792FAF8221249504605F055
:10077000AFFCC6F5807108EB06004B4614A2FBF7F0
:1007800051FE532441463846FDF7FEFE05E0601950
:1007900090F82600242806D04924404606F0EAFCBA
:1007A0002046BDE8F087532441463846FDF7ECFE6D
:1007B000F3E70000560B0020008801082A47455443
:1007C0002A2046747049503A5B25735D2100000071
:1007D0002A5345542A2046747049503A5B25735D6C
:1007E000210000002DE9F04707463C46A07821791A
:1007F000303800EBC00202EB001001EB8001E07822
:100800006FF02F02303800EB800002EB40000D1833
:10081000DFF8A4A0F8222749504602F048FD4FF423
:100820008076304606F0AAFC8046224B23A2903305
:10083000994631464046FBF7F5FD064694F82300FD
:10084000312804D1611991F82610242902D03028CA
:100850001DD021E040214846FCF7CFF92A4604F19B
:1008600026014846FCF712FAF8221249504605F0D4
:100870002FFCC6F5807108EB06004B4615A2FBF76E
:10088000D1FD532441463846FDF77EFE05E0601950
:1008900090F82600242806D04924404606F06AFC39
:1008A0002046BDE8F087532441463846FDF76CFEEC
:1008B000F3E70000560B0020008801082A47455442
:1008C0002A2046747050617373776F72643A5B25A7
:1008D000735D21002A5345542A2046747050617379
:1008E00073776F72643A5B25735D21002DE9F047E1
:1008F00007463C46A0782179303800EBC00202EB75
:10090000001001EB8001E0786FF02F02303800EB2F
:10091000800002EB40000D18DFF8A4A0F822274960
:10092000504602F0C4FC4FF48076304606F026FCB8
:100930008046224B23A25033994631464046FBF76E
:1009400071FD064694F82300312804D1611991F80D
:100950002610242902D030281DD021E0402148460D
:10096000FCF74BF92A4604F126014846FCF78EF9BC
:10097000F8221249504605F0ABFBC6F5807108EB32
:1009800006004B4615A2FBF74DFD53244146384661
:10099000FDF7FAFD05E0601990F82600242806D03E
:1009A0004924404606F0E6FB2046BDE8F087532484
:1009B00041463846FDF7E8FDF3E70000560B0020FE
:1009C000008801082A4745542A20467470557365EB
:1009D000726E616D653A5B25735D21002A53455443
:1009E0002A20467470557365726E616D653A5B2599
:1009F000735D210010B58A07120F0F23934021F079
:100A00000304054921448C689C438C608B689040AA
:100A100003438B6010BD0000000001402DE9F04150
:100A20000022CC7804F00F03E40601D58C78234330
:100A30000C784FF00F0714F0FF0F4FF0010C1CD093
:100A400005680CFA02F40E882640A64211D19600E1
:100A500007FA06F825EA080503FA06F848EA050544
:100A6000CE78282E02D0482E02D002E0446100E069
:100A70000461521C082AE4D305600A88FF2A1ED9A3
:100A80004568002202F108060CFA06F40E8826409A
:100A9000A64210D1960007FA06F825EA080503FADF
:100AA00006F848EA0505CE78282E00D14461CE78B4
:100AB000482E00D10461521C082AE3D34560BDE8EA
:100AC000F0810000F0B58DB00446F8222349244897
:100AD00002F0EDFB23A104F1260005F0FFFD18B1A3
:100AE00049240DB02046F0BD4FF40076304606F0A4
:100AF00045FB07461D48054601F0F0FD1748F0305C
:100B0000A0F12002A0F1E003CDE90932A0F110012B
:100B1000CDE90B10164A6038A2F10903CDE9053280
:100B20009039CDE90710111FA0F18C029038C378DD
:100B3000CDE90225019304918178009143780D4A13
:100B400031463846FBF76EFC39462046FDF71CFD62
:100B50005324384606F00EFBC3E70000560B002076
:100B6000008801084745545F494150002C07002088
:100B70009A1C0020A0C804080EB50F4A1268009203
:100B80000D4A121D126801920B4A08321268029235
:100B900000290BD0012904D00C226946FDF7B7FCCF
:100BA0000EBD0C226946FDF7B2FC0EBD0C22694653
:100BB000FCF76CF80EBD0000E8F7FF1F27484278ED
:100BC000011D0D2A48D2DFE802F0474747174727A3
:100BD000372F471F47070F00027802EB420201EB55
:100BE0008202527802702EE0027802EB420201EBA0
:100BF00082029278027026E0027802EB420201EB58
:100C00008202D27802701EE0027802EB420201EB0F
:100C100082021279027016E0027802EB420201EBC6
:100C20008202527902700EE0027802EB420201EB7E
:100C300082029279027006E0027802EB420201EB36
:100C40008202D279027000224270007800EB4000EC
:100C500001EB800080680047704700005C000020C6
:100C600070B58388002B08D003889B1CC3F309034D
:100C7000038000231380831D21E0022070BD1488AF
:100C8000641C14800488E45C01F8014B0488641C33
:100C9000C4F30904048014888588AC4203D2048814
:100CA000B4F5806F0BD300F031FB662210A117A0C2
:100CB000FBF796FB19A0FBF793FB022070BD04889D
:100CC000E45C562CDBD10488641CC4F3090404449E
:100CD000A479782CD3D10188891CC1F30901018042
:100CE00081881288891A091F8180002070BD000048
:100CF0002E2E5C53595354454D5C5359534C494225
:100D00005C7379736C69622E630000004C6F6745F9
:100D100072723A2025732C25640000000000000048
:100D200000220280827001460322014802F0BFBA0D
:100D30000090010810B5F821FBF75FFFBDE81040F7
:100D4000F8220249024802F0B2BA0000560B002015
:100D500000880108F8B504460D4616460B480121E7
:100D600050F8240001F0ACFD08481C3030F81500A4
:100D7000ADF800008DF8036003208DF802000448F0
:100D8000694650F82400FFF749FEF8BD90C50408F5
:100D9000F8050020162204A10DA0FBF721FB10A0EE
:100DA000FBF71EFBFEE700002E2E5C53544D333242
:100DB000463130785F46574C69625C7372635C738E
:100DC000746D3332663130785F69742E63000000D1
:100DD0004C6F674572723A2025732C256400000021
:100DE000486172644661756C745F48616E646C65DD
:100DF0007221000010B5FEF7CFFABDE81040FEF7F3
:100E000069BA0000092818D2DFE800F00507090BCD
:100E10000D0F111315000AA070470CA070470EA00B
:100E2000704710A0704712A0704714A0704715A01B
:100E3000704717A0704719A070471BA070470000AB
:100E400048545450434F4E5445535400454E524518
:100E50005148454144455200434C4F534554494D38
:100E600045000000424F44595459504500000000CD
:100E700053455455524C434D44000000485454507F
:100E800055524C00504F5354524551434D4400006D
:100E9000504F535452455142554600004854545007
:100EA0005245414400000000CEDEB4CBC3FCC1EE8D
:100EB00000000000002808D0A0F50070BD3807D061
:100EC000012808D005A0FDF743BA0AA0FDF740BAF3
:100ED0000FA0FDF73DBA14A0FDF73ABA485454509C
:100EE000285329206F74686572206572726F722EA4
:100EF0000000000048747470204F7065726174695E
:100F00006F6E207375636365737366756C2E000076
:100F10004854545028532920756E6B6E6F776E209D
:100F20006572726F722E0000485454502853292065
:100F300074696D656F75742E0000000010B5002196
:100F40000846FEF7EDFD03280AD100210120FEF737
:100F5000E7FD032804D1BDE810400021FEF7E0BD05
:100F600010BD10B50424FFF7E9FF032801D0204687
:100F700010BDBDE8104000F001B8000070B51020B1
:100F800006F0FCF805462946022001F0B7FB0328CD
:100F900007D029460220FDF7C8F90446032C02D0E9
:100FA00005E0032070BD294603A0FDF7D1F92846CE
:100FB00006F0E0F8204670BD48545450B1BEB5D894
:100FC0004950A3BA257300002DE9F04100240426FE
:100FD000FFF768F9304F01203870304DD5F8E40044
:100FE000FBF716FDD5F8E41082B2022004F012FCE3
:100FF00039E06420FEF75CF855F8EC1F284805F04E
:101000006DFB68606868EC3D002823DBD5F8F010C4
:1010100023480C30085C302819D055F8F01F2048C0
:101020002A68401C095C6420303941431C48801CFC
:10103000105C2A68303800EB800001EB4001184852
:10104000C01C105C08440226FFF734FF12E00020A9
:101050000326F9E7D5F8F410124805F03FFB002805
:1010600001DB022606E02046641CB5F8E810E4B275
:101070008842BED300203870304602F075FC04462A
:101080000820FFF7BFFE0146224607A0FDF7C4FF78
:101090003046BDE8F0810000D40100205C0400204F
:1010A000F41D0020B41C00202573202573000000CF
:1010B00002494AF6AA20086070470000003000404C
:1010C0002DE9F04707463C46DFF8A890F82228496A
:1010D000484602F0ECF84FF48075284606F04EF8CA
:1010E0000646DFF88C8024A2294698F80130304665
:1010F000FBF798F9054694F82300312804D124A180
:10110000A01C05F0EBFA20B194F8230030281DD084
:1011100021E094F82600302803D0312801D0502453
:101120001AE088F80100F8221149484604F0D0FF7F
:1011300098F80130C5F58071701916A2FBF772F9A5
:10114000532431463846FDF71FFA05E010A1A01CD4
:1011500005F0C4FA30B14924304606F00BF82046B9
:10116000BDE8F087532431463846FDF70DFAF3E722
:10117000560B0020008801082A4745542A2049615F
:1011800070466C61673A5B25635D212000000000BA
:10119000303031002A5345542A20496170466C6131
:1011A000673A5B25635D210010B504462046FFF7D2
:1011B000B7FD2046BDE8104002F01EBD002140F8FA
:1011C000191F41608160C1600161416119381921B5
:1011D000FBF713BD7CB504463E4800F097F8204667
:1011E000FFF7A8FD5B202070302060703220A070D7
:1011F0003120E070207CFF2809D104F1100040214B
:101200000546FBF7FAFC34A12846FBF7D2FB94F81D
:101210005000FF2809D104F1500040210546FBF79A
:10122000ECFC2FA12846FBF7C4FB94F89000FF28A4
:1012300009D104F1900040210546FBF7DEFC29A10D
:101240002846FBF7B6FB94F8D000FF2809D104F13B
:10125000D00010210546FBF7D0FC26A12846FBF75D
:10126000A8FB94F8E000FF2816D0A8B1254926482D
:1012700002F000FC94F8F000FF2818D0B8B1214922
:101280002148103102F003FC5D2084F8F70020466D
:10129000BDE87C4002F0B8BC04F1E0001021054636
:1012A000FBF7ABFC13A12846FBF783FBE2E700202A
:1012B000C4F8F000A4F8F400009001900A226946F6
:1012C00041F6583005F0DCF9694604F1F000FBF70F
:1012D00070FBD9E7500700202F41424D000000006D
:1012E00041424D0053686F703334343739343734EA
:1012F000390000003132312E34312E37392E383753
:1013000000000000360C0020AA010020002101800E
:10131000418081804FF48061801DFBF76EBC00002E
:101320002DE9F0418388161D33444FF48067BB429A
:1013300002D30120BDE8F08145881223841D2B557E
:1013400043885B1CC3F309034380458834232B5532
:1013500043885B1CC3F30903438000230BE011F8AF
:10136000015BB0F802C00CF8045045886D1CC5F351
:10137000090545805B1C9342F1DB428856211155DB
:101380004188491CC1F309014180428878211155E7
:101390004188491CC1F30901418081883144818021
:1013A0008188B94209D3FFF7B1FF432204A10BA002
:1013B000FBF716F80DA0FBF713F80020BAE70000C2
:1013C0002E2E5C53595354454D5C5359534C49424E
:1013D0005C7379736C69622E630000004C6F674523
:1013E00072723A2025732C25640000000000000072
:1013F0002DE9FE430646DDF828900C461546984632
:101400002A4621463046FFF7A5FC282D01D0482D5D
:1014100035D10121084601F053FA1A4F385D8DF895
:1014200000008DF8019000258DF802508DF80350D2
:10143000684600F087FAA7F15000015D4438805DEE
:10144000FFF7D8FAA7F1400656F8240001908DF86E
:1014500008508DF8098001258DF80A5001A8FEF783
:10146000D7FE56F82400FEF7B3FE385700F01F01F0
:101470008D404009800000F1E020C0F80051BDE837
:10148000FE8300001CC6040870B5064600204FF01D
:10149000804105F083F904460D46304609F05EFBB5
:1014A00005F07CF922462B4609F07EF909F010FB85
:1014B000044951F82000002802D0BDE870400047E0
:1014C00070BD0000A45B002010B50C46084A52F81D
:1014D0002030002B09D0972206A10BA0FAF780FF3D
:1014E0000DA0FAF77DFF204610BD42F82040FAE734
:1014F000A45B00202E2E5C53595354454D5C494F3C
:101500005C696F2E630000004C6F674572723A2071
:1015100025732C2564000000494F2043616C6C62E8
:1015200061636B207265706561742072656721006C
:10153000044A52F82000C268034B33F811104A40A5
:10154000C2607047F8050020ACC5040801490920B5
:10155000487070475C00002038B506240C234822F0
:10156000194600200094FFF743FF082348220B216F
:1015700000200094FFF73CFF0823482209210220A5
:101580000094FFF735FF082348220721022000942A
:10159000FFF72EFF08234822062102200094FFF7C0
:1015A00027FF082348220F2103200094FFF720FF84
:1015B000082348220D2103200094FFF719FF482239
:1015C0000B210320FFF7C6FB482208210020FFF76C
:1015D000C1FB482209210220FFF7BCFB4822082159
:1015E0000220FFF7B7FB48220E210320FFF7B2FBD2
:1015F000BDE8384048220C210320FFF7ABBB0000B8
:1016000001490520487070475C0000200149062010
:10161000487070475C0000200149072048707047FF
:101620005C00002001490320487070475C000020E6
:1016300004F0A6FCFDF7E7FCFCF739FF642007F097
:101640002DFFF5E7102209210420FFF783BB0000DE
:10165000024C204607F022FFFBE70000A0860100B5
:1016600070B514221149124801F021FE0F4C4FF0C1
:10167000503000252268011182420FD122698A422E
:101680000CD121890BA0FCF763FE1448616801F0BE
:10169000DDFD2581BDE8704001F032BE2060216192
:1016A0002581BDE87040FEF7ABBE0000681C00203D
:1016B00000F00708B1BEB5D8C8D5D6BEB4E6B4A20E
:1016C000D2E7B3F6A3BA2564B4CE202E0D0AB1BE7C
:1016D000B5D8C8D5D6BE3A200000000000F80708EB
:1016E000FEE7FFF76BFA142007F0D8FEF9E70000D9
:1016F00001490B20487070475C000020072813D276
:10170000DFE800F00406080A0C0E100007A070477E
:1017100008A070470AA070470CA070470EA0704741
:1017200010A0704712A0704715A070475455524E34
:101730004F46460048414E445348414B4500000047
:101740005155455259434F4E46494700434C4F531C
:101750004545434F0000000053415645434F4E4618
:1017600049470000515545525952454C4553450093
:101770005155455259564F4C5441474500000000C1
:10178000CEDEB4CBC3FCC1EE00000000002906D0C1
:10179000034A02EB80029268891A00F015B870477C
:1017A0005805002010B50446204600F05FF8411CA3
:1017B00005D0044901EB84018968084410BD00206C
:1017C00010BD00005805002070B5134A13181B7E89
:1017D000002B12D0114B53F820308B421AD90F4BEB
:1017E000083B53F82030B1FBF3F102EB80021069A3
:1017F00030F811300020002408E0116888470120EB
:1018000070BD15690E1825F81640401C9842F8DB8B
:10181000002070BD022070BD5805002014C50408CA
:1018200001E000F8011B521E531CFAD17047000062
:1018300070B504460B480C4E002150F8240006EB0E
:10184000840542002869FFF7EBFF064800211030AD
:1018500050F82420A868FFF7E3FF0120311908762B
:1018600070BD000004C50408580500202DE9F041B2
:1018700005460F460024DFF8888008EB0500007E4F
:10188000002803D1D8F80010284688474FF0FF32CF
:10189000FFB11C4E56F82500B7FBF0F3B7FBF0F193
:1018A00000FB117000B15B1C1648083850F8251079
:1018B000491E002921DB08EB8507386930F811C083
:1018C000BCF1000F08D000249C4213D1002298B232
:1018D0000AE01046BDE8F081641CF5E73C6901EBC5
:1018E000020C24F81C00521C9A42F7D356F825002B
:1018F0004843EFE7491E0029E0DA1046EAE7000016
:10190000580500200CC5040810B5002200210A4B20
:101910000A4C53F8203004EB800005E0046934F8E9
:10192000114004B1521C491C8B42F7D86420424339
:10193000B2FBF3F0C0B210BD04C504085805002086
:101940007047000070B50F23C27801260178002A85
:101950001ED0144A126802F4E062C2F5E062120A74
:10196000C2F10404D3404578A54082781A402A4346
:10197000120101F1E02181F80024007800F01F013C
:101980008E404009800000F1E020C0F8006170BD89
:1019900001F01F0086404809800000F1E020C0F8F7
:1019A000806170BD0CED00E0024908430249086007
:1019B000704700000000FA050CED00E0024A1140FB
:1019C000014302480160704780FFFF1F08ED00E0FF
:1019D00010B50B281DD2DFE800F006080A0C0E1027
:1019E000121416181A000DA010BD0FA010BD10A0E3
:1019F00010BD11A010BD12A010BD13A010BD16A0E7
:101A000010BD18A010BD1AA010BD1CA010BD1FA0B5
:101A100010BD22A0FEF710FD26A010BD5155455265
:101A2000594943434944000053455443530000007F
:101A300051554552594353005345545053000000EB
:101A4000515545525950530051554552594E4554E0
:101A5000494E464F000000005155455259435351DD
:101A600000000000434F46434F4E54455854000079
:101A7000414354434F4E544558540000444541435C
:101A800054434F4E544558540000000051554552A0
:101A900059434F4E544558540000000045433230DE
:101AA00020CEDED0A7654E6574436D644E756D2102
:101AB00000000000CEDEB4CBC3FCC1EE000000008D
:101AC00008B50026894D8A4C4FF4FA78894F00E119
:101AD0002E70FBE02878401CC1B22970022904D97D
:101AE00085A004F04FFA02F0B1FEAF2288A141F2C6
:101AF000707000F0BDFA0021206807F0C9FEC043F5
:101B0000C0070CD084A002F0ADF9FDF70FFE03284A
:101B10000DD083A004F036FA85A0FCF719FC002153
:101B2000206807F0B5FEC043C00708D02AE00121B5
:101B3000206807F0EFFE81A0FCF70AFCEFE7002128
:101B4000206807F0A5FEC04380071BD57EA002F0E9
:101B500089F91E2005F012FB81461E214846FDF73B
:101B60001DFE032816D0484604F00CFA0F21206809
:101B700007F08EFEFDF78CFD4846FCF7E9FB484672
:101B800005F0F8FA0021206807F082FEC043C00784
:101B900005D023E00221206807F0BCFEECE700211D
:101BA000206807F075FEC043800717D40021206825
:101BB00007F06EFEC043400710D565A002F052F951
:101BC000FCF710FC032811D00421206807F060FE08
:101BD00063A0FCF7BDFB65A004F0D4F900212068E8
:101BE00007F056FEC043C0070CD027E00421206850
:101BF00007F090FE61A14C2003F0F2FA65A0FCF71B
:101C0000A7FBEBE70021206807F042FEC0438007F6
:101C100014D40021206807F03BFEC04300070DD517
:101C2000FFF79FF9032811D00821206807F030FE44
:101C30005BA0FCF78DFB5EA004F0A4F900212068F6
:101C400007F026FEC04300071CD025E008212068CD
:101C500007F060FE5AA002F005F901F061FB814631
:101C600059A14C2003F0BCFAB9F1030F04D05BA0DA
:101C700004F088F902F0EAFD62A0FCF769FB01F0CC
:101C80001FFBDBE76348FDF77DFE6248401FFDF761
:101C9000F3FEFDF755FB2E705F4800231A461946E8
:101CA000006808F04DF819215C48FAF7A6FF4FF4D8
:101CB0008470009016A35AA219215848FAF7B2FB73
:101CC0005648FCF745FB5AA0FCF742FB404607F09C
:101CD000E5FB0121386807F01DFE0021206807F0B0
:101CE000D7FDC04300077FF4F5AEF1E60000002009
:101CF0003C00002040000020CFB5CDB3CDF8C2E7B6
:101D0000B1C0C0A3A3ACD6D8C6F4CFB5CDB3210023
:101D10006D61696E2E630000CED5CAD6D6D03A006A
:101D2000C4A3BFE9B0B2D7B0D2ECB3A32100000086
:101D3000CED5CAD6CAA7B0DC00000000CED5CAD620
:101D4000B3C9B9A600000000C8EBCDF8D6D03A0060
:101D5000C1ACBDD3544350B7FECEF1C6F73A000034
:101D6000544350C1ACBDD3CAA7B0DC00544350C1EA
:101D7000ACBDD3CAA7B0DC21000000004465766981
:101D800063652074637020636F6E6E657463656451
:101D900021000000544350C1ACBDD3B3C9B9A60063
:101DA00048545450B3F5CABCBBAFCAA7B0DC00005E
:101DB00048545450B3F5CABCBBAFCAA7B0DC21002D
:101DC000D7A2B2E1D6D03A00446576696365205265
:101DD000656769737465722100000000487474704F
:101DE000B3F5CABCBBAF4F4BA3ACD7A2B2E1C7EBB4
:101DF000C7F3CAA7B0DCA3ACD6D8C6F4CFB5CDB371
:101E000021000000D3B2BCFED7A2B2E1B3C9B9A68B
:101E1000A3A10000961C002044000020E206002040
:101E2000257320256420CACDB7C545433230210033
:101E3000CACDB7C545433230D7CAD4B4210000005B
:101E40002DE9F04F8146DDE909BA0E460025580715
:101E500005D0012000EBD30702EB090815E0DF08ED
:101E6000FAE73146484600F0A1FA4C4609E0284618
:101E70006D1C1AF800005A46012100F00DFB641C8D
:101E8000E4B2A045F3D8761CF6B2BE42E9D3BDE871
:101E9000F08F000038B5102204210020FEF75AFF11
:101EA000102205210020FEF755FF102206210020F8
:101EB000FEF750FF102207210020FEF74BFF1022F3
:101EC00005210220FEF746FF554C012525606420C0
:101ED000FDF7EEF8002020606420FDF7E9F82560AA
:101EE00000221146AE2000F0D7FA0022114602204F
:101EF00000F0D2FA00221146102000F0CDFA0022A4
:101F00001146402000F0C8FA00221146812000F05E
:101F1000C3FA00221146FF2000F0BEFA002211464B
:101F2000A12000F0B9FA00221146C82000F0B4FA4E
:101F300000221146A62000F0AFFA00221146A82088
:101F400000F0AAFA002211463F2000F0A5FA002274
:101F50001146D32000F0A0FA00221146104600F0EE
:101F60009BFA00221146D52000F096FA0022114675
:101F7000802000F091FA00221146D92000F08CFA5E
:101F800000221146F12000F087FA00221146DA20E3
:101F900000F082FA00221146122000F07DFA0022A1
:101FA0001146DB2000F078FA00221146402000F0B4
:101FB00073FA00221146202000F06EFA002211462A
:101FC000022000F069FA002211468D2000F064FA28
:101FD00000221146142000F05FFA00221146A420CE
:101FE00000F05AFA00221146A62000F055FA00220D
:101FF0001146AF2000F050FA00221146AF2000F049
:102000004BFA00F099F80021084600F0CFF905A03E
:10201000002300901A461021012000F0C5F838BDB9
:1020200094012242EACC20B3CF20BFC620BCBC0022
:102030002DE9F8430446DDF820800E4691461F4600
:10204000002510E000904B4642463146204600F005
:10205000C7F904EB5800C4B2782C02D90024761CCE
:10206000F6B26D1CEDB2785D0028EBD1BDE8F883C7
:10207000FEB50D46144602461B480023194600686B
:1020800007F038FD01281BD0C02005F077F8064680
:10209000CDE9015415480090A0F11E0314A2C021FF
:1020A0003046FAF7BFF9304603F06CFF3046FCF7D4
:1020B0004FF9304605F05EF8BDE8FE4002F0C6BBC1
:1020C0000A481E211E38FAF798FD08482B4616A22A
:1020D0001E211E380094FAF7A5F9BDE8FE4003481A
:1020E0001E38FCF735B9000044000020E20600204D
:1020F000C9CFB4CE3A25732C20C9CFB4CE3A2573BC
:102100002C20B5B1C7B0257320256420C7C0D5BC2D
:1021100045433230CAA7B0DCA3ACCFB5CDB3C8EDD0
:10212000D6D8C6F4A3A10000257320256420C7C01B
:10213000D5BC45433230210030B5002505F1B00053
:102140000022C0B2114600F0A7F900221146022079
:1021500000F0A2F900221146102000F09DF90024A1
:1021600000220121104600F097F9641CE4B2802C93
:10217000F6D36D1CEDB2082DE0D330BD08B51021AB
:1021800040060091010E002202A31046FFF750FF07
:1021900008BD0000202020202020202020202020FA
:1021A00020202020000000000FB42DE9FE4F0C4637
:1021B000934600254FEA54088020B0FBF8F64FEA1A
:1021C0004B07102C1BD0042002900DF14409CDF8D0
:1021D0000490701C04F0D2FF82464B46711C50469E
:1021E000109AFAF7E3F88146B1450BD90AEB0600DD
:1021F00010F8010C7F2805D9A6F1010905E041205E
:102200000290E2E7B14500D9B1460C98012802D00E
:1022100002280AD105E0A6EB0900400808FB00F5FA
:1022200003E0A6EB090008FB00F5B9F1000F7CDD27
:102230005846FFF7A3FF00268BE01AF806107F2907
:1022400009D80091F9B2E8B222460F9B00F0C8F815
:1022500005EB54057CE0002077E0102C02D00C2C1C
:1022600038D071E0C0EBC00202EB8203434A03EBBB
:10227000020898F82020914266D10AEB060298F8ED
:10228000213052789A425FD1F9B2E8B200F08EF86C
:102290004FF0000B07E018F80B0001210F9A00F037
:1022A000FBF80BF1010BA345F5D3781CC1B2E8B2E2
:1022B00000F07CF8A34607E018F80B0001210F9A04
:1022C00000F0EAF80BF1010BBBEB440FF4D325440B
:1022D000761C3DE000EBC00202EB4203274A6C3A59
:1022E00003EB020898F8182091422DD10AEB060260
:1022F00098F8193052789A4226D1F9B2E8B200F033
:1023000055F84FF0000B07E018F80B0001210F9A69
:1023100000F0C2F80BF1010BA345F5D3781CC1B254
:10232000E8B200F043F8A34608E016E018F80B0006
:1023300001210F9A00F0B0F80BF1010BBBEB440F39
:10234000F4D32544761C03E0401C029A904284D3C7
:10235000761C4E45FFF471AF08E007D0B12208A10A
:102360000DA0FAF73DF810A0FAF73AF85046BDE88C
:10237000FE0F5DF814EB04F0FDBE000007B4040886
:102380002E2E5C48415244574152455C4F4C4544C7
:102390005C6F6C65642E63004C6F674572723A2007
:1023A00025732C25640000000000000010B50446D1
:1023B000B031C8B20022114600F06EF8A41CC4F37C
:1023C0000310002240F01000114600F065F804F000
:1023D0000F000022BDE81040114600F05DB800007B
:1023E0002DE9F041804606980E461F46002420380D
:1023F000C5B2B8F17F0F02D9A046B61CF6B20C2ABE
:1024000006D0102A19D0BDE8F0411CA0FEF714B880
:10241000761CF1B24046FFF7C9FF1D4905EB4500A8
:1024200001EB40053A46285D012100F035F8641CB7
:10243000E4B2062CF6D3BDE8F08131464046FFF702
:10244000B5FF144800EB05153A46285D012100F060
:1024500023F8641CE4B2082CF6D3761CF1B2404693
:10246000FFF7A4FF002428193A46007A012100F062
:1024700013F8641CE4B2082CF5D3DCE74E6F20207F
:1024800043484152484947485F65202E00000000FC
:10249000EABC040812BF0408F0B503460025002674
:1024A0000127164C01290CD00022C4F89861C4F809
:1024B0009061C4F894613AB118060DD5C4F89C61D6
:1024C0000CE0C4F89871F2E7180602D5C4F89C71C4
:1024D00004E0C4F89C6101E0C4F89C71C4F89471F4
:1024E00004F024F85806030E6D1CEDB2082DE0D35D
:1024F000C4F89071C4F89871F0BD0000000021424A
:102500001CB50446CDE900230B46002122460846AF
:10251000FDF712FD03280DD107490B69074A303436
:102520009A5CA24205D10A690449891C515C302990
:1025300000D002201CBD0000D0030020BD1C0020E4
:102540004FF48030FDF744BE014908627047000037
:1025500000000E42014908617047000000000E4271
:10256000034A116821F0E001014311607047000047
:10257000007000403EB50121080700F093F90124E6
:102580008DF808408DF8094000258DF80A508DF827
:102590000B4002A8FFF7D6F96846FDF773FE20044A
:1025A00000908DF8045008208DF805008DF8064045
:1025B0006846FDF72DFEC020FFF7D2FF0120FFF790
:1025C000C9FF3EBD30B5A1B02448F9F709FF244842
:1025D000F9F706FF234C2448211D01F06AFA224B2B
:1025E0000B222533002121A0F9F7FAFE1E481930ED
:1025F000054600F073F829461B4801F04FFA2946BA
:102600001FA0F9F7EDFEA17821A03039F9F7E8FE17
:1026100001211548FEF7B0FA134A182121A0F9F755
:10262000DFFE11480B2131300446FCF79FFD2246A6
:102630000B2121A0F9F7D4FE0848F9F7D1FE80213B
:1026400001A8FAF7FCFA234620A2802101A8F9F795
:10265000E9FE01A803F096FC21B030BD0CC80408C7
:1026600050C80408560B0020130700200D0A426FC3
:102670006F74B0E6B1BE203A20252A2E2A730000DE
:102680000D0A41505020B0E6B1BE203A202573001B
:102690000D0A52756E4170704E756D3A2041505062
:1026A000256400000D0AC9E8B1B8B1E0BAC5203A06
:1026B00020252E2A730000000D0AD6D8C6F4D4AD0A
:1026C000D2F2203A20252E2A73000000D6D8C6F474
:1026D000D4ADD2F23A25732E000000000021016033
:1026E0004160018181720B2201A1FAF7CFBA00008B
:1026F0004A616E2032312032303231002DE9F04112
:1027000004460F46224600210A20FDF75BFB0646E1
:10271000032E20D1214D012C20D0022C25D0032CBA
:102720002AD01FA1214803F0D9FFC5F82801D5F808
:10273000280100280EDBD5F828111C483034083059
:10274000085CA04206D1D5F8281118480A30085C68
:10275000312818D002263046BDE8F08110A1134878
:1027600003F0BCFFC5F82801E1E711A10F4803F011
:10277000B5FFC5F82801DAE710A10C4803F0AEFF59
:10278000C5F82801D3E7D5F82811084810230F30E1
:10279000014422223846FCF727F8DCE79C0200209F
:1027A0002B51494143543A2031000000B41C002011
:1027B0002B51494143543A20320000002B514941EA
:1027C00043543A20330000007CB502460021022029
:1027D000FDF7B2FB0646032E2BD10020009001909E
:1027E000162004F0CBFC0446134DA96C1348085C7A
:1027F0002070A96C11481023093001442C22601C60
:10280000FBF7F2FF601CFAF703F9A96C14300B4ACE
:1028100005230A3A114401442C226846FBF7E4FFE1
:1028200021786B46621C06A0FCF7F6FB204604F0FC
:10283000A1FC30467CBD0000D0030020BE1C00205F
:10284000544350204368616E6E616CA3BA256320C7
:10285000A1A320B7FECEF1C6F74950A3BA2573A1B4
:10286000A320B7FECEF1C6F7B6CBBFDAA3BA257365
:1028700000000000034A516821F4404101435160C7
:102880007047000000100240054A002903D051693A
:1028900001435161704751698143516170470000A4
:1028A00000100240054A002903D0D1690143D161DB
:1028B0007047D1698143D161704700000010024028
:1028C000054A002903D091690143916170479169DC
:1028D000814391617047000000100240054A0029C1
:1028E00003D0D1680143D1607047D1688143D16082
:1028F0007047000000100240014908607047000066
:10290000400442420248416A41F08071416270478E
:102910000010024010B5264A516801F00C01254B09
:10292000002927D0042927D0082927D0036051681F
:1029300001F0F0010909204B5C5C0168E140416055
:10294000546804F4E064240A1C5D21FA04F48460F1
:10295000546804F46054E40A1B5DD940C1605268B5
:1029600002F44042920B144B1B1F9A5CB1FBF2F134
:10297000016110BD0360DAE70360D8E7516801F434
:102980007011536803F48033022404EB914133B196
:1029900053689B0307D5094B59430160C7E7074BB1
:1029A00059430160C3E7034B59430160BFE700008F
:1029B0000010024000127A002C06002000093D00A1
:1029C000034600205909094A01290AD002290AD0E0
:1029D000516A03F01F02012393400B4200D00120F3
:1029E00070471168F5E7116AF3E700000010024034
:1029F000084900220A7001F82029012805D004287E
:102A000002D1052081F820007047012081F82000C4
:102A10007047000020100240014908607047000024
:102A20008004424201490860704700003C04424271
:102A300002490A6A02430A6270470000001002401D
:102A400010B504460748FEF761FC05230C22214619
:102A5000042002F00DFEBDE810400349042003F0FD
:102A600035B900005A1400207135040810B5044629
:102A7000102200210320FEF76DF9094B00221A6095
:102A80000848FEF743FC05230C222146032002F0F0
:102A9000EFFDBDE810400449032003F017B9000022
:102AA0008081224260180020F535040810B502200C
:102AB00000F0C6F900280DD04FF40030FDF788FB78
:102AC000022000F0B5F800F0ADFBBDE81040022098
:102AD00000F0FEBD10BD00002DE9F05F002301787D
:102AE000C278303901EB4104C4EBC11102EBC104DF
:102AF00042786421303A4A438178303901EB8101D0
:102B000002EB4101214430398DB24179827930396B
:102B100001EB81046FF02F0101EB44042244D7B292
:102B2000027A447A303A02EB820201EB42022244FA
:102B3000D6B2C27A047B303A02EB820201EB420247
:102B4000224402F0FF08827BC47B303A02EB82020F
:102B500001EB4202224402F0FF09827C407C3038C3
:102B600000EB800001EB4000104400F0FF0AA5F2EA
:102B7000B270822802D30220BDE8F09F40F2B27406
:102B8000DFF89CB009E02046FBF7E2FC08B15B44AB
:102B900001E024480344641CA4B2AC42F3D37F1E7A
:102BA000FFB20024DFF880B010E01BF8040040F210
:102BB000A321484303EBC0132846FBF7C9FC18B117
:102BC000012C01D119480344641CA4B2BC42ECD3CB
:102BD000761E40F2A320464303EBC610C8EB481113
:102BE000C1EB082100EB0110C9EB091100EB8100DA
:102BF00000EB0A040120FFF7A7FC00F021F800F029
:102C000011FB204600F0F4FA00F00CFB00F020F875
:102C100000F008FB0020FFF797FC0320ACE7000062
:102C20000085E2018033E10138C6040880510100CB
:102C300002490A8882430A80704700000428004045
:102C40000248018841F010010180704704280040CB
:102C50000248018821F010010180704704280040DB
:102C60002DE9F04788B0044600F0E4FA00F0DEF801
:102C70000646DFF8AC81B6FBF8F36A480A270188FC
:102C8000994277D0038040F2B2754FF4B7794FF490
:102C9000B67A0FE02846FBF75BFC38B14B4502D310
:102CA000A3F5B77304E06D1CADB205E0A3F26D139C
:102CB0006D1CADB25345EDD80195BDF804104FF42D
:102CC0007A70B1FBF0F130312170BDF80410B1FB26
:102CD000F0F200FB12126421B2FBF1F230326270AA
:102CE000BDF80420B2FBF0F500FB1520B0FBF1F2BB
:102CF00001FB1200B0FBF7F03030A070BDF804000B
:102D0000B0FBF7F107FB11003030E0700025DFF871
:102D100018910DE0BDF80400FBF71AFC08B1012D75
:102D20007AD019F80500984204D81B1A6D1CADB270
:102D30001C2BEFD26D1C04955B1C03939DF81000B7
:102D4000B0FBF7F0303060719DF81000B0FBF7F188
:102D500007FB11003030A0719DF80C00B0FBF7F0BC
:102D6000303020729DF80C00B0FBF7F107FB11002A
:102D700030306072B6FBF8F008FB10604FF4616110
:102D8000B0FBF1F20792B0FBF1F201FB12033C221F
:102D9000B3FBF2F30693B0FBF1F301FB1300B0FBBE
:102DA000F2F102FB110005909DF81C00B0FBF7F05A
:102DB0003030E0729DF81C00B0FBF7F107FB11000A
:102DC000303020739DF81800B0FBF7F03030A0735E
:102DD0009DF81800B0FBF7F107FB11003030E073ED
:102DE0009DF81400B0FBF7F0303060749DF81400CB
:102DF000B0FBF7F107FB11003030A0749DF80C20F8
:102E00009DF81010BDF8040000F02AF8029008B0F8
:102E10000320BDE8F087FFE71D2B8BD31D3B85E723
:102E2000805101001406002038C6040803480088B9
:102E30000249091F098840EA014070471C280040E8
:102E400006490988C2B21140044A121F1288024280
:102E500002D009B1012070470020704704280040CB
:102E600030B56423B0FBF3F4E4B2B0FBF3F503FB3D
:102E70001500132C01D96430C0B200EB9003072475
:102E8000B3FBF4F504FB1533084D1A440D4415F853
:102E9000015C2A4492B2800703D1032901D2521E59
:102EA00092B2B2FBF4F004FB102030BD2CC6040833
:102EB00010B50120FFF7C4FF38B10120FFF7B8FEBD
:102EC00000F0B0F9012000F003FC0220FFF7B8FF8A
:102ED000002809D00220FFF7ABFE00F0A3F9BDE8FF
:102EE0001040022000F0F4BB10BD0000054A00298C
:102EF00003D01188014311807047118881431180EC
:102F000070470000002800402DE9F04107460024EA
:102F10004E48202181722D21C17101713A21017425
:102F2000417301214FF0C050FFF7BCFC012108465E
:102F3000FFF7C6FC0120FFF707FB0420FBF798FA18
:102F400045F25006B0425ED0FBF788FA0120FFF749
:102F50004FFDFFF775FE00F065F96FF07F4500E06B
:102F6000641C4120FFF72CFD08B9AC42F8D3DFF810
:102F7000E080444505D24FF48070FFF759FD0124ED
:102F80001AE000240120FFF747FD00E0641C6120E7
:102F9000FFF716FD08B9AC42F8D3444523D24FF4ED
:102FA0000070FFF745FDCA222AA12FA0F9F718FAF1
:102FB00031A0F9F715FA00240120FFF733FD00F0E6
:102FC00031F9DCB147F6FF7000F022F900F02AF980
:102FD00000F028F9FFF73CFE00F024F93146042008
:102FE000FBF750FA15E0CF221AA11FA0F9F7F8F964
:102FF00021A0F9F7F5F90220BDE8F08149F640403B
:1030000000F006F9E2E700F00DF901210846FFF7AC
:103010006DFF00F007F901210846FFF767FF00F098
:1030200001F901210220FFF761FF00F0FBF8002009
:10303000FFF78AFA384600F023F80448FFF710FE3D
:103040000E49012000F054FB0320D5E7E45B00208B
:10305000F0FFFF002E2E5C53595354454D5C5254E3
:10306000435C7274632E63004C6F674572723A2042
:1030700025732C256400000000000000CD370408F3
:1030800008B503218DF800108DF8010000208DF89F
:10309000020001208DF803006846FEF753FC08BDCE
:1030A0002DE9F05F00230178C278303901EB41044B
:1030B000C4EBC11102EBC10442786421303A4A43A7
:1030C0008178303901EB810102EB41012144303933
:1030D0008DB241798279303901EB81046FF02F0193
:1030E00001EB44042244D7B2027A447A303A02EB2C
:1030F000820201EB42022244D6B2C27A047B303A09
:1031000002EB820201EB4202224402F0FF08827BC2
:10311000C47B303A02EB820201EB4202224402F00D
:10312000FF09827C407C303800EB800001EB4000DE
:10313000104400F0FF0AA5F2B270822802D30220E8
:10314000BDE8F09F40F2B274DFF894B009E0204689
:10315000FBF7FEF908B15B4401E022480344641C1C
:10316000A4B2AC42F3D37F1EFFB20024DFF878B0E4
:1031700010E01BF8040040F2A321484303EBC01306
:103180002846FBF7E5F918B1012C01D11748034493
:10319000641CA4B2BC42ECD3761E40F2A32046438A
:1031A00003EBC610C8EB4811C1EB082100EB01107E
:1031B000C9EB091100EB810000EB0A040120FFF7C5
:1031C000C3F9FFF73DFD00F02DF8204600F018F898
:1031D00000F028F8FFF73CFD00F024F80320AFE7EB
:1031E0000085E2018033E10138C604088051010006
:1031F000024A010C1180111D0880704720280040F0
:10320000024A010C1180111D0880704718280040E7
:10321000034AC0F303411180111D0880FFF718BD58
:1032200008280040024801888906FCD57047000044
:10323000042800400448018821F008010180018829
:103240000907FCD570470000042800402DE9F04133
:1032500005460E464FF40067384603F08FFF804660
:10326000C6F3CF240BE03A464146284600F01FF84B
:103270003A464146002002F0CDFA05F50065641E8D
:10328000A4B2F0D239464046F9F7B7FCC6F30A04B7
:1032900022464146284600F00AF8224641460020D0
:1032A00002F0B8FA4046BDE8F04103F063BF03E026
:1032B00010F8013B01F8013B521E92B2F8D2704760
:1032C00010B50C480078002812D110220A490B488A
:1032D000F9F743FB40B1FCF75FF8BDE8104014225A
:1032E00005490648F9F7D2BCBDE81040FCF708B81C
:1032F00010BD00005C000020E45B002000070020FF
:1033000010B5054C2046FDF7E7F82046BDE8104013
:103310001422024902F0DCBE00F00708681C0020FD
:10332000F0B585B001213748FDF726FC03F02FF8F2
:103330000746344803F033F8024633A1384603F019
:1033400011F8384603F0B0F8044621462FA0FBF7E9
:1033500063FE2146324800F039FB0446032C0DD0B1
:1033600030480821006806F093FA2FA002F00AFE08
:10337000384603F022F805B02046F0BDFDF724FEE4
:103380000446032CF4D17B212B48F9F736FB03F0DC
:1033900055F8064630000FD028A103F035F8054651
:1033A00015B1E86804280FD0022427A0FDF744F8DF
:1033B000304603F002F8DBE703F020F8014627A0CF
:1033C000FAF7C6FF0224F3E7132228482969F9F720
:1033D0005DFC2648FFF764FE132224496846F9F78E
:1033E0008DFB9DF80900401C8DF8090020A0008885
:1033F000ADF80B006846FFF76FFB1EA02969FBF7CD
:103400000BFED5E7130700206D616300D3B2BCFE4D
:10341000D7A2B2E14A534F4EA3BA25730000000071
:10342000C00100203C0000204874747020706F734D
:1034300074206572722E0000F41D0020737973549D
:10344000696D6532000000004E6F20226A736F6E56
:103450005F74696D6522202E00000000636A736F3F
:103460006E206572723A257300000000E45B002054
:10347000303100002573CEAABBF1C8A1B5BDB5C4DB
:10348000B7FECEF1C6F7CAB1BCE42E0038B504468B
:103490001DA104F1260003F021F910B150252846A2
:1034A00038BD53251AA12046FBF76EF8C82005F059
:1034B000F5FF204C002341F288321946206806F0BF
:1034C00019FB012803D101F0CBFAFCF7E1F8002346
:1034D0001A461946206806F033FC19211648F9F7F8
:1034E0008CFB4FF48770009014A319A21921124885
:1034F000F8F798FF1048FAF72BFF19A002F042FDE9
:1035000001F0A4F9CBE70000434D445F525354004F
:103510002A5345542A205573657220636F6E747266
:103520006F6C20646576696365207265737461727F
:103530007421000044000020E2060020555345524B
:10354000434D445C75736572636D642E63000000C7
:10355000257320256420CACDB7C5454332302100EC
:10356000D6D8C6F4C3FCC1EEC8EDD6D8C6F4210047
:1035700010B50A4601460548FDF7D2FE002804D0E2
:10358000BDE8104002A0FCF757BF10BD5A14002040
:103590007352533233325175657565D2E7B3F6A372
:1035A000A100000008B500244FF4806509E0314611
:1035B0000AA0FAF7CDFE304603F0DCFD642005F0EA
:1035C0006DFF284603F0DAFD064600946A46314650
:1035D0000748FDF745FB0028EDD1E8E75273323389
:1035E0003220726563646174613A2573202E000095
:1035F0005A14002010B50A4601460548FDF790FE12
:10360000002804D0BDE8104002A0FCF715BF10BD93
:10361000601800207352533438355175657565D282
:10362000E7B3F6A3A100000008B500244FF48065BD
:1036300009E031460AA0FAF78BFE304603F09AFD06
:10364000642005F02BFF284603F098FD0646009401
:103650006A4631460748FDF703FB0028EDD1E8E74D
:10366000527334383520726563646174613A25732E
:10367000202E00006018002000B585B013220D49EF
:103680006846F9F73BFA9DF80900401C8DF80900DF
:1036900009A00088ADF80B006846FFF71DFA054841
:1036A00002F070FC05A002F06DFC01F0CFF805B04F
:1036B00000BD0000E45B0020303100005274635F05
:1036C000416C725F43616C6C6261636B210000004E
:1036D0000649012805D0022807D18868002804D0AF
:1036E00000474868002800D00047704714060020B3
:1036F00010B50C46144901280BD0022816D03D22E3
:1037000012A117A0F8F76CFE19A0F8F769FE204681
:1037100010BD486840B132220CA111A0F8F760FE3C
:103720001AA0F8F75DFEF2E74C60F0E7886840B158
:10373000392206A10AA0F8F753FE1CA0F8F750FEA4
:10374000E5E78C60E3E70000140600202E2E5C53B2
:10375000595354454D5C5254435C7274632E63005C
:103760004C6F674572723A2025732C256400000067
:103770005274635F526567486F6F6B43616C6C6234
:1037800061636B204661696C65642100527463203B
:1037900053656354692043616C6C6261636B207292
:1037A0006570656174207265672100005274632042
:1037B000416C7254692043616C6C6261636B20726E
:1037C0006570656174207265672100000148FFF72C
:1037D00047BA0000E45B00202DE9F84307463C4669
:1037E000DFF8BC90F8222D494846FFF760FD4FF402
:1037F0008075284603F0C2FC06462A488046FEF73C
:103800006DFFCDF80080DFF8948027A2294698F854
:1038100002303046F8F706FE054694F823003128BA
:1038200004D12EA1A01C02F059FF20B194F823006E
:10383000302821D025E094F82600302807D0312800
:1038400005D0322803D0332801D050241AE088F85C
:103850000200F8221149484602F03AFC98F802307A
:10386000C5F5807170191EA2F8F7DCFD53243146AE
:103870003846FAF789FE05E018A1A01C02F02EFFD9
:1038800030B14924304603F075FC2046BDE8F8838A
:10389000532431463846FAF777FEF3E7560B0020FB
:1038A000008801082C0700202A4745542A20527519
:1038B0006E4170704E756D3A5B41505025635D20CE
:1038C000212020202A4745542A20417070566572D5
:1038D00073696F6E3A5B25735D20210030303100D3
:1038E0002A5345542A2052756E4170704E756D3AB8
:1038F0005B41505025635DD6D8C6F4BAF3C9FAD0FF
:10390000A721000005280ED2DFE800F00305070913
:103910000B0006A0704708A070470AA070470BA0D4
:1039200070470CA070470DA070470000496E5061B1
:1039300072616D45727200004F7574506172616DF5
:103940004572720052554E455252000052554E4F2C
:103950004B00000054494D454F555400CEB4D6AAF3
:10396000B4EDCEF30000000005280ED2DFE800F031
:10397000030507090B0006A0704708A070470AA0BE
:1039800070470BA070470CA070470DA07047000057
:10399000496E506172616D45727200004F757450CE
:1039A0006172616D4572720052554E45525200006F
:1039B00052554E4F4B00000054494D454F55540051
:1039C000CEB4D6AAB4EDCEF3000000002DE9FF413D
:1039D00004460F46606800F0D1F84FF49676304602
:1039E00003F0CCFB05463846F9F712F8D4E901316B
:1039F000CDE90207CDE90013314628462268F8F7E1
:103A000011FD0246002A01DDB24204DD02240CA0B1
:103A1000FCF712FD0CE000210620FCF781F80446BB
:103A2000032C05D12A4600210720FCF779F804462B
:103A3000284603F09FFB04B02046BDE8F08100005B
:103A4000686561646572426F647942756620D2E789
:103A5000B3F6A3A12D2DD4F6BCD3485454505F43E4
:103A60004D445041434B5F4C454ECAFDD6B5A1A3D2
:103A70000000000070B504460D461021601CF9F7E7
:103A8000BCF82946601CBDE87040F8F792BF10B53D
:103A900004460846F8F738FF608210BD10B50446AA
:103AA0000B2204F11900F9F7F1F8002084F8250041
:103AB00010BD10B504460B2204F12500F9F7E6F815
:103AC000002084F8310010BDAFF300800CB5002257
:103AD000019200922748016841F4803101604FF45F
:103AE000A063016801F4003100910199491C019122
:103AF000009911B901999942F3D10168890302D55E
:103B00000121009100E000920099012930D11A4969
:103B10000A6842F010020A600A6822F003020A6092
:103B20000A6842F002020A604168416041684160EF
:103B3000416841F480614160416821F47C11416039
:103B4000416841F4E8114160016841F08071016011
:103B500001688901FCD5416821F003014160416899
:103B600041F0020141604168C1F381010229FAD1AB
:103B70000CBD00000010024000200240F8B50446D1
:103B80002046F8F745FF0A30064603F0F7FA0546E7
:103B900011A313A2314628460094F8F743FC2846A7
:103BA000F8F736FF024600210420FBF7B9FF044670
:103BB000032C0BD12A4600210520FBF7B1FF044658
:103BC000032C03D1294608A0FAF7C2FB284603F0CC
:103BD000D1FA2046F8BD0000687474703A2F2F00A7
:103BE0002573257300000000504F53542055524C4C
:103BF0003A25732E0000000001460322014802F01E
:103C000067BA0000009001080146F822014802F05E
:103C10005FBA0000008801087CB502F0B1F905F038
:103C2000F5FAFAF749FCFDF7E5F805F065FE5549A8
:103C3000086005F061FE54490860012005F01CFF92
:103C4000524908605248012300901A46642151A04D
:103C500006F022FC534CA06306F036FA0246002020
:103C6000034600900121A06B06F068FC02F088F981
:103C7000022104F10800CDE90010CE0100233246F4
:103C800049A14B4806F0E2F904F10C000921CDE905
:103C900000100023324647A1494806F0D7F904F145
:103CA00010000521CDE900100023324645A1484807
:103CB00006F0CCF904F114001F21CDE90010002317
:103CC000802244A1454806F0C1F904F120000325F3
:103CD000CDE900500023324641A1444806F0B6F930
:103CE00004F12C000621CDE900100023802240A120
:103CF000434806F0ABF904F128000721CDE9001094
:103D0000002332463FA1424806F0A0F904F13000FA
:103D10001D21CDE90010002332463EA1404806F0A7
:103D200095F904F11800CDE90050002332463DA179
:103D30003F4806F08BF9012504F11C00CDE9005045
:103D400000236A023BA13E4806F080F904F13400EA
:103D5000CDE90050002332463AA13D4806F076F9FD
:103D600004F124002021CDE900100023324639A1BE
:103D70003B4806F06BF9606805F0C8FBBDE87C4085
:103D800005F080BA400000203C00002044000020E4
:103D9000C1320408526566726573682054696D65A6
:103DA00000000000000000204E65745461736B0039
:103DB000C11A040852733233325461736B0000002D
:103DC000A535040852733438355461736B00000014
:103DD000293604084C65645461736B00311604087D
:103DE0004D656E755461736B00000000E3160408A6
:103DF00054637048656172745461736B0000000015
:103E0000214C040854637055705461736B000000BA
:103E1000394F040855636D645461736B00000000F2
:103E20003D5D04085463705572635461736B000008
:103E3000D1500408546370446F776E5461736B0003
:103E4000754A040844656275675F7461736B0000AE
:103E5000E95D04084C6973745461736B00000000E1
:103E60005116040808B5002300901A461021184680
:103E7000FEF79AF908BD000008B514A001230090D0
:103E80001A4610210020FEF78FF9134800230090F6
:103E9000022210211846FEF787F90F484038F8F73C
:103EA000B7FD102809D90C480023303800900322B0
:103EB00010211846FEF778F908BD08A000230090ED
:103EC000032210211846FEF76FF908BD465450D55D
:103ED000CBBAC53A00000000A60B0020200000006D
:103EE00008B514A0012300901A4610210020FEF707
:103EF0005BF9134800230090022210211846FEF7B8
:103F000053F90F488038F8F783FD102809D90C4879
:103F1000002370380090032210211846FEF744F960
:103F200008BD08A000230090032210211846FEF7C8
:103F30003BF908BD465450C3DCC2EB3A0000000018
:103F4000E60B00202000000008B514A0012300901B
:103F50001A4610210020FEF727F91248002300908E
:103F6000022210211846FEF71FF90E48C038F8F754
:103F70004FFD102809D90B480023B03800900322C8
:103F800010211846FEF710F908BD07A00023009085
:103F9000032210211846FEF707F908BD46545020A9
:103FA00049503A00260C00202000000038B514A02B
:103FB000012300901A4610210020FEF7F5F8134C5B
:103FC00000230222102118460094FEF7EDF8204647
:103FD000F8F71EFD102809D904F110000023009005
:103FE000032210211846FEF7DFF838BD08A0002391
:103FF0000090032210211846FEF7D6F838BD0000C5
:10400000465450C2B7BEB63A00000000660B00200E
:104010002000000008B50CA0012300901A461021D2
:104020000020FEF7C1F80BA000230090022210210F
:104030001846FEF7B9F80AA00023009003221021C9
:104040001846FEF7B1F808BDB2E9D1AF465450D5D5
:10405000CBBAC500B2E9D1AF465450C3DCC2EB00C5
:10406000B2E9D1AF465450202049500008B50CA009
:1040700000230090012210211846FEF795F80BA0AE
:1040800000900123022210210020FEF78DF80AA0E3
:1040900000230090032210211846FEF785F808BD82
:1040A000B2E9D1AF465450D5CBBAC500B2E9D1AFD1
:1040B000465450C3DCC2EB00B2E9D1AF46545020A5
:1040C0002049500008B50CA00023009001221021C7
:1040D0001846FEF769F80BA0002300900222102179
:1040E0001846FEF761F80AA0009001230322102170
:1040F0000020FEF759F808BDB2E9D1AF465450D5BB
:10410000CBBAC500B2E9D1AF465450C3DCC2EB0014
:10411000B2E9D1AF465450202049500008B50CA058
:1041200000230090012210211846FEF73DF80BA055
:1041300000230090022210211846FEF735F80AA04D
:1041400000900123032210210020FEF72DF808BD66
:10415000B2E9D1AF465450C3DCC2EB00B2E9D1AFF3
:104160004654502020495000B2E9D1AF465450C2C5
:10417000B7BEB60008B514A0012300901A4610215E
:104180000020FEF711F812480023009002221021AF
:104190001846FEF709F80E48D038F8F739FC102811
:1041A00009D90B480023C03800900322102118467B
:1041B000FDF7FAFF08BD07A000230090032210219D
:1041C0001846FDF7F1FF08BD5443502049503A000E
:1041D000360C00202000000008B514A00123009038
:1041E0001A4610210020FDF7DFFF1348002300903E
:1041F000022210211846FDF7D7FF0F48E038F8F7E4
:1042000007FC102809D90C480023D038009003225D
:1042100010211846FDF7C8FF08BD08A00023009034
:10422000032210211846FDF7BFFF08BD544350B6C6
:10423000CBBFDA3A00000000460C0020200000004E
:1042400008B50CA0012300901A4610210020FDF7AC
:10425000ABFF0BA000230090022210211846FDF7AF
:10426000A3FF0AA000230090032210211846FDF7A7
:104270009BFF08BDB2E9D1AF544350202049500004
:10428000B2E9D1AF544350B6CBBFDA0020000000F2
:1042900008B50CA000230090012210211846FDF75C
:1042A00083FF0BA000900123022210210020FDF7C4
:1042B0007BFF0AA000230090032210211846FDF77F
:1042C00073FF08BDB2E9D1AF5443502020495000DC
:1042D000B2E9D1AF544350B6CBBFDA0020000000A2
:1042E00038B513A0012300901A4610210020FDF7D5
:1042F0005BFF102002F042FF0446114811A210217A
:1043000083782046F8F78EF8002302221021184601
:104310000094FDF749FF10A0002300900322102114
:104320001846FDF741FF2046BDE8384002F022BFA5
:10433000B5B1C7B0D4CBD0D0415050BAC53A0000C7
:10434000560B002052756E4170704E756D3A5B25AC
:10435000635DA1A3000000002000000010B5084923
:1043600031204870F822074801F0B2FE06A0F9F7A4
:10437000EFFF0220FAF79CFEBDE8104000F066BA9D
:10438000560B002000880108C9FDBCB6C9E8B1B8C9
:10439000A3ACBCB4BDABD6D8C6F4000008B50CA025
:1043A000012300901A4610210020FDF7FDFE0BA00E
:1043B00000230090022210211846FDF7F5FE0AA006
:1043C00000230090032210211846FDF7EDFE08BDE2
:1043D000B2E9D1AFB5B1C7B041505000C1A2BCB431
:1043E000C9FDBCB6415050002000000008B50CA02B
:1043F00000230090012210211846FDF7D5FE0BA0E6
:1044000000900123022210210020FDF7CDFE0AA01A
:1044100000230090032210211846FDF7C5FE08BDB9
:10442000B2E9D1AFB5B1C7B041505000C1A2BCB4E0
:10443000C9FDBCB6415050002000000038B512A0A4
:10444000012300901A4610210020FDF7ADFE19202F
:1044500002F094FE044601212046FCF78DFB002368
:1044600002220C2118460094FDF79EFE04F115006F
:104470000023009003220C211846FDF795FE2046EC
:10448000BDE8384002F076BE4D414349443A000051
:1044900038B511A0012300901A4610210020FDF725
:1044A00083FE0C2002F06AFE04462046FEF716F951
:1044B00000230222102118460094FDF775FE09A082
:1044C00000230090032210211846FDF76DFE2046C0
:1044D000BDE8384002F04EBE41505020B0E6B1BEBB
:1044E000BAC53A002000000008B50CA001230090D6
:1044F0001A4610210020FDF757FE0BA00023009064
:10450000022210211846FDF74FFE0BA00023009059
:10451000032210211846FDF747FE08BDB2E9D1AFCE
:104520004D41434944000000B2E9D1AF4150502011
:10453000B0E6B1BE00000000B2E9D1AF424F4F5427
:10454000B0E6B1BE0000000008B50CA0002300904A
:10455000012210211846FDF727FE0BA00090012331
:10456000022210210020FDF71FFE0BA00023009067
:10457000032210211846FDF717FE08BDB2E9D1AF9E
:104580004D41434944000000B2E9D1AF41505020B1
:10459000B0E6B1BE00000000B2E9D1AF424F4F54C7
:1045A000B0E6B1BE0000000008B50CA000230090EA
:1045B000012210211846FDF7F7FD0BA00023009003
:1045C000022210211846FDF7EFFD0BA000900123F9
:1045D000032210210020FDF7E7FD08BDB2E9D1AFAD
:1045E0004D41434944000000B2E9D1AF4150502051
:1045F000B0E6B1BE00000000B2E9D1AF424F4F5467
:10460000B0E6B1BE0000000008B50CA00123009088
:104610001A4610210020FDF7C7FD0BA000230090D3
:10462000022210211846FDF7BFFD0AA000230090CA
:10463000032210211846FDF7B7FD08BD465450204F
:10464000D0C5CFA20000000054435020D0C5CFA257
:1046500000000000C9E8B1B8C9FDBCB60000000008
:1046600008B50CA000230090012210211846FDF788
:104670009BFD0BA000900123022210210020FDF7DA
:1046800093FD0AA000230090032210211846FDF795
:104690008BFD08BD46545020D0C5CFA200000000BD
:1046A00054435020D0C5CFA200000000C9E8B1B8E3
:1046B000C9FDBCB60000000008B50CA000230090A6
:1046C000012210211846FDF76FFD0BA0002300907A
:1046D000022210211846FDF767FD0AA00090012371
:1046E000032210210020FDF75FFD08BD4654502035
:1046F000D0C5CFA20000000054435020D0C5CFA2A7
:1047000000000000C9E8B1B8C9FDBCB60000000057
:1047100008B50CA000230090012210211846FDF7D7
:1047200043FD0BA000230090022210211846FDF744
:104730003BFD0AA000900123032210210020FDF779
:1047400033FD08BD54435020D0C5CFA20000000067
:10475000C9E8B1B8C9FDBCB600000000C9E8B1B8ED
:10476000D0C5CFA2000000004FF0E021042804D003
:10477000086920F0040008617047086940F00400EF
:104780000861704710B505F091FC01280CD005F0C8
:104790005DF90748416811F1020F01D30021416022
:1047A0004168491C416010BDBDE8104001F0E8BB04
:1047B0002006002010B50420FFF7D6FF0C480D4955
:1047C0000D4A0068B0FBF1F31370B0FBF1F142F257
:1047D000107041430A2050804FF0E020026942F0FF
:1047E000020202614161016941F00101016110BDF4
:1047F0003C06002040420F002006002010B50F4864
:10480000016841F00101016041680D4A11404160B9
:1048100001680C4A11400160016821F480210160A7
:10482000416821F4FE0141604FF41F018160FFF7F0
:104830004BF905494FF00060086010BD00100240C0
:104840000000FFF8FFFFF6FE08ED00E071B6054836
:104850000168054A01F4E06111430160BFF34F8F25
:10486000FEE700000CED00E00400FA0510B50121A0
:104870008C07204600F073F8012808D1012120465A
:1048800000F06AF8BDE81040002000F01FBE10BD27
:1048900010B5084C0121204600F061F8012808D12C
:1048A0000121204600F058F8BDE81040012000F03A
:1048B0000DBE10BD0004004010B5084C012120467B
:1048C00000F04DF8012808D10121204600F044F8FD
:1048D000BDE81040022000F0F9BD10BD0008004006
:1048E00010B5084C0121204600F039F8012808D104
:1048F0000121204600F030F8BDE81040032000F010
:10490000E5BD10BD000C004010B5084C012120464B
:1049100000F025F8012808D10121204600F01CF8FC
:10492000BDE81040042000F0D1BD10BD00100040D3
:1049300010B5084C0121204600F011F8012808D1DB
:104940000121204600F008F8BDE81040052000F0E5
:10495000BDBD10BD00140040C9430182704702462E
:104960000020138A0B4092890A40002B02D0002AB3
:1049700000D001207047000010B586B001214FF42F
:104980000170FDF79DFF4FF40040FDF773FF174CDA
:104990002046F9F747FC002101918DF808108DF8A9
:1049A00009104FF460220392049101218DF8141034
:1049B00001A92046F9F776FC0120F9F7A1FC0121B5
:1049C0002046F9F723FC2046F9F790FC2046F9F73A
:1049D00062FC0028FAD12046F9F78DFC2046F9F751
:1049E00053FC0028FAD106B010BD0000002401409D
:1049F00005280ED2DFE800F0030507090B0006A02A
:104A0000704708A070470AA070470CA070470EA01E
:104A1000704710A0704700004F50454E534F434B16
:104A200045540000434C4F5345534F434B455400AE
:104A30005155455259534F434B45540054435053DD
:104A4000454E44434D44000054435053454E444268
:104A500055460000CEDEB4CBC3FCC1EE0000000022
:104A600010B50020F9F78BFDBDE810400120FAF7E2
:104A7000CEBA00001CB50027DFF8DC804FF4806957
:104A800057E036A1304601F029FE0546002D46DBF1
:104A90004FF4007002F072FB04464FF480700090F7
:104AA000711900230A222046F9F788FE2046F7F7FD
:104AB000AFFF217828290CD194F82510262908D198
:104AC000211811F8052C242A03D111F8031C2929D7
:104AD00007D0214625A0F9F73BFC204602F04AFB0F
:104AE00021E06178412915D0432908D0214627A02B
:104AF000F9F72EFC2DA1522000F072FBEDE782B2F7
:104B000021463148FCF70CFC0028E6D02FA0FBF72B
:104B100093FCE2E7214632A0F9F71AFCDDE73146C3
:104B200037A0FBF789FC304602F024FB032004F099
:104B3000B5FC0221D8F8000004F0ECFE484602F073
:104B40001DFB0646019701AA31463448FCF788F858
:104B50000028E8D195E70000400000202B5149557E
:104B600052433A202272656376220000544350CAB1
:104B7000D5B5BDCFC2D0D027B7C727B7A8CAFDBE0D
:104B8000DDD6A1A3BA25732000000000544350CA0B
:104B9000D5B5BDCFC2D0D0CEB4D6AAC0E0D0CDCA94
:104BA000FDBEDDD6A13A257320000000544350CA53
:104BB000D5B5BDCFC2D0D0CEB4D6AAC0E0D0CDCA74
:104BC000FDBEDDD6A10000005007002073557365BF
:104BD00072636D645175657565D2E7B3F6A3A10084
:104BE00054637020736572766572C8B7C8CFCAD532
:104BF000B5BDCAFDBEDDD6A13A2573200000000078
:104C000054435020CFC2D0D0CAFDBEDDBDE2CEF6A7
:104C1000CAA7B0DCA3BA257320000000341F00200F
:104C200008B54FF47A662E4C2E4D4CE04FF4DA72F4
:104C30002DA141F27070FDF71BFA2D480746FAF7D7
:104C4000A1FE2B48401F8046FAF716FF43463A461E
:104C500028A1482000F0C4FA2D4800231A4619461E
:104C6000006805F06DF819212A48F7F7C6FF4FF4E0
:104C7000DC7000901CA328A219212648F7F7D2FB6C
:104C80002448F9F765FB102002F078FA8146434684
:104C900025A210214846F7F7C5FB4846FAF7CEFA99
:104CA00010214846F7F7A9FF3B4621A210214846AC
:104CB000F7F7B8FB4846FAF7E7FA484602F05AFA1F
:104CC000304604F0EBFB1021206804F023FE0021A5
:104CD000286804F0DDFDC0434007F1D4A6E70000DA
:104CE000400000203C0000206D61696E2E630000D2
:104CF000961C00204353513A25732C2045433230F3
:104D000020566F6C746167653A25736D560000001C
:104D100044000020E2060020257320256420CACD2F
:104D2000B7C545433230210025736D5600000000A1
:104D300043535125730000002DE9F04707463C46D8
:104D4000A0782179303800EBC00202EB001001EBB3
:104D50008001E0786FF02F02303800EB800002EB2A
:104D600040000D18DFF8A4A0F82227495046FEF7AE
:104D70009EFA4FF48076304602F000FA8046224BCD
:104D800023A2E033994631464046F7F74BFB0646EF
:104D900094F82300312804D1611991F826102429B0
:104DA00002D030281DD021E010214846F7F725FF1A
:104DB0002A4604F126014846F7F768FFF82212490F
:104DC000504601F085F9C6F5807108EB06004B46A8
:104DD00014A2F7F727FB532441463846F9F7D4FBD2
:104DE00005E0601990F82600242806D049244046A2
:104DF00002F0C0F92046BDE8F0875324414638460A
:104E0000F9F7C2FBF3E70000560B00200088010809
:104E10002A4745542A2054637049503A5B25735DF4
:104E2000210000002A5345542A2054637049503A07
:104E30005B25735D210000002DE9F04707463C46E5
:104E4000A0782179303800EBC00202EB001001EBB2
:104E50008001E0786FF02F02303800EB800002EB29
:104E600040000D18DFF8A4A0F82227495046FEF7AD
:104E70001EFA4FF48076304602F080F98046224BCD
:104E800023A2F033994631464046F7F7CBFA06465F
:104E900094F82300312804D1611991F826102429AF
:104EA00002D030281DD021E010214846F7F7A5FE9A
:104EB0002A4604F126014846F7F7E8FEF82212498F
:104EC000504601F005F9C6F5807108EB06004B4627
:104ED00014A2F7F7A7FA532441463846F9F754FBD2
:104EE00005E0601990F82600242806D049244046A1
:104EF00002F040F92046BDE8F08753244146384689
:104F0000F9F742FBF3E70000560B00200088010888
:104F10002A4745542A20546370506F72743A5B25B7
:104F2000735D21002A5345542A20546370506F72D8
:104F3000743A5B25735D21001CB52D4C2D4D4BE063
:104F40004FF4806002F01AF906460020019001AA91
:104F500031462948FBF784FE002837D140F29912E8
:104F600026A141F27070FDF783F8BDF804203146A8
:104F7000244800F015FA032811D0BDF8042031466A
:104F8000204800F00DFA032809D00421206804F01D
:104F90007FFC1DA0FBF750FA1BA000F0F3FF1F4899
:104FA00000231A461946006804F0CAFE19211C485D
:104FB000F7F723FE40F2A510009010A319A21921C3
:104FC0001748F7F72FFA1648F9F7C2F9304602F0FA
:104FD000D1F8322004F062FA0821286804F09AFC23
:104FE0000021206804F054FCC0434007F1D4A7E737
:104FF0003C000020400000204E0C00206D61696ED6
:105000002E630000AA0100205463702053656E6473
:105010004461746120457272210000004400002048
:10502000E2060020257320256420CACDB7C545437C
:105030003230210070B50546052410A1284601F044
:105040004DFB002801DD002416E011A1284601F0E7
:1050500045FB002801DD04240EE012A1284601F0E2
:105060003DFB002801DD022406E013A1284601F0E3
:1050700035FB002800DD0324204670BD2B51495527
:1050800052433A2022636C6F736564220000000073
:105090002B51495552433A20227064706465616314
:1050A000742200002B51495552433A2022696E6305
:1050B0006F6D696E672200002B51495552433A20AB
:1050C00022696E636F6D696E672066756C6C220075
:1050D00008B5294C0025294E4FF4807717E0BDF81C
:1050E00000104046FFF7A6FF10B3022836D0032871
:1050F0003BD0042827D022A0FBF79EF920A000F087
:1051000041FF404602F036F8322004F0C7F904218E
:10511000306804F0FFFB384602F030F88046009516
:105120006A4641461B48FBF79BFD0028E9D1D6E7BC
:105130000421206804F0ACFB17A0FBF77DF916A052
:1051400000F020FFDDE70F21206804F0A1FB17A08D
:10515000FBF772F915A000F015FFD2E717A0FBF7D7
:105160006BF916A000F00EFFCBE719A0FBF764F96E
:1051700017A000F007FFC4E73C000020400000201B
:1051800054637020756E6B6E6F776E20757263203E
:105190002E0000003A23002054637020736572765D
:1051A000657220636C6F736564202E0054637020F9
:1051B000504450206465616374202E005463702055
:1051C000696E636F6D696E672066756C6C202E006A
:1051D00054637020696E636F6D696E67202E0000E6
:1051E0000FB4F8B50646032540F2492001F0C6FF8A
:1051F000044608AB00934FF40077394604F12600CB
:10520000079AF7F7D3F8002801DDB8420BDD8322B7
:105210002CA131A0FBF710F9204601F0ABFF0220D2
:10522000F8BC5DF814FB282222706670642290FBA3
:10523000F2F13031A17090FBF2F102FB11010A2270
:1052400091FBF2F13031E17090FBF2F102FB1100C1
:1052500030302071274908786071401CC0B2087056
:10526000392801D930200870042223A1A01DF7F7A6
:105270000DFD012104F10A00FBF77EFC3B2184F8BF
:1052800022103022022104F12300F7F7AEFC262180
:1052900084F8251003221AA12046F7F74CFB20467C
:1052A000F7F7B6FB82B221461648FCF739F820B171
:1052B000A22204A114A0FBF7BFF8204601F05AFF78
:1052C0002846ADE7555345525F5443505C757365AE
:1052D000725F7463702E630025732C25643A7570B9
:1052E00044617461427566207370696C6C6F766599
:1052F00072A3A100A80100204D41433A0000000024
:10530000245829004E0C002025732C25643A735430
:105310006370305175657565207370696C6C6F765C
:105320006572A3A10000000070B504462078F9F76B
:1053300026F903280CD1A38A628A2078611CFDF724
:10534000DFF80546032D02D12078FDF73DFA284607
:1053500070BD000070B5102001F010FF0546294611
:105360000120FDF7CBF9032807D029460120F8F7E3
:10537000DCFF0446032C02D005E0032070BD294663
:1053800003A0F8F7E5FF284601F0F4FE204670BDC3
:10539000544350B1BEB5D84950A3BA25730000009C
:1053A0002DE9F84F06468A469146B9F1000F0DD017
:1053B0000025A84600240427FAF76CFF3278364E01
:1053C000B16D4B46022000F073FA0DE00320BDE8FA
:1053D000F88F1420F9F76CFE3E213048F7F7A1FA58
:1053E00010B14FF0010804E028466D1CEDB24628CC
:1053F000EFD3B8F1010F10D03846FEF783FA044618
:105400000320FFF7F5FA01462448009024A3224622
:1054100026A0FBF711F83846D9E74A465146022044
:1054200000F0F8F930E06420F9F742FEF16F1B4814
:1054300001F054F9C6F88000D6F8800000280DDB92
:1054400003273846FEF75EFA04460420FFF7D0FA39
:105450000146224618A0F9F7DFFDDCE7D6F88410F4
:105460000E4801F03BF900280EDB02273846FEF714
:1054700049FA04460420FFF7BBFA0146074B2246CF
:105480000FA0FAF7D9FFC6E72046641CB6F87810DB
:10549000A4B28842C7D3BEE7D0030020B41C0020CA
:1054A000CEB4CAD5B5BD223E22000000257320250A
:1054B00073202573202573002573202573000000B9
:1054C000257320257320257300000000034951F83F
:1054D0002000002800D0004770470000F85B002043
:1054E000014901200870704778050020014901201A
:1054F0004870704778050020014901208870704786
:105500007805002001490120C87070477805002007
:1055100070B51C4C40F22441204600F02AFBA0B19B
:10552000194D0021686AF9F75BFC2088201D00886E
:10553000686AF9F729FDC0F5807082B2134903202B
:1055400000F0B4FB032000F06BF840F2255529462B
:10555000204600F00EFB18B12946204600F0E4FA80
:1055600040F227752946204600F003FB20B10022B7
:105570002946204600F01DFB2046BDE87040402132
:1055800000F0CEBA004C0040C8050020445900206D
:105590002DE9F0411F4D40F22551284600F0E9FA6F
:1055A0001D4C002658B1AA882168481C20601B4861
:1055B0004254216846542068FF2800DB266040F2F0
:1055C00024473946284600F0D4FA88B12888A888AC
:1055D0002068124982B2042000F068FB4FF4807109
:1055E0000E48F7F72CFB26603946284600F09CFA57
:1055F00040F227742146284600F0BBFA002806D066
:1056000021462846BDE8F041002200F0D2BABDE8AC
:10561000F08100000050004074050020445A002032
:105620002DE9F0410446104D104E0021285D56F83A
:105630002000F9F7D5FB05F10A0705F1280037F836
:10564000141050F82400F7F7D8FA285D37F8141032
:1056500056F82000F9F7D5FC285D012156F8200006
:10566000BDE8F041F9F7BCBB20C50408C80500201F
:105670002DE9F04387B004460D46164698460121B1
:105680000846FDF71DF95F481822015D401F005DC7
:10569000FBF760FB5B4804220A30015D401F005DA0
:1056A000FBF758FB5848002C7ED050F8240001210D
:1056B000FDF7F8F802950025ADF80C50ADF80E5046
:1056C000ADF81050ADF81450ADF812604D4E02A96F
:1056D0000F3656F8240000F087FA56F824004FF4ED
:1056E000587100F01DFABDF8120006F11409000708
:1056F00021D5042C1FD056F824000122802100F06F
:1057000027FA414F00950195183F59F82410385D4C
:1057100010230022F9F772FB06F12400002150F853
:105720002420385DF9F740FF3848012150F8242043
:10573000385DF9F739FFBDF81200400759D53248F6
:105740001038005D8DF818008DF819808DF81A500A
:1057500001208DF81B0006A8FCF7F4F856F8240089
:10576000012240F2244100F024FA042C3BD056F8E8
:1057700024000122402100F0EBF9CDE90058224835
:1057800059F824101430A0F1280550F82420285D81
:105790000023F9F733FB05F10A001D4F30F8141010
:1057A000285D57F8200000E018E0F9F72AFC1748B8
:1057B0000021103050F82420285DF9F7F5FE134839
:1057C0000121203050F82420285DF9F7EDFE285DF6
:1057D000012157F82000F9F703FB0AE000680121D6
:1057E000FDF76EF866E7012240F22551306900F0BE
:1057F000E0F956F82400012100F09EF907B0BDE859
:10580000F08300008105002034C504080056002004
:10581000C80500202DE9F047044688461646B8F131
:10582000000F23D0002E21D0042C21D01D4FDFF8F3
:1058300078900021385D59F82000F9F7D1FA1B4D16
:1058400000202855385D59F82000C0F80C80385DDC
:10585000314659F82000F9F7D4FB385D012159F899
:105860002000F9F7BDFA285D0028FCD0BDE8F087DC
:1058700000250E4F40211837386900F073F90EE00B
:1058800018F8051057F8240000F00CFA57F8240017
:10589000402100F067F90028F8D06D1CADB2B54288
:1058A000EED3E3E71CC50408C805002078050020F6
:1058B0000FB470B586B004460CA801903A4E10E0C3
:1058C0005C2916D0252930D0401C0B9056F82400B6
:1058D00000F0E8F956F82400402100F043F90028D0
:1058E000F8D00B9801780029EAD106B070BC5DF8B9
:1058F00014FB401C0B9001786E290DD0722902D048
:10590000401C0B90E6E756F824000D2100F0CAF980
:105910000B98401C0B90DDE756F824000A2100F09C
:10592000C1F90B98401C0B90D4E7401C0B900178F8
:1059300064291BD0732902D0401C0B90CAE7019840
:1059400020C801900BE056F8240000F0ABF956F89F
:105950002400402100F006F90028F8D06D1C2978B9
:105960000029F0D10B98401C0B90B3E701980199E6
:105970000068091D01910A2202A900F081FE02AD12
:105980000BE056F8240000F08DF956F82400402171
:1059900000F0E8F80028F8D06D1C29780029F0D133
:1059A0000B98401C0B9095E79005002070B51B4CA0
:1059B00040F22441204600F0DCF8A0B1184D00214F
:1059C0002869F9F70DFA2088201D00882869F9F761
:1059D000DBFAC0F5807082B21249002000F066F94F
:1059E0000020FFF71DFE40F225552946204600F015
:1059F000C0F818B12946204600F096F840F2277505
:105A00002946204600F0B5F8002806D02946204651
:105A1000BDE87040002200F0CCB870BD00380140F5
:105A2000C80500204456002070B51B4C40F22441AC
:105A3000204600F09EF8A0B1184D00216869F9F7E2
:105A4000CFF92088201D00886869F9F79DFAC0F514
:105A5000807082B21249012000F028F90120FFF77E
:105A6000DFFD40F225552946204600F082F818B1A6
:105A70002946204600F058F840F22775294620466E
:105A800000F077F8002806D029462046BDE870408F
:105A9000002200F08EB870BD00440040C805002010
:105AA0004457002070B51B4C40F22441204600F0C2
:105AB00060F8A0B1184D0021A868F9F791F9208885
:105AC000201D0088A868F9F75FFAC0F5807082B2DF
:105AD0001249022000F0EAF80220FFF7A1FD40F28F
:105AE00025552946204600F044F818B1294620469D
:105AF00000F01AF840F227752946204600F039F8E0
:105B0000002806D029462046BDE87040002200F05B
:105B100050B870BD00480040C8050020445800201F
:105B20008A05C9430180704740F66A120A0A0121BA
:105B30009140C94301807047002904D0818941F414
:105B4000005181817047818921F400518181704722
:105B5000002A03D0828A0A4382827047828A8A435B
:105B6000828270470246002012880A4200D001203B
:105B7000704770B5002440F66A12C1F3421301F079
:105B80001F05012606FA05F2012B0CD0022B0DD0C1
:105B9000838A1340090A8E40008830400BB100B15F
:105BA0000124204670BD83891340F3E7038A134024
:105BB000F0E710B540F66A13C1F3421301F01F0479
:105BC0000121A140012B07D0022B07D014303AB19C
:105BD00002680A43026010BD0C30F8E71030F6E7A7
:105BE00002688A43026010BD30B585B004460D4698
:105BF000208A4CF6FF710840E98801432182A08980
:105C00004EF6F3110840A9882A8911436A89024394
:105C10001143A181A08A4FF6FF410840A9890143A1
:105C2000A1826846FCF776FE1D48844201D10398A4
:105C300000E00298A189090408D500EBC00101EB3E
:105C4000001029684900B0FBF1F007E000EBC0014B
:105C500001EB001029688900B0FBF1F06422B0FB71
:105C6000F2F109010B096FF018056B4300EB83009B
:105C7000A3891D044FF0320307D503EBC000B0FB2E
:105C8000F2F000F00700084306E003EB0010B0FB61
:105C9000F2F000F00F000843208105B030BD000095
:105CA00000380140C1F308018180704730B40C46D0
:105CB000054951F82030002B03D0204630BC114656
:105CC000184730BC704700003056002010B50C4615
:105CD000084A52F82030002B09D0522206A10CA00D
:105CE000F6F77EFB0EA0F6F77BFB204610BD42F8D0
:105CF0002040FAE7305600202E2E5C53595354456D
:105D00004D5C55534152545C75736172742E63003F
:105D10004C6F674572723A2025732C256400000091
:105D2000556172742043616C6C6261636B207265B3
:105D300070656174207265672100000008B5002558
:105D40000F4C4FF400760AE0BDF800103846F8F723
:105D5000D1FC384601F00EFA322003F09FFB2021DF
:105D6000206803F0D7FD304601F008FA0746009599
:105D70006A4639460348FAF773FF0028E9D1E3E79A
:105D80004000002050070020FEE7000010B5044648
:105D90000748FBF7BBFA05230C2221460020FFF73A
:105DA00067FCBDE8104003490020FFF78FBF0000EB
:105DB00054100020B95D040810B50A460146054894
:105DC000FBF7AEFA002804D0BDE8104002A0FAF7B5
:105DD00033BB10BD54100020735573625175657547
:105DE00065D2E7B3F6A3A10008B500254FF400760D
:105DF0001CE02046F6F70CFE217828290CD194F8F7
:105E00002510262908D1221812F8051C242903D1AF
:105E100012F8031C292916D021461AA0F8F798FA7F
:105E2000204601F0A7F9322003F038FB304601F09C
:105E3000A5F9044600956A4621461A48FAF710FF6C
:105E40000028EDD1D5E76278412A15D0632A08D021
:105E5000214615A0F8F77CFA1BA15220FFF7C0F9E4
:105E6000DEE782B221461F48FBF75AFA0028D7D056
:105E70001DA0FAF7E1FAD3E7214620A0F8F768FA67
:105E8000CEE70000555342CAD5B5BDCFC2D0D0270A
:105E9000B7C727B7A8CAFDBEDDD6A1A3BA25732010
:105EA0002E00000054100020555342CAD5B5BDCF76
:105EB000C2D0D0CEB4D6AAC0E0D0CDCAFDBEDDD609
:105EC000A1A3BA2573202E00555342CAD5B5BDCF24
:105ED000C2D0D0CEB4D6AAC0E0D0CDCAFDBEDDD6E9
:105EE000A1000000500700207355736572636D6454
:105EF0005175657565D2E7B3F6A3A100555342C944
:105F0000CFCEBBBBFAC8B7C8CFCAD5B5BDCAFDBED8
:105F1000DDD6A1A3BA2573202E00000010B5FBF733
:105F20001BFB0F490C20FBF7CFFA0E490B20FBF7A8
:105F3000CBFA0D490920FBF7C7FA0C490D20FBF7F6
:105F4000C3FA0B490720FBF7BFFA0A490F20FBF7FA
:105F5000BBFABDE8104008490620FBF7B5BA0000BF
:105F6000F116040899E40308251604084D150408E1
:105F700001160408191604080D160408532070476A
:105F8000FBF796B82DE9F84F05462846F6F740FD91
:105F900000287BD02846F6F73BFD14301FFA80F826
:105FA000404601F0EBF8074600260024384B39A2A2
:105FB000414638460095F6F735FA80B200F0010107
:105FC00001EB5005FAF7EEFA3520FAF77FFA10E008
:105FD0000A20F9F76DF80A2C09D931A0FAF72CFA42
:105FE000FAF7E0FA3846BDE8F84F01F0C3B8641C90
:105FF000A4B20120FAF7A2FA0128E9D0DFF8B490A0
:10600000DFF8B4A031E02020FAF760FA701C81B20A
:10601000B85D08B940F02D004A1C795C96B240EAA0
:106020000124200A01D144F43454D9F80400C8F5FD
:106030000061884207D30020C9F80400B9F80800BD
:10604000401CA9F80800D9F804005044410501D1CA
:10605000FAF742FAD9F8040021465044FAF788FAD0
:10606000D9F80400801CC9F804006D1EADB2CAD274
:10607000FDF746F9FAF774FA10A0D9F80410F8F70A
:1060800067F93846BDE8F84F01F074B8BDE8F88FFD
:10609000EF5B00202A25732025732A2000000000D2
:1060A000D0B4466C617368C3A6B5C8B4FDB3ACCABE
:1060B000B1A3A100681C002000F80708466C6173BA
:1060C00068C6ABD2C6B3A4B6C83A25237800000090
:1060D0002DE9F04107460E46002402F0010000EBD6
:1060E00052052120FCF76CFC01280AD0A82241A10E
:1060F00046A0F6F775F949A0F6F772F90220BDE857
:10610000F081FAF74FFAA7F10060B0F5002F01D245
:1061100078050BD0AE2237A13CA0F6F761F93FA07D
:10612000F6F75EF9FAF71CFA0220E8E7B5F5006F1A
:106130000BD9B4222FA135A0F6F752F937A0F6F704
:106140004FF9FAF70DFA0220D9E73520FAF7BEF930
:106150003846FAF7C1F904281BD0BB2225A12BA091
:10616000F6F73EF92DA0F6F73BF912E00A20F8F712
:106170009FFF0A2C0BD9C2221EA124A0F6F730F9EA
:1061800026A0F6F72DF9FAF70DFA0220B7E7641CFE
:10619000A4B20120FAF7D2F90128E7D023E02020A9
:1061A000FAF794F930787178B61C40EA0121384644
:1061B000FAF7DEF9002410E00A20F8F779FF1E2C28
:1061C00009D9D3220BA111A0F6F70AF913A0F6F70B
:1061D00007F9022093E7641CA4B22020FAF7AEF975
:1061E0000128E9D1BF1C6D1EADB2D8D2FAF7B8F9BB
:1061F000032084E72E2E5C53595354454D5C464C86
:106200004153485C666C6173682E63004C6F674550
:1062100072723A2025732C256400000000000000F3
:10622000490050EAC12018BF04204A0D18BF40F0B1
:10623000010040F2FF72B2EB515F08BF40F0020074
:10624000012808BF052070472DE9F0414F1E00EBE3
:10625000C7010446D1E9000115461E4637F0060283
:106260000DD02A46334604F0C9FC7F1E04EBC70359
:10627000D3E9002304F0DCF937F00602F1D1022F54
:1062800025D0042F13D0062F18BFBDE8F0812A4671
:10629000334604F0B3FCD4E90A2304F0C9F92A46D2
:1062A000334604F0ABFCD4E9082304F0C1F92A46D4
:1062B000334604F0A3FCD4E9062304F0B9F92A46D6
:1062C000334604F09BFCD4E9042304F0B1F92A46D8
:1062D000334604F093FCD4E9022304F0A9F92A46DA
:1062E000334604F08BFCD4E90023BDE8F04104F010
:1062F0009FB90000002213461046014904F054BA29
:106300000000F03F012204F0BFBF04F091B9002269
:1063100013461046114604F047BA40F201320020FD
:106320004FF0E04104F0B0BF024A0020110704F032
:10633000ABBF000001FDFFFF30380A2801D2012069
:10634000704700207047704702469068002901D0CE
:1063500010B991607047104610B10268002AFAD156
:1063600002F0FEBE70B505460E461446002C0DD058
:10637000206A08B100F0FEFE304600F0C0F820624E
:1063800021462846BDE87040FFF7DEBF70BD10B55E
:1063900000F048F8002801D00621C16010BD70B59A
:1063A000054600F03FF804462CB10420E060284682
:1063B00000F0A5F82061204670BD70B5044619E0D4
:1063C0002568A089C00503D4A06808B1FFF7F5FFD0
:1063D000A089C00503D4206908B100F0CBFEA089D4
:1063E000800503D4206A08B100F0C4FE204600F006
:1063F000C1FE2C46002CE3D170BD000001480068AE
:1064000070470000D001002070B50D46846800E0A0
:1064100024682CB12946206A00F04BF80028F7D1F7
:10642000204670BD10B5282000F0A8FE04461CB11F
:1064300028212046F6F703FC204610BD0022114615
:10644000AFF300802DE9F04104460D469046FFF77A
:10645000E9FF0646134F00203860C6B1204602F01F
:106460004FFE0146304600F027FE04468CB1B8F1DD
:10647000000F13D0204602F043FE0446207868B196
:106480003046FFF79AFF3C600020BDE8F081002015
:10649000FBE73046FFF791FF0020F6E705B12C60DF
:1064A0003046F2E7D001002000230122194602F015
:1064B0002BB870B504460D46002C01D02DB10AE072
:1064C0000DB1012070BD002070BD012070BD20788D
:1064D00098B1641C6D1C2078F5F75BFF06462878A0
:1064E000F5F757FF8642F2D02078F5F752FF0446C1
:1064F0002878F5F74EFF201A70BD002070BD70B5EA
:1065000006463046F6F784FA451C284600F036FE6B
:10651000041E06D02A4631462046F6F7EFFA2046FA
:1065200070BD204600F026FE002070BD0320401EF6
:10653000C0B2FCD2704770B50446002C08D0236866
:1065400033B1A26850186168814203DB981870BDAE
:10655000002070BD01F07AFB0646304600F00EFECA
:10656000054665B1D4E900122846F6F7C7FA206857
:1065700000F000FE66602560A068284470BD2068B9
:1065800000F0F8FD00206060206070BD2DE9F04152
:10659000C1F30A52A2F2FF362F4A304B0D46044691
:1065A000142E2FDA002E12DA04F042F800221346DD
:1065B00004F022FC4CD2002DA4BF0024254647DA6B
:1065C00025F00040204318BF254D41D018E0DFF8EA
:1065D00094C02CFA06F705EA070C5CEA040C08BF25
:1065E000BDE8F08104F024F80022134604F004FC16
:1065F0002ED2002D03DA4FF48010F0400544BD4345
:10660000002425E0332EC8BFBDE8F081A6F1140CAC
:106610004FF0FF3727FA0CF73C4208BFBDE8F08186
:1066200004F020FC0022134604F0E6FB10D2002DFB
:106630000DDA142E08BF6D1C09D0C6F134000121FB
:1066400001FA00F02044A04238BF6D1C0446BC4350
:1066500029462046BDE8F0819C7500883CE4377EE1
:106660000000F0BFFFFF0F000449C2B20B689A8020
:1066700009680A885206FCD5704700009005002082
:10668000F0B503460025084600260A2A01D0067008
:10669000F0BD002B1DD005DA4FF02D0200F8012BC4
:1066A000C3F1000342F210724FF00A0793FBF2F4B9
:1066B00054EA050C06D004F1300500F8015B04FB38
:1066C0001233012592FBF7F2002AEFDC0670084630
:1066D000F0BD3022027046700846F0BD2DE9F0474B
:1066E000824689465046F6F793F987B24846F6F750
:1066F0008FF986B200250024304600F03FFD804629
:106700004146484600F021F80DE01AF8050019F856
:106710000410884204D16D1CADB2641CA4B202E026
:106720006CB118F80440BD4201D2B442EDD34046EA
:1067300000F020FDB44205D3A81BBDE8F0876D1C16
:10674000ADB2F0E74FF0FF30F7E72DE9F041054635
:106750000C462846F6F75CF980B2002100B12170A2
:106760000122002312E0AE5CEF5CBE420CD1521C51
:1067700092B25B1C9BB2AE5CEF5CBE4201D0A354F4
:1067800004E0E65CA65401E023B1E35C8242EAD374
:10679000BDE8F081521C92B2A154F7E72DE9F04D0B
:1067A000C84A002490B0914205DA21F00043934298
:1067B00001D805D120B110B0BDE8F04DFFF7A2BD62
:1067C000B1F5801F1BDA53EA000209D0002911DA63
:1067D0000120F6F79CFA10B0BDE8F04DFFF797BD29
:1067E0000220F6F794FAFFF785FD10B081F0004122
:1067F000BDE8F08D6FF03504362204F045FD04EB62
:106800002152C1F31308B049A2F2FF33414401F40D
:10681000801282F07F6103EB225281F0405100929E
:1068200041EA08010022A94B04F00EFC044608F1DD
:106830000200A74EC0F313000D467E44032867D222
:10684000D6E90023204604F007F91ED1009800285D
:1068500002BFD6E9000110B0BDE8F08D04F067F981
:1068600007460C469B4A9C4B04F0C8F906460D4669
:106870009A4A9B4B3846214604F0C0F910B0324684
:106880002B46BDE8F04D03F0D3BE4FF05532954B8B
:106890002046294604F0B2F90022934B04F0E2FAB4
:1068A00006460F4622462B461046194604F0A6F926
:1068B00032463B4604F0A2F9064600980F46F0B176
:1068C00004F035F980468A46824A834B04F096F9F3
:1068D00032463B4604F0C6FA22462B4604F0B4FB8F
:1068E00005460C467D4A7E4B4046514604F086F9EB
:1068F00010B02A462346BDE8F04D04F0A5BB0B4678
:1069000010B0324620462946BDE8F04D04F09CBB4D
:1069100000224FF08043204603F08AFE02460B46D9
:106920002046294603F040FF06460F46009804F033
:10693000FEF8CDE9040132463B461046394604F0E4
:106940005DF90C9069480C9A4044019009910B46FE
:10695000104604F053F98246024665488B46C8F15A
:1069600051080B4608F5D72803217844FFF76CFC43
:1069700052465B4604F042F90A905E480D91524639
:106980005B4604217844FFF75FFC099B0C9A04F0F6
:1069900035F9844601980D9B40EA080860460A9A3A
:1069A00003F046FE83460891B8F1000F4EDD4FF02C
:1069B000FF322046294604F067FC22462B4604F0AD
:1069C0001DF9804600988A4660B3DDE90401414A1A
:1069D000414B04F013F9099100905A464046514644
:1069E000089B03F025FE32463B4604F007F9099B5D
:1069F000009A03F01DFE4246534604F033FA224645
:106A00002B4604F021FB04460D46DDE90401334A20
:106A1000334B04F0F3F810B022462B46BDE8F04D9E
:106A200004F012BB5A464046089B03F001FE324672
:106A30003B4604F0E3F84246534604F013FA10B024
:106A400022462B46BDE8F04D04F00CBA009840B346
:106A5000DDE904011F4A204B04F0D0F880468A4645
:106A60005A4620462946089B04F0EEFA32463B4639
:106A700004F0C4F84246534604F0E6FA22462B4698
:106A800004F0E2FA04460D46DDE90401134A144B12
:106A900004F0B4F810B022462B46BDE8F04D04F0E7
:106AA000D3BA0B465A462046294604F0CDFA324660
:106AB0003B4604F0A3F810B022462B46BDE8F04D4B
:106AC00004F0D0B90000F07F645F09000000F03FDF
:106AD0000A5F0000763C7935EF39EA3D0000E0FEC0
:106AE000422EE63F5555D53F0000E03F86EBF9FFCB
:106AF0001A5D0000185D00001CB54FF470314FF0B6
:106B00000060FAF75BFFFFF73BFA4FF44070FAF7CB
:106B10004BFF0E48FAF75EFB0D48FAF745FB0D48B0
:106B2000FAF74CFB0C48FFF731F9FFF729FA0B484D
:106B30002021CDE90010CA00002309A10B4803F071
:106B400085FA02F013FE00201CBD0000560B002049
:106B500058000020130700202465030004000020D3
:106B600073746172745F7461736B0000193C040884
:106B70002DE9F04107460878234E5B2803D03160A9
:106B80000020BDE8F0810520F860481C02F0B8FA4A
:106B9000044620785D2811D0FFF744FC0546B86014
:106BA00070B1204602F0ACFA0146284600F084FAA3
:106BB00002F0A6FA0446200004D016E0601CE0E7CC
:106BC0000020DEE70020DCE7FFF72CFCB0B12860F6
:106BD00045600546601C02F093FA0146284600F025
:106BE0006BFA02F08DFA044654B120782C28EBD0D1
:106BF00020785D2806D034600020C2E70020C0E77E
:106C00000020BEE7601CBCE7D00100200178A1F1A4
:106C10003002092A01D811460AE0A1F14102052AF1
:106C200001D8373904E0A1F16102052A0AD85739A1
:106C30000A01401C0178A1F13003092B04D8303A35
:106C400011440EE000207047A1F14103052B02D84A
:106C5000373A114405E0A1F16103052B0BD8573AEF
:106C600011440A01401C0178A1F13003092B04D81A
:106C7000303A11440EE000207047A1F14103052B8A
:106C800002D8373A114405E0A1F16103052B0AD877
:106C9000573A114409014078A0F13002092A04D87A
:106CA00030390844704700207047A0F14102052A9E
:106CB00002D8373908447047A0F16102052A02D88A
:106CC0005739084470470020704700002DE9F34F02
:106CD00085B08A460024254659490020CDE90201A5
:106CE000002637468346012001909AF800002D289F
:106CF00005D154490020CDE902010AF1010A9AF8B0
:106D00000000302801D10AF1010A9AF80000313858
:106D1000082817D89AF80000303803F008FF80469A
:106D200089460022484B2046294603F067FF424629
:106D30004B4603F07DFC04460D461AF8010F30382F
:106D40000928E7D99AF800002E2827D19AF80100DF
:106D5000302823D3392821D80AF1010A9AF80000F3
:106D6000303803F0E4FE804689460022364B204648
:106D7000294603F043FF42464B4603F059FC0446C4
:106D80000D4600222E4B3046394604F05DF906468A
:106D90000F461AF8010F30380928DFD99AF8000099
:106DA000652801D045281DD11AF8010F2B2802D0E3
:106DB0002D2803D010E00AF1010A0DE04FF0FF305A
:106DC00001900AF1010A07E00BEB8B0100EB410B8C
:106DD0000AF1010AABF1300B9AF80000A0F1300182
:106DE0000929F1D901980BFB00F003F0A0FE32460F
:106DF0003B4603F01DFC02460B460020124900F002
:106E000039FA06460F46DDE9020122462B4603F019
:106E1000F5FE32463B4603F0F1FE04460D4605986A
:106E2000C0E906452046294603F052FE059948610F
:106E300005980321C16007B05046BDE8F08F0000FF
:106E40000000F03F0000F0BF000024402DE9F041B9
:106E500007460878384E7B2803D031600020BDE813
:106E6000F0810620F860481C02F04AF905462878AF
:106E70007D2818D0FFF7D6FA0446B860A8B1284696
:106E800002F03EF90146204600F058F802F038F9C9
:106E900068B1216921620027276101783A2908D069
:106EA00030600020DBE7681CD9E70020D7E700202E
:106EB000D5E7401C02F024F90146204600F0FCF81A
:106EC00002F01EF90546280028D1C8E7FFF7AAFA04
:106ED000A8B1206044600446681C02F011F9014624
:106EE000204600F02BF802F00BF950B12169216225
:106EF000276101783A2906D030600020AFE70020F2
:106F0000ADE70020ABE7401C02F0FAF8014620464E
:106F100000F0D2F802F0F4F8054645B128782C28A4
:106F2000D4D028787D2804D03560002097E7002051
:106F300095E7681C93E70000D00100202DE9F04799
:106F400080460D466C1C00202978222908D058481C
:106F500005600020BDE8F087641C5C2A00D1641C39
:106F60002278222A02D00AB1401CF5D1401C00F040
:106F700005F90746380004D0681C3C464FF4806988
:106F80001AE00020E6E75C2903D004F8011B401C4E
:106F900012E0461C3078722825D006DC622816D014
:106FA000662818D06E2804D119E074281FD07528DF
:106FB00021D004F8010B701C0178222901D000298E
:106FC000E1D100212170017822296AD06AE00820ED
:106FD00004F8010BEFE70C2004F8010BEBE70A20A3
:106FE00004F8010BE7E70D2004F8010BE3E70920A3
:106FF00004F8010BDFE7701CFFF708FE0546361D9D
:10700000A5F55C404845D6D3002DD4D0A5F5584011
:10701000484513D270785C28CDD1B0787528CAD194
:10702000F01CFFF7F3FDB61DA0F55C414945C2D247
:10703000C5F3090161F39F2000F580350421802DFF
:1070400001D2012108E0B5F5006F01D2022103E071
:10705000B5F5803F00D20321601801291AD002291A
:1070600011D0032908D0042919D105F0BF0242F03C
:10707000800200F8012DAD0905F0BF0242F0800248
:1070800000F8012DAD0905F0BF0242F0800200F8C2
:10709000012DAD09074A525C2A4300F8012D44181E
:1070A00089E7401CC8F810700421C8F80C1051E79B
:1070B000D001002094B3040870B505460C46002C9E
:1070C00020D0042224A12046F5F7C1FCE0B105221E
:1070D00023A12046F5F7BBFCD0B1042222A1204613
:1070E000F5F7B5FCC0B1207822281AD02D2803D09E
:1070F000A0F1300109291AD821462846BDE8704080
:10710000FFF7E4BD002070BD0220E860201D70BDC7
:107110000020E860601D70BD0120E8606861201DEE
:1071200070BD21462846BDE87040FFF707BF5B28C9
:1071300005D07B2809D00E480460002070BD214690
:107140002846BDE87040FFF713BD21462846BDE83C
:107150007040FFF77BBE00006E756C6C0000000095
:1071600066616C7365000000747275650000000054
:10717000D001002001460020FAF708BB70B5064692
:1071800031460020FAF70EFB04460020FAF7BCFB5C
:1071900005464B2D08D9182215A11CA0F5F720F99A
:1071A00029461EA0F5F71CF924B131462046F5F713
:1071B00024FD1BE020220EA114A0F5F711F92946A9
:1071C0001EA0F5F70DF90020FAF732FB314600203A
:1071D000FAF7E8FA04464CB9252205A10BA0F5F709
:1071E000FFF823A0F5F7FCF8FDF730FB204670BD53
:1071F0002E2E5C53595354454D5C535953504F52A6
:10720000545C737973706F72742E63004C6F6745B2
:1072100072723A2025732C25640000000D0AB6AF67
:10722000CCACC4DAB4E6D5BCD3C3D2D1B3ACB9FDCF
:10723000A3BA25642525A3A10D0A00000D0AC4DA0E
:10724000B4E6D5BCD3C3A3BA256425252D2DB6AF8E
:10725000CCACC4DAB4E6D2E7B3F6A3A1B3F5CABCAA
:10726000BBAFB6AFCCACC4DAB4E6BFD5BCE4A3A127
:10727000000000002DE9F04D1D460C4698B0174661
:1072800021F0004123F00043002814BF4FF0010C0F
:107290004FF0000C0CEB440CFE4A0CEB02064FEADC
:1072A000620C66452BD33E0018BF012606EB45064F
:1072B0001644F94A964222D3F84A53EA070C02D000
:1072C000944205D148B918B000201146BDE8F08DB0
:1072D000002808BF4FF0000C01D04FF0010C0CEB60
:1072E000440212F5001F0AD8002F14BF4FF0010C02
:1072F0004FF0000C0CEB450212F5001F07D918B037
:107300003A462B462146BDE8F04DFEF7FEBF00226F
:10731000DFF88CA3002CB8BF534526DADFF884C30E
:107320006345A8BF022220DADFF870C39C451CDC4D
:10733000DFF874C30CEB235CBCF1140F08DDCCF157
:10734000340627FA06FC0CFA06F6BE420DD108E018
:107350005FB9CCF1140623FA06FC0CFA06F69E423D
:1073600003D10CF00102C2F1020251EA000C19D162
:10737000002D17DA002C18BF022A01D0012A07D0ED
:107380000220F5F7C4FC18B0BDE8F04DFEF7B2BF1F
:107390000220F5F7BCFCFEF7ADFF18B081F000410C
:1073A000BDE8F08DB7F1000C6CD1534525D104F147
:1073B000804212F5801201BF00280020B74918B0A2
:1073C00008BFBDE8F08DB548884207DC002DA1BF9D
:1073D0006046294618B0BDE8F08D07E0281E05DAA2
:1073E00080F0004118B06046BDE8F08DAF497944A7
:1073F000D1E9000118B0BDE8F08DDFF8A0C2634507
:1074000025D1002D1FDA19B1514512D1D8B909E0A3
:10741000002840F0EC82A24A214618B062F31E0117
:10742000BDE8F08D0020214618B060F31E01BDE8D4
:10743000F08D08DA18B02346BDE8F04D0246002072
:10744000614603F0B1B918B02146BDE8F08D514551
:1074500018DAB5F1804F0DD0A5F1005CBCF1FF5CEE
:1074600010D1B4F1000C0DDB18B06146BDE8F04D51
:1074700001F050BE234618B00246BDE8F04D194653
:1074800003F0BCBB060024F0004C3BD1D9B1514500
:1074900033D1002C06DD002DA1BF0020514618B0CD
:1074A000BDE8F08D002C01DD002D1BDB002C13DA74
:1074B000002D11DB012A4FF0000014BF78497C49F0
:1074C00018B0BDE8F08D022A18BF002C0AD0012A9E
:1074D00008D1002C06DA0AE0002CB8BF002D11DA22
:1074E000012A04D0002018B00146BDE8F08D18B084
:1074F00000204FF00041BDE8F08DA1F14050B0F107
:107500007F601AD0012000EBE47050EA020421D021
:10751000624C521E4FF0000B104304BF4FF0000BA3
:10752000644C654883427CDD644A654893421FDDB4
:10753000884217DB002D25DB37E0002C00DA4AB14A
:10754000022A0CBF01204FF0FF3018B0BDE8F04D0B
:1075500003F0EDBA0120F5F7DAFB18B0BDE8F04D05
:10756000FEF7D5BE4D4A8A4202DC002D0ADC1CE043
:10757000814202DA002D18DA04E0484B994220DDFE
:10758000002D12DD0220F5F7C2FBFEF7C6FE054610
:107590000E46002253465846214603F02FFB18B0F2
:1075A00066F31E012846BDE8F08D0220F5F7AFFB1B
:1075B000FEF7BAFE0A46214618B062F31E01BDE886
:1075C000F08D00223046614603F03EFD80460E46B7
:1075D0006FF0010203F058FE4FF05532394B03F0C3
:1075E00041FC4246334603F009FB0022364B03F0D0
:1075F00039FC82464246334604911046194603F050
:10760000FDFA5246049B03F0F9FA8A4600904FF0C7
:10761000C0422E4B4046314603F0F0FA2C4A2B4B29
:1076200000E027E0CDE906015146009803F0E6FAB4
:1076300082460191274A284B4046314603F0DEFA44
:107640005246019B03F000FD82460B46024605911F
:10765000DDE9060102F0ECFFDDE90623002688469D
:10766000304603F0F1FC5246059B03F0FBFB02465B
:1076700000F07EB90020B1F5801F07DA35223046D0
:10768000614603F001FE06466FF0340000EB215026
:1076900024E00000FFFF1F00FFFF0F000000F03F8D
:1076A0000000F07F0000404301FCFFFF5653000044
:1076B0000000F0FF0000F0BF0000E0410000F043D8
:1076C000FFFFEF3F5555D53F0000E03F4715F73F1F
:1076D000FE822B6544DF5DF80BAE543EA0F2FF3016
:1076E0000190C1F3130040F07F6141F040510291DD
:1076F000FE498842D8BF002004DDFD498142C8BF51
:10770000012001DD0D9008E000200D900198401C43
:1077100001900298A0F5801002900299F5487844F3
:107720000B910D9900EBC100D0E900230F93304677
:107730000A920B9903F088FCCDE90601DDE90A21E4
:1077400030460F9B02F074FF02460B460020EA49C8
:1077500003F02AF8059102460B460090DDE9060188
:1077600003F04CFA1490E5488A464FF0000878443C
:107770000299006812904FF0005040EA61010D98A4
:107780000F9B01EB804000F5002109910A9A1298A5
:1077900003F05AFC32460B9B03F064FB424653460F
:1077A00003F02CFA0646029140465146099B129A74
:1077B00003F024FADDE9062303F054FB3246029B72
:1077C00003F042FC059B009A03F018FA0091149A0A
:1077D000049053461046194603F010FA0646024636
:1077E000C7480B46029106217844FEF72DFDCDE9EE
:1077F0000510029B32461046194603F0FFF9DDE9F9
:10780000053203F0FBF905910646534640461946FA
:10781000149A02F00DFF009B049A03F0EFF9324630
:10782000059B02F005FFCDE9051042465346104680
:10783000194603F0E3F90022B24B02910A9002F0DC
:10784000F7FEDDE9053202F0F3FE0E464246AD4B8F
:10785000404603F0F9FB029B0A9A03F0F5FBDDE9D1
:10786000053203F0FFFA424602910A903346104671
:10787000514603F0C3F9CDE906015346149A029923
:107880000A9803F0BBF98A460290334642460099B3
:10789000049803F0B3F95346029A02F0C9FE8246F7
:1078A0000B4602460591DDE9060102F0C1FEDDE965
:1078B000062300208846064603F0C6FB5246059B79
:1078C00003F0D0FA824609914FF060428E4B304669
:1078D000414603F093F9049006918C4A8A4B504636
:1078E000099903F08BF982460291894A894B304607
:1078F000414603F083F95246029B02F099FE864B03
:107900007B440D9A03EBC203D3E9002302F090FEFF
:107910000E900791019803F00AF90591DDE906132D
:1079200082460E9A049802F083FE7C4A7A440D9BAC
:1079300002EBC303D3E900230093029202F078FE26
:107940005246059B02F074FE002688465246304699
:10795000059B03F079FB009B029A03F075FB069BE5
:10796000049A03F071FB079B0E9A03F07BFA024620
:1079700000200B4602903846294603F03FF9824624
:1079800001912B4638461946029A03F05DFB3246B8
:10799000434603F033F95246019B02F049FE074685
:1079A0008A46324643462946029803F027F905469F
:1079B0000E463A46534602F03BFE594A88469142EB
:1079C00021DBA8EB020353EA000210D12A4633461A
:1079D00003F03AFBCDE90401524A534B3846514675
:1079E00002F026FEDDE9042303F006FA21D202208C
:1079F000F5F78DF9FEF791FC0A46214618B062F3BF
:107A00001E01BDE8F08D494B28F000429A4210D388
:107A1000474A08EB020353EA00027FF4C6AD2A4648
:107A2000334603F011FB3A46534603F0E5F97FF67F
:107A3000BCAD0022019228F000403E493E4A01EBD5
:107A40002051824223DA481C4FF4801121FA00F0C1
:107A500040443A4AC0F30A517A44394BA1F2FF310B
:107A6000CB4020EA0303C0F3130040F48010C1F1BF
:107A70001401C84012680190B8F1000FBCBF404229
:107A800001902846314603F0DFFA05460E462A46A5
:107A900033463846514602F0CBFD4FF000084246CF
:107AA000284B4046059103F0A9F8CDE90601264A86
:107AB000264B4046059903F0A1F8009102902A4612
:107AC00033464046059903F0BFFA3A46534603F061
:107AD000C9F91F4A1F4B03F091F8009B029A02F06C
:107AE000A7FD0746884602460B4635E08E98030000
:107AF0007AB60B009E4F00000000F03FD64F00000A
:107B0000044F00000000084009C7EE3FFD033ADCC7
:107B1000F5015B14E02F3EBEDC4D0000A04D0000DF
:107B200000009040FE822B654715973C00CC9040AA
:107B300000346F3F01FCFFFF0000E03FEC4C000011
:107B4000FFFF0F00432EE63F396CA80C615C20BE9E
:107B5000EF39FAFE422EE63FDDE9060102F068FD4C
:107B6000DDE9062305460E4603F06EFA3A46434623
:107B700003F078F90F462A4633460090104619461E
:107B800003F03CF8824602462E4888460B46052103
:107B90007844FEF759FB5246434603F02FF82A4635
:107BA000334603F05FF980468A463B462846314615
:107BB000009A03F023F83B46009A02F039FD069143
:107BC000009000224FF080434046514603F03CFABB
:107BD0000F460C90424653462846314603F00EF8B5
:107BE0003B460C9A02F0E0FD069B009A03F02CFA4B
:107BF0002A46334603F028FA0022134B03F032F9E9
:107C0000054601980E4601EB00510815002810DCCE
:107C100028463146019A03F037FBFEF701FB0428A2
:107C200008BFFEF781FB28463146019A03F02CFB82
:107C300005460B4618B02A4658462146BDE8F04D89
:107C400002F0DCBF8C4B00000000F03F401E40EA19
:107C5000600040EAA00040EA201040EA202040EA0C
:107C60002040401C704700002DE9FF4F81B0834643
:107C700090461F464FF000094FF0050ADBF8080058
:107C800000260025002401E0761C00680028FBD1B6
:107C90007EB1002F61D0BE6801213846FEF74BFC53
:107CA000D8B15B210170B868401CB860DBF808509F
:107CB0003FE02FB103213846FEF73DFC044603E0C8
:107CC0000320FFF75BFA04461CB163A12046F4F7DA
:107CD00070FE204605B0BDE8F08F0020FAE702995B
:107CE0003B464246491C284600F00EFC384601F04F
:107CF0003AFAB8602868D8B1B8F1000F02D04FF056
:107D0000020901E04FF0010909F101013846FEF7CF
:107D100012FCF0B12C2100F8011BB8F1000F02D0C9
:107D2000202100F8011B00210170B8684844B860A8
:107D30002D680DB1002CD2D002213846FEF7FBFB96
:107D400048B15D21017000214170386800EB0609DF
:107D50007FE00020BEE70020BCE7B0000090FFF706
:107D60000DFA0746380005D00099F4F768FFDBF8F4
:107D700008B01EE00020ADE7029900234246491CEE
:107D8000584600F0C1FB29466D1C47F8210068B138
:107D9000F4F73EFE0146B8F1000F01D0012000E0EB
:107DA0000020084482440AF1020A00E00124DBF8C2
:107DB00000B0BBF1000F01D0002CDDD01CB9504643
:107DC000FFF7DCF98146B9F1000F00D1012474B14D
:107DD000002405E057F8240008B1FFF7CBF9641C34
:107DE000B442F7DB3846FFF7C5F9002072E75B20A5
:107DF00089F800004C464FF0000A04F801AF002556
:107E00001EE057F82500F4F703FE834657F82510C7
:107E10005A462046F4F772FE5C44701E85420AD032
:107E20002C2004F8010BB8F1000F02D0202004F838
:107E3000010B84F800A057F82500FFF79BF96D1C93
:107E4000B542DEDB3846FFF795F95D20207084F8F7
:107E500001A048463EE700005B5D00002DE9F047C9
:107E600007460E46DFF83481D7E90645002213465F
:107E70002046294602F0F0FD12D12EB102213046F3
:107E8000FEF759FB814603E00220FFF777F98146B0
:107E9000B9F1000F7ED042A00088A9F8000079E077
:107EA000786902F044FE22462B4603F0CDF821F01B
:107EB00000410022434602F065FE21D8394A3A4B80
:107EC0002046294602F05EFE1AD80022374B204693
:107ED000294602F091FF13D82EB115213046FEF746
:107EE0002AFB814603E01520FFF748F98146B9F1E6
:107EF000000F4FD02EA148467A69F4F77DFA49E089
:107F00002EB140213046FEF716FB814603E04020AB
:107F1000FFF734F98146B9F1000F3BD020462946DE
:107F2000FEF734FB22462B4603F08EF821F0004189
:107F30000022434602F026FE0ED825F000412046DE
:107F40001C4A1D4B02F01EFE06D222462B461BA1E8
:107F50004846F4F751FA1DE0204625F00041064658
:107F60000F46184A184B02F00DFE06D3304639462C
:107F70000022164B02F040FF06D222462B4614A1E7
:107F80004846F4F739FA05E022462B4611A1484647
:107F9000F4F732FA4846BDE8F08700000000B03C34
:107FA000300000000000C0FFFFFFDF410000E0C123
:107FB0002564000044F3C2E4E4E9634C252E3066F6
:107FC000000000008DEDB5A0F7C6B03E65CDCD41F7
:107FD00025650000256600002DE9F04F85B00646B6
:107FE000894615461C4600200490072002904FF059
:107FF000000BB06800270021019101E07F1C0068A0
:108000000028FBD137B1002C70D0A76895B34FF092
:10801000020A32E04CB115B109F1040100E003217C
:108020002046FEF788FA024607E015B109F1040080
:1080300000E00320FFF7A2F8024662B110467B2160
:1080400000F8011B85B10A2100F8011B002109235A
:10805000A9F1010906E0002005B0BDE8F08F00F8A5
:10806000013B491C4945FADB7D210170002141702B
:108070001046F1E7FFE74FF0010A0AF1010120463F
:10808000FEF759FA88B17B2100F8011B15B10A21CE
:1080900000F8011B4FF0000880F80080A0685044F1
:1080A000A060B66809F101095DE00020D4E78DB158
:1080B00049462046FEF73FFA10B10021092204E0AC
:1080C0000020C9E700F8012B491C4945FADBA068EC
:1080D0004844A0602146306A00F044F9204601F08F
:1080E00042F8A0601DB14FF0020A02E05DE04FF0DF
:1080F000010A51462046FEF71EFAA8B13A2100F8BF
:10810000011B0DB109210170A0685044A0602346F5
:108110002A464946304600F0F7F9204601F023F898
:10812000A0601DB1012002E0002095E70020316829
:1081300009B1012100E0002100EB010A0AF101016F
:108140002046FEF7F8F9A0B1316811B12C2100F8F2
:10815000011B15B10A2100F8011B80F80080A068FE
:108160005044A0603668002EA1D125B109F101016B
:1081700002E0002070E702212046FEF7DCF928B17A
:108180005DB100270921A9F1010904E0002063E79E
:1081900000F8011B7F1C4F45FADB7D21017080F840
:1081A0000180206838440490D7E0BC002046FEF7E8
:1081B000E5FF80465FEA080016D02046FEF7DEFFA6
:1081C00082465FEA0A0011D021464046F4F737FDA7
:1081D00021465046F4F733FDB46809F101098DB327
:1081E00002984844029031E0002035E74046FEF70F
:1081F000C1FF002030E70021206A00F0B3F80390AF
:108200004AF82B0000232A464946204600F07CF914
:1082100059460BF1010B48F82100039999B190B12F
:10822000F4F7F6FB06460398F4F7F2FB311815B1A4
:1082300009F1020000E00020014402980844801C7B
:10824000029002E002E0012001902468002CD2D1CB
:10825000019818B90298FEF791FF0490049808B9A4
:10826000012001900198B0B100240AE05AF82400DE
:1082700008B1FEF77FFF58F8240008B1FEF77AFF37
:10828000641CBC42F2DB5046FEF774FF4046FEF72A
:1082900071FF0020E0E604997B200870049C641CB8
:1082A00015B10A2004F8010B4FF0000B84F800B060
:1082B00000263BE03DB10020092102E004F8011B4B
:1082C000401C4845FADB5AF82600F4F7A1FB009061
:1082D0005AF826102046009AF4F710FC009804443F
:1082E0003A2004F8010B15B1092004F8010B58F8E5
:1082F00026102046F4F75DFB58F82600F4F788FBBB
:108300000444781E864202D02C2004F8010B15B1DB
:108310000A2004F8010B84F800B05AF82600FEF792
:1083200029FF58F82600FEF725FF761CBE42C1DB68
:108330005046FEF71FFF4046FEF71CFF4DB10020E0
:108340000921A9F1010902E004F8011B401C48457C
:10835000FADB7D20207084F801B004987CE6006987
:10836000AFF300802DE9F04705468A46002400213E
:10837000A9460AE0421E1F2A11D322280FD05C28EA
:108380000DD00020014309F1010999F800000028EF
:10839000F0D18046222721B12DB32E4645E00120A1
:1083A000F0E7A9EB0506BAF1000F05D0F11C504625
:1083B000FEF7C1F8044603E0F01CFEF7DFFE0446BA
:1083C0007CB1277004F1010929464846F4F7F1FA17
:1083D00009F8067009EB060080F801802046BDE828
:1083E000F0870020FBE7BAF1000F05D003215046CB
:1083F000FEF7A1F8044603E00320FEF7BFFE0446A3
:108400002CB13CA12046F4F7D4FA2046E7E700203F
:10841000E5E7494638A0F4F784FA08B1641C03E0A4
:10842000B9F1200F00D2641D761C96F80090B9F1C6
:10843000000F01D0641CECD1BAF1000F05D0E11C93
:108440005046FEF778F8064603E0E01CFEF796FE7D
:1084500006462EB1304600F8017B4FF05C0925E05E
:108460000020BCE71F2907D9222905D05C2903D0A9
:1084700000F8011B6D1C19E000F8019B044615F87B
:10848000012B0C2A25D006DC082A1ED0092A2CD064
:108490000A2A06D121E00D2A23D0222A12D05C2AF2
:1084A0000CD017A12046F3F7A7FF601D29780029FB
:1084B000D8D1077080F80180304690E784F80090AA
:1084C000601CF3E72770601CF0E762202070601CDE
:1084D000ECE766202070601CE8E76E202070601CCE
:1084E000E4E772202070601CE0E774202070601CBC
:1084F000DCE7000022220000225C080C0A0D0900C3
:10850000752530347800000070B50024002809D0AB
:1085100093B3057B072D68D2DFE805F0121E06290C
:108520002F343800002070BD05211846FEF703F8EF
:108530000446002C59D02EA12046F4F73AFA54E014
:1085400006211846FDF7F7FF0446002C4DD02AA15E
:108550002046F4F72EFA48E005211846FDF7EBFF18
:10856000044624B326A12046F4F723FA3DE0194639
:10857000FFF774FC044638E00CE01946FFF7EFFE05
:10858000044632E0FFF770FB04462EE0FFF724FDBF
:1085900004462AE0037B072B27D2DFE803F0090E0D
:1085A0000413181D220012A0FDF7A9FF04461CE0C9
:1085B00011A0FDF7A4FF044617E011A0FDF79FFFEF
:1085C000044612E00021FFF749FC04460DE00021BB
:1085D000FFF7C5FE044608E00023FFF745FB04460D
:1085E00003E00023FFF7F8FC0446204670BD0000BE
:1085F0006E756C6C0000000066616C7365000000B5
:1086000074727565000000002DE9F04104460F46C4
:10861000174EF5683068001D00F0B4FD38B93068B9
:1086200090F82C1001208840316981433161601C31
:1086300007D137B13168BDE8F041091D0D4800F0A0
:10864000D9BD2C4430684460AC4206D23168B06B6E
:10865000091DBDE8F04100F0B5BD3168706B091D22
:1086600000F0B0FDB06A844200D2B462BDE8F0818F
:108670007406002020B7002070B5044600F0C6FD47
:108680001D4DA868401CA860286810B1686938B101
:108690000CE02C60A868012808D100F0DBF905E0A7
:1086A0002868E16AC06A884200D82C60686A401C69
:1086B00068626064E06A01212A698140114329618E
:1086C0000E4900EB800001EB8000211D00F092FDBF
:1086D00000F0D8FD686900280CD02868E16AC06AFB
:1086E000884207D206494FF080500860BFF34F8F91
:1086F000BFF36F8F70BD00007406002050B40020DF
:1087000004ED00E010B500F081FD0E4C2068A0B92A
:108710000D4800F049FD0C48143000F045FD0A48B2
:10872000E0601430206100221021052001F0B0F932
:10873000206010B105A100F07BFEBDE8104000F004
:10874000A1BD0000B006002034B70020546D725166
:108750000000000070B5124E124D1CE001F050F800
:10876000306820B1002401F021FEA4B901E0012409
:10877000F9E700F04BFDF068C468201D00F002FD31
:10878000A868401EA8606868401E686000F07AFD16
:10879000204600F054F868680028DFD170BD000062
:1087A0000CB700207406002030B40B46026C002A7F
:1087B0000CD0C1681144C1604468A14201D3016872
:1087C000C160C16830BC1846F4F798B930BC704736
:1087D0002DE9F041044617460026A56B226C002ABD
:1087E00010D0C7B1E068F4F789F9E168206C091A84
:1087F000E1602268914202D26168081AE060022FAB
:1088000016D017E02068A8B9606801F0D9FC0646C8
:10881000002060600EE0A068F4F770F9216CA06899
:108820000844A0606168884204D32068A06001E029
:1088300005B16D1E6D1CA5633046BDE8F08110B515
:108840000446206B00F052FD2046BDE8104000F0C9
:108850004DBD00000749CA681168002904D00021F5
:10886000016019B1002070470121F9E7D068006864
:1088700070470000B00600204FF4B0410F48420797
:1088800006D0C01D20F007000C49411AC1F5B041C7
:108890000B4A1060002353600144083921F007019E
:1088A000103A11604B600B600B1A43600160406826
:1088B000906050604FF00040D0607047105C002026
:1088C00060060020074E4FF08054074DFFF742FF2F
:1088D00030680128FAD92C60BFF34F8FBFF36F8F38
:1088E000F4E7000050B4002004ED00E0002808D0B8
:1088F000002141600160C16000231A46194601F061
:108900001FBA704770B51D46049C00290BD0226029
:10891000E06321640121204601F0BCF984F8505045
:108920000020A06470BD2460F2E700002DE9F0474C
:10893000DDE908580A9C81460E4617469A46B9005A
:10894000A522206BF4F751F9206B7F1E00EB870006
:1089500020F00707780705D040F22E3219A11EA09B
:10896000F3F73EFD00202218315C82F83410315CB0
:1089700011B1401C1028F6D3002684F84360202D46
:1089800000D31F25E562E5642665201D00F017FC75
:1089900004F1180000F013FC2461C5F12000A0616F
:1089A0006462666584F8586052464946384600F06D
:1089B00099FB2060B8F1000F01D0C8F80040BDE875
:1089C000F08700002E2E5C4672656552544F535C52
:1089D0007461736B732E63004572726F723A257304
:1089E0002C25640D0A0000002DE9F047DDE908940C
:1089F00006460D4617469846002D05D14FF4C6721F
:108A00000AA110A0F3F7ECFC002C0DD0FFF77AFEC2
:108A10002660A561E761C4F82080C4F82490201D79
:108A2000BDE8F04700F0CBBBBDE8F0872E2E5C46DA
:108A300072656552544F535C74696D6572732E6331
:108A4000000000004572726F723A25732C25640D88
:108A50000A00000070B50024114D04EB840005EB02
:108A6000800000F0A1FB641C202CF6D30D4800F020
:108A70009BFB0C48143000F097FB0A48283000F0AC
:108A800093FB08483C3000F08FFB0648503000F064
:108A90008BFB0548034941631431816370BD0000BD
:108AA00050B40020D0B600207406002030B5134921
:108AB00000E011460A688242FBD34B685C1884428E
:108AC00003D140681844486008460D68446823187C
:108AD000AB420DD1094B103B1B689A4206D052683D
:108AE000224442600A681268026002E0036000E00B
:108AF0000260814200D0086030BD000060060020A6
:108B000070B50024416000610C4D91420AD8D11A21
:108B10008269914201D301240EE0011D286900F011
:108B200051FB09E09A4203D2994201D3012403E0A8
:108B3000011DE86800F046FB204670BDB00600202D
:108B400010B5044600F062FBA06B20B1002400F0D9
:108B500099FB204610BD0124F9E710B5044600F04A
:108B600055FBA06BE16B884201D1012400E0002499
:108B700000F088FB204610BD2DE9F3410F46009818
:108B8000846C0026002C05D140F6CE1216A11BA045
:108B9000F3F726FCA06BE16B884205D340F6CF12B9
:108BA00011A116A0F3F71CFCA06BE16B88420CD25C
:108BB00094F945503A4669462046FFF709FE0646B5
:108BC000681C05D06D1C84F845503046BDE8FC811A
:108BD000606A0028F9D004F1240001F04BFB002862
:108BE000F3D00126F1E700002E2E5C467265655237
:108BF000544F535C71756575652E63004572726FD5
:108C0000723A25732C25640D0A000000F8B505465C
:108C10000E461348C068C068C468201D00F0B2FA50
:108C2000E069012816D1A0692B4641193246204639
:108C3000FFF766FF70B100200346014600902A4608
:108C4000204601F07BFC28B94FF4027205A10BA06D
:108C5000F3F7C6FB616A01B02046BDE8F040084763
:108C6000B00600202E2E5C4672656552544F535C50
:108C700074696D6572732E63000000004572726F37
:108C8000723A25732C25640D0A00000070B586B079
:108C90002F4E53E00298002803DADDE903200599FE
:108CA00090470298002849DB049C606910B1201DA0
:108CB00000F068FA01A800F0A9F8054602980A2811
:108CC0003CD2DFE800F00505053B273805053B27CA
:108CD0000398A169034601442A462046FFF710FF86
:108CE00000282BD0616A20468847E069012825D1F9
:108CF000002000900398A1690023421819462046DD
:108D000001F01CFCD0B940F2213212A117A0F3F7F8
:108D100067FB13E00398A06128B94FF44E720DA1D0
:108D200012A0F3F75DFBA0692B4641192A462046A5
:108D3000FFF7E6FE02E0204600F0D8FA00231A46CC
:108D400002A9306800F0D6FE0028A3D106B070BD9D
:108D5000B00600202E2E5C4672656552544F535C5F
:108D600074696D6572732E63000000004572726F46
:108D7000723A25732C25640D0A000000F8B50646EA
:108D80000D4600F03DFD684600F040F804460098AE
:108D900010B101F00BFBF8BD45B9A64206D801F0B1
:108DA00005FB21463046FFF731FFF8BD0C481DB1E9
:108DB0000169096891B10025311B2A46006800F05D
:108DC00049FB01F0F3FA0028EFD106494FF080503B
:108DD0000860BFF34F8FBFF36F8FF8BD0125EBE73E
:108DE000B006002004ED00E00748416B0968002947
:108DF00005D0416BC968C9684968816270474FF006
:108E0000FF318162704700007406002070B505468E
:108E100001F05AF90446074EB068844204D200F0CB
:108E20000BF80120286001E000202860B460204693
:108E300070BD0000B0060020F8B5184E25E0C068EF
:108E40000568C468201D00F09DF9616A20468847C6
:108E5000E069012819D1A0692844A84206D96060B8
:108E60002461211DF06800F0ADF90EE000200346FA
:108E7000014600902A46204601F060FB28B940F2E6
:108E8000923207A10CA0F3F7ABFAF0680168002951
:108E9000D5D1F0683169F1603061F8BDB0060020CD
:108EA0002E2E5C4672656552544F535C74696D6535
:108EB00072732E63000000004572726F723A257360
:108EC0002C25640D0A00000008484068401C04D0AE
:108ED000F52207A111A0F3F783FA502080F311883F
:108EE000BFF34F8FBFF36F8FFEE7000068060020CF
:108EF0002E2E5C4672656552544F535C706F7274CF
:108F000061626C655C525644535C41524D5F434D07
:108F1000335C706F72742E63000000004572726FD4
:108F2000723A25732C25640D0A00000008B56846C6
:108F3000FFF790FC0099FFF721FFFFF7A7FEF6E788
:108F40002DE9F041044600F061F994F9455004F12F
:108F5000240613E0A06C38B100212046FFF70CFE78
:108F600050B100F039FB07E0606A48B1304601F0CB
:108F700081F908B100F030FB6D1E6DB2002DE9DC07
:108F80004FF0FF3684F8456000F07CF900F03EF9C0
:108F900094F9445004F1100709E0206948B13846BB
:108FA00001F068F908B100F017FB6D1E6DB2002DDD
:108FB000F3DC84F84460BDE8F04100F063B90000E0
:108FC0002DE9F0410546002600F01AFC304F3868C4
:108FD00008B9FFF751FCF86805424BD175B1083567
:108FE00068070BD005F00700C0F1080005446807CA
:108FF00004D0C02227A131A0F3F7F2F9002D39D017
:109000007868854236D8224910310846046801E064
:10901000214604466068A84202D220680028F7D1A1
:109020003868844226D00E68083620680860606878
:10903000401B102811D904EB05085FEA487004D0E2
:10904000ED2214A11DA0F3F7CBF96068401BC8F80E
:10905000040065604046FFF729FD61687868401AA2
:109060007860BA68904200D2B860F86801436160E5
:109070000020206001F09AF9700705D040F22D120F
:1090800004A10EA0F3F7ACF93046BDE8F081000072
:10909000500600202E2E5C4672656552544F535C7C
:1090A000706F727461626C655C4D656D4D616E6769
:1090B0005C686561705F342E630000004572726FFA
:1090C000723A25732C25640D0A00000004490868D3
:1090D000002803D00868026D521C026508687047BA
:1090E0007406002020384FF08073C36121F0010125
:1090F00081610249416140F820297047C98E040806
:1091000000E0401C002804D00178002901D020296B
:10911000F7D970472DE9F04106460F4601F0AEFE43
:10912000041E0D4618BF0120284320F00040C0F166
:109130007F6000F1E040C00F0ED0301C18BF01204E
:10914000384320F00040C0F17F6000F1E040C00FE4
:1091500004BF0120F3F7DBFD20462946BDE8F0817E
:1091600001604860704710B50446002C08D02068A4
:1091700030B1A1680844F3F74BFCA168084410BD66
:10918000002010BD0169D0E901329A60D0E90123C5
:109190005A604A68824201D182684A6000220261B4
:1091A0000868401E0860704700F1080141604FF0F8
:1091B000FF328260C16001610021016070470021BF
:1091C0000161704730B50C68621C02D000F10802E2
:1091D00002E0026904E01A4653681D68A542FAD904
:1091E00053684B6099608A60516008610168491C4E
:1091F000016030BD42684A6093688B609368596033
:10920000916008610168491C01607047502080F33B
:109210001188BFF34F8FBFF36F8F09494868401C17
:10922000486001280AD10748006810F0FF0F05D0F8
:109230004FF4C07204A10FA0F3F7D2B8704700003A
:109240006806002004ED00E02E2E5C467265655233
:10925000544F535C706F727461626C655C5256441B
:10926000535C41524D5F434D335C706F72742E639B
:10927000000000004572726F723A25732C25640D50
:109280000A00000010B5094C6068002805D140F2C2
:10929000871207A111A0F3F7A3F86068401E606071
:1092A000002801D180F3118810BD0000680600205D
:1092B0002E2E5C4672656552544F535C706F72740B
:1092C00061626C655C525644535C41524D5F434D44
:1092D000335C706F72742E63000000004572726F11
:1092E000723A25732C25640D0A00000070B5002821
:1092F0002AD008380446154D6068E968084205D14F
:109300004FF4A27212A11CA0F3F76AF8206828B1EA
:1093100040F245120EA118A0F3F762F86068E96800
:10932000084211D02268002A0ED18843606000F004
:1093300067FA60686968084468602046FFF7B6FB12
:10934000BDE8704001F032B870BD0000500600204A
:109350002E2E5C4672656552544F535C706F72746A
:1093600061626C655C4D656D4D616E675C686561E1
:10937000705F342E630000004572726F723A25737D
:109380002C25640D0A000000054864210068B0FB2C
:10939000F1F14FF0E020491E416107210161704762
:1093A0003C06002010B5F2F7CFFF104C10280CD36C
:1093B00000F1E02090F8F0032178884205D240F2D5
:1093C000AE220BA115A0F3F70BF818480068A168AE
:1093D00000F4E060884207D9BDE8104040F2BE22A8
:1093E00003A10EA0F2F7FCBF10BD0000680600202C
:1093F0002E2E5C4672656552544F535C706F7274CA
:1094000061626C655C525644535C41524D5F434D02
:10941000335C706F72742E63000000004572726FCF
:10942000723A25732C25640D0A0000000CED00E053
:1094300010B50022064B53F832401CB1521C082ACA
:10944000F9D310BD43F8321003EBC201486010BDE0
:1094500010B4002070B504460D461646FFF7D6FE40
:1094600094F944304FF000005B1C01D184F84400B3
:1094700094F94510491C01D184F84500FFF702FF1B
:10948000A06B28B93246294604F1240000F0D6F832
:109490002046BDE87040FFF753BD000010B50446FC
:1094A0000020002C10D00E48006B28B140F2D242B0
:1094B0000CA111A0F2F794FF00F0A2F900212046C0
:1094C000FFF7A2F800F072FF002807D10E494FF015
:1094D00080500860BFF34F8FBFF36F8F10BD000047
:1094E000740600202E2E5C4672656552544F535C04
:1094F0007461736B732E63004572726F723A2573D9
:109500002C25640D0A00000004ED00E070B504464F
:10951000FFF77CFE234D04B92C68201DFFF732FEB7
:1095200058B9E06A204A00EB800152F8211021B9B5
:1095300001218140286988432861A06A18B104F19B
:109540001800FFF71FFE686A401C686228688442A2
:1095500007D1211D1548FFF74DFE6868401C686063
:1095600007E0A868401EA8602046FFF768F9FFF7EB
:109570003BFCFFF787FE6869002812D02868844208
:109580000FD1286B28B14FF48D6209A10DA0F2F71D
:1095900027FF10494FF080500860BFF34F8FBFF393
:1095A0006F8F70BD7406002050B400200CB70020EF
:1095B0002E2E5C4672656552544F535C7461736B1A
:1095C000732E63004572726F723A25732C25640DF9
:1095D0000A00000004ED00E001490120C861704765
:1095E0007406002070B504460D46002C05D140F6E7
:1095F0000F3208A10CA0F2F7F3FE0F4801682046D5
:109600001831FFF7DFFD2846BDE870400121FEF765
:10961000FBBF00002E2E5C4672656552544F535CB2
:109620007461736B732E63004572726F723A2573A7
:109630002C25640D0A0000007406002070B5064653
:109640000D461446002E05D140F63A3209A10EA06F
:10965000F2F7C6FE1048016830461831FFF7CAFD20
:109660000CB14FF0FF3521462846BDE87040FEF7AB
:10967000CBBF00002E2E5C4672656552544F535C82
:109680007461736B732E63004572726F723A257347
:109690002C25640D0A0000007406002070B50446F5
:1096A000002839D01D4DE06A2968C96A884233D242
:1096B000A069002804DB2868C06AC0F12000A0610E
:1096C000E06A174E00EB8000616906EB8000814282
:1096D0001FD1201DFFF756FD012150B9E06A00EBB4
:1096E000800256F8222022B92A6901FA00F082434A
:1096F0002A612868C06AE0622A69814011432961B1
:1097000000EB800006EB8000211DBDE87040FFF7F4
:1097100071BD2868C06AE06270BD00007406002058
:1097200050B4002010B50446002C05D140F6CA32D2
:1097300004A109A0F2F754FE0B48016A2160C06839
:10974000606010BD2E2E5C4672656552544F535CAE
:109750007461736B732E63004572726F723A257376
:109760002C25640D0A000000740600201CB5174863
:109770000024CDE900402346822215A1164800F0BE
:1097800065FC012801D100F09FFE01280AD0401C91
:109790001BD102B04FF4F162BDE810400FA114A03C
:1097A000F2F71EBE502080F31188BFF34F8FBFF336
:1097B0006F8F06484FF0FF312C38816201214161E3
:1097C000C460BDE81C4000F007B91CBDA006002025
:1097D00049444C4500000000C58804082E2E5C4614
:1097E00072656552544F535C7461736B732E6300E2
:1097F0004572726F723A25732C25640D0A000000C1
:109800000248016B491C0163704700007406002088
:1098100070B5144D286B002802D00120E86170BD9E
:109820000020E8612869B0FA80F0C0F11F000E4EF8
:1098300000EB800456F8240028B940F6FF220BA163
:109840000FA0F2F7CDFD06EB840041684968416046
:1098500000F10802914201D1496841604068C06846
:10986000286070BD7406002050B400202E2E5C4687
:1098700072656552544F535C7461736B732E630051
:109880004572726F723A25732C25640D0A00000030
:1098900070B50E460446002805D140F2DF120BA138
:1098A00011A0F2F79DFD300E05D04FF4F07207A124
:1098B0000DA0F2F795FDFFF7A9FC256825EA060043
:1098C0002060FFF7DFFC284670BD00002E2E5C46AE
:1098D00072656552544F535C6576656E745F67724E
:1098E0006F7570732E6300004572726F723A257344
:1098F0002C25640D0A00000010B51C20FFF760FB4A
:10990000044624B100202060201DFFF74DFC2046B6
:1099100010BD00002DE9F0418846002504460028CE
:1099200005D140F21D2221A127A0F2F759FD5FEADF
:10993000186005D040F21E221CA123A0F2F750FDB2
:10994000261D06F10807FFF75BFFF068216841EA72
:109950000801216020E046680168002201F07F4391
:1099600021F07F415FEA431C06D4D4F800C01CEA12
:10997000010F07D0012205E0D4F800C031EA0C0C39
:1099800000D101223AB1DA0100D50D43216841F03E
:10999000007100F0BDFC3046B842DCD12068A8431D
:1099A000206000F003FD2068BDE8F0812E2E5C46AB
:1099B00072656552544F535C6576656E745F67726D
:1099C0006F7570732E6300004572726F723A257363
:1099D0002C25640D0A0000001CB519490878019077
:1099E000FF200870087800909DF80000154A00F0EC
:1099F000500010700720906006E09068401E906054
:109A00009DF80000400000909DF800000006F4D48E
:109A1000107A000200F4E0609060019808700A4833
:109A2000016841F470010160016841F0704101601A
:109A3000FFF7AAFC00205060F2F750FC00201CBD8C
:109A400000E400E06806002020ED00E010B55020A2
:109A500080F31188BFF34F8FBFF36F8F00F03AFB95
:109A600018B104494FF080500860002080F311883D
:109A700010BD000004ED00E010B5024600210120F9
:109A800000F006F804462046FEF730FF204610BDE1
:109A9000F8B505460E461746002D05D14FF4C472A1
:109AA0000BA110A0F2F79CFC86B105FB06F0543028
:109AB000FFF786FA04463CB104F154023B463146B6
:109AC00028460094FEF71EFF2046F8BD0020EEE772
:109AD0002E2E5C4672656552544F535C71756575E8
:109AE000652E63004572726F723A25732C25640DE2
:109AF0000A0000002DE9FF4F83B004468A469B46CA
:109B00000026002C05D140F2DC4258A15CA0F2F7FF
:109B100067FCBAF1000F07D1206C28B140F2DD429A
:109B200052A157A0F2F75CFC00F0C0FA38B90598D2
:109B300028B14FF49C624DA151A0F2F751FC4FF0B7
:109B400000094FF08057DFF84881FFF75FFBA56BF6
:109B500095B3E66851462046FEF726FEBBF1000F9E
:109B600013D0E660606A50B104F1240000F082FB7B
:109B700028B1C8F80070BFF34F8FBFF36F8FFFF7A6
:109B800081FB012007B0BDE8F08F6D1EA563206842
:109B900010B9FFF79BFA606020690028EFD004F14C
:109BA000100000F067FB0028E9D0C8F80070BFF390
:109BB0004F8FBFF36F8FE2E7FFE7059808B126B13B
:109BC00007E0FFF75FFB0020DCE701A8FFF7AAFD35
:109BD0000126FFF757FBFFF713FEFFF717FB94F97A
:109BE0004400401C01D184F8449094F94500401C85
:109BF00001D184F84590FFF745FB05A901A800F0C5
:109C0000DDF958B12046FFF79BF900F0CFFB204665
:109C1000FEF796FF002898D00020B3E72046FEF715
:109C20008FFFE0B1206830B9FFF7F0FA6068FFF706
:109C300035FDFFF727FB04F124000599FFF7D2FC5F
:109C40002046FFF77DF900F0B1FB00287FF47DAFDF
:109C5000C8F80070BFF34F8FBFF36F8F75E72046D2
:109C6000FFF76EF900F0A2FB6FE700002E2E5C46B6
:109C700072656552544F535C71756575652E63004E
:109C80004572726F723A25732C25640D0A0000002C
:109C900004ED00E070B504460D46002C05D140F2FD
:109CA0001B121DA121A0F2F79BFBFFF7AFFAD4E92D
:109CB0000F20216802FB001161600021A16321686F
:109CC000A160E06B2268216C401E00FB0121E16075
:109CD0004FF0FF3084F8440084F8450004F1100090
:109CE0004DB1FFF761FA04F12400FFF75DFAFFF7C9
:109CF000C9FA012070BD21690029F8D000F0BAFA34
:109D00000028F4D00D494FF080500860BFF34F8F0A
:109D1000BFF36F8FEBE700002E2E5C467265655235
:109D2000544F535C71756575652E63004572726F93
:109D3000723A25732C25640D0A00000004ED00E042
:109D40002DE9FF4782B004468A4698460025002C3C
:109D500005D140F2D92254A158A0F2F741FBBAF143
:109D6000000F07D1206C28B140F2DA224EA153A097
:109D7000F2F736FBB8F1020F08D1E06B012805D0ED
:109D800040F2DB2248A14DA0F2F72AFB00F08EF949
:109D900038B9049828B140F2DE2243A147A0F2F777
:109DA0001FFB4FF000094FF08056484FFFF72EFA87
:109DB000A06BE16B884206D3B8F1020F03D0049880
:109DC00060B37DB333E0424651462046FEF700FDC6
:109DD000A16C51B141462046FEF7CEFEC0B13E60B7
:109DE000BFF34F8FBFF36F8F12E0616A51B104F17F
:109DF000240000F03FFA58B13E60BFF34F8FBFF32D
:109E00006F8F05E020B13E60BFF34F8FBFF36F8FC0
:109E1000FFF738FA012006B0BDE8F087FFF732FA05
:109E20000020F8E7FFE76846FFF77CFC0125FFF715
:109E300029FAFFF7E5FCFFF7E9F994F94400401C23
:109E400001D184F8449094F94500401C01D184F874
:109E50004590FFF717FA04A9684600F0AFF830B153
:109E60002046FFF76DF800F0A1FA0020D3E7204666
:109E7000FEF773FE88B104F110000499FFF7B2FBFE
:109E80002046FFF75DF800F091FA00288ED13E6081
:109E9000BFF34F8FBFF36F8F88E72046FFF750F86F
:109EA00000F084FA82E700002E2E5C46726565524F
:109EB000544F535C71756575652E63004572726F02
:109EC000723A25732C25640D0A00000004ED00E0B1
:109ED0002DE9F0470446894615469846002C05D1E1
:109EE00040F29F322CA131A0F2F77AFAB9F1000FBB
:109EF00007D1206C28B14FF4687227A12BA0F2F78C
:109F00006FFAB8F1020F08D1E06B012805D040F2DA
:109F1000A13221A125A0F2F763FAFFF743FA5020FE
:109F2000EFF3118780F31188BFF34F8FBFF36F8F6B
:109F3000A06BE16B884207D3B8F1020F04D0002078
:109F400087F31188BDE8F08794F945604246494699
:109F50002046FEF73DFC701C04D0761C84F845605A
:109F60000120EDE7A06C012648B141462046FEF7EE
:109F700003FE0028F4D0002DF2D02E60F0E7606AD6
:109F80000028EDD004F1240000F074F90028E7D097
:109F9000002DE5D02E60E3E72E2E5C4672656552FB
:109FA000544F535C71756575652E63004572726F11
:109FB000723A25732C25640D0A00000070B5044622
:109FC0000D46002C05D140F6D43216A11AA0F2F7A6
:109FD00007FA2DB940F6D53212A117A0F2F700FA10
:109FE000FFF714F9184AD06829684B1C08D0236879
:109FF000126A934206D06268824203D801240DE0BF
:10A0000000240BE06268801A884206D2081A286091
:10A010002046FFF787FB002400E00124FFF732F918
:10A02000204670BD2E2E5C4672656552544F535CBF
:10A030007461736B732E63004572726F723A25738D
:10A040002C25640D0A000000740600202DE9FF5F36
:10A050008146DDE90E788A4616469B46B000FEF73B
:10A06000AFFF054628000AD05C20FEF7A9FF044692
:10A070000CB1256304E02846FFF738F900E000241E
:10A080008CB10020CDE90240CDE900785B46324634
:10A0900051464846FEF74AFC2046FEF7EDFA0120FD
:10A0A00004B0BDE8F09F4FF0FF30F9E70548416983
:10A0B000002903D0006B18B10020704701207047C1
:10A0C00002207047740600200148C06870470000F5
:10A0D000740600202DE9F04100262E4F386B002831
:10A0E00008D0B869401CB861F86900B10126304653
:10A0F000BDE8F081FD686D1CFD608DB9786B00686E
:10A1000028B140F6DE1224A128A0F2F769F9786B95
:10A11000B96B7963B863386A401C3862FEF764FE35
:10A12000B86ADFF8988085420DD3786B006838B143
:10A13000786BC068C468606885420ED2B86202E07D
:10A140004FF0FF30B8623868C06A00EB800058F802
:10A1500020000128C8D90126C6E7201DFFF712F804
:10A16000A06A18B104F11800FFF70CF8E06A0121A9
:10A170003A6981401143396100EB800008EB8000AF
:10A18000211DFFF737F8E06A3968C96A8842CCD3E5
:10A190000126CAE7740600202E2E5C4672656552C1
:10A1A000544F535C7461736B732E63004572726F0E
:10A1B000723A25732C25640D0A00000050B400206B
:10A1C00070B50446002600283CD01F4D2868844204
:10A1D00005D04FF46D621DA121A0F2F701F9206DA9
:10A1E00028B940F6D26219A11DA0F2F7F9F8206D46
:10A1F000401E2065E26CE16A914223D010BB201D15
:10A20000FEF7C0FF1A4A012150B9E06A00EB800353
:10A2100052F8233023B92B6901FA00F083432B61F4
:10A22000E06CE062C0F12000A061E06A2B6981402F
:10A230001943296100EB800002EB8000211DFEF72D
:10A24000D9FF0126304670BD740600202E2E5C46D4
:10A2500072656552544F535C7461736B732E630067
:10A260004572726F723A25732C25640D0A00000046
:10A2700050B400202DE9F041C068C468002C05D11D
:10A2800040F66A3216A11BA0F2F7AAF804F11800F2
:10A290000746FEF777FF1B4D2A6B012662B1394650
:10A2A0001948FEF7A7FFE06A2968C96A884215D9EC
:10A2B0000120EE61BDE8F081201DFEF763FFE06A3A
:10A2C0002A6906FA00F111432961104900EB800068
:10A2D00001EB8000211DFEF78DFFE4E70020E9E798
:10A2E0002E2E5C4672656552544F535C7461736BDD
:10A2F000732E63004572726F723A25732C25640DBC
:10A300000A00000074060020F8B6002050B40020B7
:10A3100070B506460C461A4D286B002805D140F64C
:10A32000A23218A11CA0F2F75BF844F000403060A4
:10A33000F4682CB940F6AA3212A117A0F2F750F82F
:10A340003046FEF71FFF201DFEF71CFFE06A0126C6
:10A350002A6906FA00F111432961134900EB8000D4
:10A3600001EB8000211DFEF745FFE06A2968C96AFC
:10A37000884202D90120EE6170BD002070BD00004E
:10A38000740600202E2E5C4672656552544F535C55
:10A390007461736B732E63004572726F723A25732A
:10A3A0002C25640D0A00000050B400202DE9F04176
:10A3B000002400272B4D286B002805D140F2EC72B9
:10A3C00029A12EA0F2F70CF8FEF720FF286B401E03
:10A3D0002863286BF0BBA868E0B3DFF8B0800126E3
:10A3E0001DE0D8F80C00C46804F11800FEF7CAFE9E
:10A3F000201DFEF7C7FEE06A2A6906FA00F1114344
:10A400002961234900EB800001EB8000211DFEF74C
:10A41000F1FEE06A2968C96A884200D3EE61D8F883
:10A4200000000028DDD10CB1FEF7DEFCAC6944B1C0
:10A43000FFF750FE00B1EE61641E002CF8D1002041
:10A44000A861E86930B10127124938070860BFF3F5
:10A450004F8F00E001E0BFF36F8FFEF713FF384628
:10A46000BDE8F081740600202E2E5C4672656552B0
:10A47000544F535C7461736B732E63004572726F3B
:10A48000723A25732C25640D0A000000F8B60020EE
:10A4900050B4002004ED00E02DE9FC4706460A9D7B
:10A4A0000F46904699462C20FEF78AFD04463CB1A3
:10A4B000CDE900544B46424639463046FEF794FA01
:10A4C0002046BDE8FC8700001CB50024FEF71AF901
:10A4D0000C48006860B10B481F21001DCDE9001039
:10A4E00000234FF4827208A10948FFF7AFFD04462C
:10A4F0002CB940F2331207A10CA0F1F771FF2046EE
:10A500001CBD0000B0060020546D7220537663001D
:10A510002D8F04082E2E5C4672656552544F535C95
:10A5200074696D6572732E63000000004572726F6E
:10A53000723A25732C25640D0A0000002DE9FF47AF
:10A54000DDF830A005460E46904699460027002DBE
:10A5500005D14FF4D37215A11AA0F1F741FF1D4C9C
:10A560002068F8B10096CDF804800295062E13DA23
:10A57000FFF79CFD022807D000231A466946206891
:10A58000FFF7DEFB07460DE00023524669462068D0
:10A59000FFF7D6FB074605E000234A466946FFF76A
:10A5A00097FC074604B03846BDE8F0872E2E5C467F
:10A5B00072656552544F535C74696D6572732E6396
:10A5C000000000004572726F723A25732C25640DED
:10A5D0000A000000B006002010B500290AD0087853
:10A5E000002807D005487844F3F708FA002801D07E
:10A5F000002010BD0248784410BD0000462700002E
:10A600003E27000010B500290AD00878002807D09E
:10A6100005487844F3F7F2F9002801D0002010BD76
:10A620000248784410BD00002A28000022280000BB
:10A6300010B591EA030F48BF83F0004300F10C8589
:10A64000841A71EB030C05D2121943EB0C03001BA7
:10A6500061EB0C01DFF824E14FEA1154A4EB135C29
:10A660001EEA430F18BF9EEA445F73D023EA0E032D
:10A67000DCF1200E21EA045143F4801332D322FA94
:10A680000CFE10EB0E0023FA0CFE41EB0E01CCF198
:10A69000200E03FA0EFE10EB0E0051F10001B1F591
:10A6A000801FCCF1200E32D201EB045112FA0EF2CF
:10A6B000BDE8104058BF7047401C38BF5FEA4202F7
:10A6C00018BF7047002814BF20F0010041F10001BD
:10A6D0004FEA410313F5001F38BF7047A1F1C04195
:10A6E00000F084BB012A43EB0302ACF1200CDCF147
:10A6F0001F0E32BF4FF0000E23FA0CF310EB0300D5
:10A7000041EB0451B4EB115FD0D0A1EB045101F542
:10A71000801149085FEA300001EB04510ED350F17B
:10A72000000038BF12FA0EFE08D1BDE81040C9E79C
:10A73000401C38BF5FEA4202CAD1C3E7BDE81040FF
:10A740004FEA410313F5001F38BF7047A1F1C04124
:10A7500000F04CBB9EEA445F08D011EA5E0FBDE8F2
:10A76000104004BF01F0004100207047BDE81040D8
:10A7700070B500F0EDFA00BF64FBBE3E0000E0FFE4
:10A7800002494FF0000000F04DBD00BF0000F87F0F
:10A79000491058BFC1F140415B1058BFC3F140435D
:10A7A0008B42EFF3008070472DE9C04130B4DFF8F1
:10A7B000A0C23CEA111418BF3CEA131400F0EC806C
:10A7C00081EA03051CEA111444EAD57418BF1CEA97
:10A7D000131500F0C780A4EB05044FF0004545EACF
:10A7E000C12145EAC32341EA505143EA525304F1DF
:10A7F0007F74994204F500344FEAC0204FEAC22228
:10A8000008BF904200F09C804FEA13650FF240169B
:10A81000765D4FEA134506FB05F7C7F1807706FB27
:10A8200007F74FEAD737A7FB03687642C8F58038A9
:10A83000A7FB06CE38BFA8F1010807FB08E64FF0DA
:10A84000000EA6FB028CE6FB03CEDCF1000CCEF181
:10A85000004E38BFAEF1010EA6FB0C584FF00007BA
:10A860004FF00005E6FB0E87A1FB08C6A0FB07CE54
:10A8700016EB0E0645F10005E1FB076515F1E04E0C
:10A880007EBFA4F580345FEA46066D4116F180076D
:10A8900045F100054FEA17274FEA066647EA0567C4
:10A8A000A6F1DE46B6F1805F4FEA15251FD938467E
:10A8B00024F0010C05EBC471BCF1FE6F01EB0C112F
:10A8C00002D8F0BCBDE8008124425CBF01F5801EC7
:10A8D0009EEAC47F02D4F0BCBDE80081244238D493
:10A8E000F0BCA1F1C041BDE8004100F07FBA4FEAE1
:10A8F000D22242EA43524FEAD323A7FB02864FEA11
:10A90000D02040EA415007FB03661EEA0E0F4FEAD3
:10A91000D12105FB026658BFA6EB0056B6EB0056E8
:10A920004FEA520E4EEAC37E18EB0E0E56EB530E54
:10A93000BDD518EB02085E417F1C55F10005B6E756
:10A940004FF480154FF000074FF000064FF000085D
:10A95000ADE7F0BC4FF0000001F1C04101F0004153
:10A96000BDE8008111EA0C1F0CEA131500D00CE0C1
:10A9700013EA0C1F00F025804FF00000F0BC81EAC4
:10A98000030101F00041BDE80081F0BCBDE80041D9
:10A9900081EA030100F02ABAF0BCBDE8004170B5BD
:10A9A00000F0D6F9097EFC3E00F007B881EA030109
:10A9B0004FF0000001F00041704781EA030100F010
:10A9C00015BAF0BCBDE800414FF0000021497047C6
:10A9D000FFFDFBF9F7F5F4F2F0EEEDEBE9E8E6E464
:10A9E000E3E1E0DEDDDBDAD8D7D5D4D3D1D0CFCDEB
:10A9F000CCCBCAC8C7C6C5C4C2C1C0BFBEBDBCBB24
:10AA0000BAB9B8B7B6B5B4B3B2B1B0AFAEADACAB1E
:10AA1000AAA9A8A8A7A6A5A4A3A3A2A1A09F9F9EF8
:10AA20009D9C9C9B9A9999989797969595949393AA
:10AA3000929191908F8F8E8E8D8C8C8B8B8A898941
:10AA400088888787868585848483838282818180C4
:10AA50000000FF070000F87F51EA030C17D41CF533
:10AA6000801F58BFBCF5801F00F10680994218BFB7
:10AA7000704708BF9042704707D711F5801F58BF35
:10AA800013F5801F19D499427047894270471CF50D
:10AA9000801F08D5BCF5801FF7D58B4218BF7047C3
:10AAA00008BF824270474FF4001C1CEB410F38BFB7
:10AAB0001CEB430F01D28B42704770B500F048F990
:10AAC000922449004FF000514FF08053FFF760BED1
:10AAD0004FEA41034FEA5353A3F58063D3F11E03BA
:10AAE000C8BFD3F1210C0CDD4FF0004242EAC12275
:10AAF00042EA505232FA03FC8CEAE17CACEBE170A2
:10AB00007047102BC4BF0020704703F5787CBCF160
:10AB1000FF3F04D06FF0004282EA2100704770B519
:10AB200000F016F94992248000207047F2E710F0F7
:10AB3000004248BF4042B0FA80F310FA03F10AD055
:10AB4000C3F11D0303F580634FEA415002EB03524A
:10AB500002EBD12170474FF000007047B0FA80F34C
:10AB600010FA03F10AD0C3F11D0303F580634FEA25
:10AB700041504FEA035202EBD12170474FF00000E1
:10AB80007047000051EA030C17D41CF5801F58BF12
:10AB9000BCF5801F00F10680994218BF704708BFBE
:10ABA0009042704707D711F5801F58BF13F5801FDB
:10ABB00019D499427047894270471CF5801F08D507
:10ABC000BCF5801FF7D58B4218BF704708BF824283
:10ABD00070474FF4001C1CEB410F38BF1CEB430FB8
:10ABE00001D28B42704770B500F0B2F89224490050
:10ABF0004FF000514FF08053FFF7CABDDFF848C156
:10AC000070B51CEA111E1EBF1CEA13159EEA0C0F3C
:10AC100095EA0C0F00F06F8081EA030423EA4C13DD
:10AC20004EEAD47E21EA4C1141F4801143F48013A2
:10AC3000AE44A1FB024CA0FB0365AEF17F7E36194A
:10AC400055EB0C05A1FB034C4CF10003A0FB021CCF
:10AC500016EB0C06654153F10003094218BF46F09C
:10AC6000010613F4007F0BD14FEA03314FEA0530A0
:10AC7000340341EA155140EA16506FF003020AE02E
:10AC80004FEAC3214FEAC520F40241EA555140EA98
:10AC900056506FF0020202EB2E4201EB025585EA9C
:10ACA000CE710AD05FEA440C18BF24F0004450F182
:10ACB000000041F1000120EAD47040F2FE7C6245C0
:10ACC00000D270BDA84214BF4FF080444FF0404402
:10ACD000002E08BF0024BEF1806FA8BFA1F1C041C3
:10ACE000BDE8704080F282804FF0000001F1C04169
:10ACF00001F0004170479EEA0C0F0CEA131518BFD3
:10AD000095EA0C0F06D04FF0000081EA030E0EF01A
:10AD1000004170BD00F01CF88900013E00F007B84A
:10AD200000F009B84FEA430C5FEA5C5C08D081EAA6
:10AD3000030100F05BB84FEA410C5FEA5C5CF6D1BE
:10AD40004FF00000014970470000FF070000F87F46
:10AD50000EF1020E2EF0030E5EF8046B364205D49F
:10AD6000012A43EB030515F5001F12D8012841EB1A
:10AD7000010C1CF5001F0CD80ED14FEAD17C15F543
:10AD8000001F0CEB4C0C0CF1020C08BF4CEBD37CFD
:10AD900004E04FF0080C01E04FEAD37C0CEB4C05CB
:10ADA00026FA05F606F00706B6F1040C06D20EEBFD
:10ADB000860CBDE870404CF0010C6047DFE80CF0F9
:10ADC000090B02024FF000414FF00000A1F50021F5
:10ADD00070BD19461046012851EB010418BFD4F587
:10ADE000001484BF002001F0004170BD0808A0F5E8
:10ADF00000114FEA3101704753EA010C17D41CF5DA
:10AE0000801F58BFBCF5801F00F106808B4218BF21
:10AE1000704708BF8242704707D713F5801F58BF9D
:10AE200011F5801F19D48B4270479B4270471CF567
:10AE3000801F08D5BCF5801FF7D5994218BF704711
:10AE400008BF904270474FF4001C1CEB430F38BF03
:10AE50001CEB410F01D2994270470FB40CBC03BCEC
:10AE6000FFF7C1BE91EA030F10B581F000413FF535
:10AE7000E7AB83F0004300F0EFB800002DE9F041AC
:10AE800001F5801CBCF5001FC0F2C3804FEA115CC5
:10AE900021EA0C510CF1FD0C41F480115FEA5C0CCD
:10AEA0000CF5C07C01D3400049413DA4890241EA30
:10AEB000905187028E0E0A0CA45D04FB04F602FB7F
:10AEC00006F6C6F14046A4FB0662F60D46EA4226A7
:10AED00006FB06F4A4FB01235242C3F1404338BFF2
:10AEE0005B1EA6FB02420024E6FB0324D20B42EACF
:10AEF0004446A6FB0623A1FB02E2A3FB07E4A41839
:10AF00004FF0000252F10002E3FB01426442C2F141
:10AF1000404E38BFAEF1010EA6FB04234FF00002F5
:10AF2000E6FB0E32A2FB03464FF00004B61954F1C3
:10AF30000004E2FB0264A1FB06E6A4FB07E816EBB3
:10AF400008064FF0000858F10008E4FB016876425B
:10AF5000C8F1405838BFA8F10108A2FB06E4A3FBE2
:10AF600008E52D194FF0000454F10004E2FB0854E9
:10AF7000A1FB05E6A7FB04E818EB06084FF0000666
:10AF800056F10006E1FB048618F1200556F1000693
:10AF9000A809A8F11B08B10908F03F08B8F10A0F89
:10AFA00040EA86601CD901EB0C51BDE8F08100BF7E
:10AFB000FCF5EEE8E2DDD8D3CFCBC7C3C0BDB9B650
:10AFC000B4B1AEACA9A7A5A3A19F9D9B9A98969555
:10AFD0009392908F8D8C8B898887868584838281DC
:10AFE000A0FB006800FB01F208EB4208B8EB8728E1
:10AFF00007D5341858EB0104D5D5401C51F1000198
:10B00000D1E7341A78EB0104CDD4401E71F1000170
:10B01000C9E75FEA4C0C5FEA9C5C0DD105D34FF0A9
:10B02000000001F00041BDE8F081BDE8F04170B5DD
:10B03000FFF78EFE6DDBFFBEBDE8F0414FF0000074
:10B04000004970470000F87F10B591EA030F48BF30
:10B0500083F000433FF5F4AA841A71EB030C07D286
:10B0600012198CF0004C43EB0C03001B61EB0C013C
:10B07000DFF8A4E14FEA1154A4EB135C1EEA430F7E
:10B0800018BF9EEA445F00F0B08023EA6E0352428C
:10B0900021EA0451C3EB6E0338BF5B1EDCF1200EC6
:10B0A00025D322FA0CFE10EB0E0043FA0CFE41EB06
:10B0B0000E01CCF1200E03FA0EFE10EB0E0051F142
:10B0C0000001CCF1200E29D412FA0EF201EB04514A
:10B0D000BDE8104058BF7047401C1CBFB2F1004F84
:10B0E000704700280CBF491C20F00100704712EB8C
:10B0F000020E43EB030218BF4FF0010E4EEA42026C
:10B10000ACF1200CDCF11E0E54D943FA0CFE10EB0E
:10B110000E0051F1FF31CCF11E0ED5D50EF1010E0E
:10B1200012FA0EFE404141EB010101EB445C5FEA83
:10B130005C5C10D910EBDE7001EB045138BFBEF13E
:10B14000004FBDE8104018BF704700280CBF491CD5
:10B1500020F00100704730D24FEAD42C11F50011D5
:10B1600024F400641BD0B1FA81F20B3AA41AA41E95
:10B17000D2F12003914030FA03F31943904001EBE0
:10B18000CC71002C01EB0451BDE81040A8BF704702
:10B1900001F1C0414FF0000001F000417047B0FAEA
:10B1A00080F310FA03F100D110BDE41A173C4805F2
:10B1B000C90AE4E701EB045110BD491001EB045149
:10B1C000BDE810404FEA300002E04FF00001704748
:10B1D0004A0008BF0042F8D0B2F5001F28BF7047F0
:10B1E00001F000414FF0000070479EEA445F07D035
:10B1F00011EA5E0FBDE8104004BF00210020704737
:10B20000BDE8104070B5FFF7A3FD00BF40DFF63E7C
:10B2100083F00041104670470000E0FFF1F7AFBE39
:10B22000F2F72CB90CF00F03092B08BF082000F02F
:10B2300059800A2B0BD0082B18BF704708BF1CF091
:10B24000400F0AD04FF000004FF0000170471CF093
:10B25000400F18BF4FF0004070471CF0100F08D08F
:10B2600020F0704300F07F4242EAD3014FEA43707E
:10B27000704700F0604021F07F4242EA000201F096
:10B280007F4040EA727070474FF0FF0C4CF4E06C66
:10B290001CEA11531CBF9CEA030C9445C2BFDA425E
:10B2A00001EB02517047002B0DD0BCF1000F0FD005
:10B2B000002A01F00041A4BF41F0E04141F07F616C
:10B2C0004FF00000704701F000414FF00000704760
:10B2D00050EA01334FF09B0C18BF4CF0806C7FF4A8
:10B2E0004FAA70471CF4801F11D01CF4E02F03D02C
:10B2F0006FEACC31490070474FF04050EFF30082C5
:10B3000022F0704242EA000282F3008870474FF058
:10B31000000070470103070F1FFFFF1F0F07030106
:10B320000000000000E0E00000FCFC000000000065
:10B330000000000000000000003F3F00003838001F
:10B34000003F3F00003F3F00003F3F000000000083
:10B35000000000000000F808E8E8E8E80808E8E86D
:10B36000E8E80808E8E8E8E80808F820E000000055
:10B370000000000000001F101717171710101717F4
:10B38000171710101717171710101F0407000000C9
:10B39000000000000000C0E0F0F8FCC05F5555D58B
:10B3A000755555555FC0000809090B0505050B09C2
:10B3B000090000EACC0011F200FC2424E41FE4851B
:10B3C000660000070A0700020B0403040E00B3CF57
:10B3D0000012D2FE5190122400FF80800001000F65
:10B3E00000000101010F000000BFC6008888FF486F
:10B3F00024E4243F24E4040000080F0008080502A8
:10B4000005080800BCBC00000000000000000000AF
:10B4100000000000000000000036360000000000C0
:10B4200000000000000000A3BA00000000000000BF
:10B43000000000000000000000000000583800007C
:10B4400000000000000000000000A3AC00000000AD
:10B4500000000000000000000000000000000018D4
:10B4600024241800000000000000000000A1A30038
:10B47000000000FE000000000000000000000000CE
:10B480000000003300000000000000000000000089
:10B49000A3A100000038340282C27C380000000002
:10B4A000000000000000000037370000000000002E
:10B4B000000000A3BF00008080BEAAAAAAEAAAAA30
:10B4C000AABE80800000048584945C542724245400
:10B4D0004C4484050400EACC004042CC0000F888CB
:10B4E000888808FF0809CA080000003F90681F10FC
:10B4F000209F4027182641F000B3CF002424A4FE4B
:10B50000A3220022CC0000FF00000000080601FF7B
:10B5100000010404040404FF02020200BFC600107C
:10B520001010FF109008888888FF88888808000419
:10B5300044827F01808040432C102846818000BCDB
:10B54000BC001010FF109000FE5252D25252525EB8
:10B55000000042827F8140308F929392FE929396B8
:10B560008000CED50000002424242424FC222222A2
:10B570002322000000020202020242827F02020233
:10B580000202020200CAD6000000F010101010FFE4
:10B5900010101010F000000000000F04040404FF5D
:10B5A000040404040F000000D6D0000000000000D6
:10B5B00001E21CE000000000000000804020100CB0
:10B5C00003000000030C3040808000C8EB0000FE48
:10B5D0000222428272022242827202FE000000FFB8
:10B5E000100806010E100806014E807F0000CDF8FD
:10B5F00000404042CC000444645C47F444444404AA
:10B60000000040201F2044444444447F44444444B8
:10B6100000C1AC00101010FF1050445465C64464C3
:10B62000544440000444827F0182824A56232252BD
:10B630004E820200BDD3000000FE222222FE00FE48
:10B64000828292A29E000080601F0242827F00FFE1
:10B65000402F102C438000B7FE00000090884C570C
:10B66000A42454548C840000000001018042221A5A
:10B6700007024282423E01010100CEF10080809E1D
:10B680009292929EE0809EB2D2929E80000808F430
:10B69000949292F10001F2929494F80800C6F70097
:10B6A0001060028C0008080809FA08080808000061
:10B6B00004047E0140404141417F414141414000FD
:10B6C000D7A200808080FE8282FE8080FE8282FE81
:10B6D0008080000080403F00407F80601F40807F6E
:10B6E000000000B2E1000000F8888888880808FFA0
:10B6F00008090AC8080080601F0010201F80402130
:10B7000016182641F800B3C900080808F808080808
:10B710001010FF101010F000001030101F088848A3
:10B72000300E014080403F0000B9A6000040301EAE
:10B73000101010FF10101010100000008181412126
:10B74000110D0301030D112141818100CAA70000E1
:10B75000FE02FA02FE4020D8171010F010100080F0
:10B7600047300F106780402116081621408000B036
:10B77000DC00080889EA1888000404FC040404FCBE
:10B780000000020100FF0186402018074080403F72
:10B790000000B3F5001010F01F10F00040E0584713
:10B7A000405060C0004022150816210000FE4242B1
:10B7B0004242FE0000CABC00008060F807000000A2
:10B7C000FF40201008040000010000FF00040201F7
:10B7D0003F40404040407800BBAF00040444C44FA9
:10B7E0004444C424242FB4240404004044242415D5
:10B7F0000C04FE040C152424444000B2CB000000CD
:10B80000F8494A4C48F8484C4A49F80000001010E2
:10B810001312121212FF1212121213101000B5A5F9
:10B8200000404042CC0000FC24A4242222A3620059
:10B83000000040201F20584750484542454850408E
:10B8400000B7B5000000FE0202F2121212F202026C
:10B85000FE00000000007F20202724242427202031
:10B860007F000000BBD800000022322AA6A262217D
:10B8700011098101000000004222130B42827E0266
:10B88000020A1223460000CFB5002030AC6330001E
:10B8900088C8A8998E88A8C88800226722121280BA
:10B8A00040300F00003F40407100CDB300808084E5
:10B8B0008484FE82838280FF8080808000008040BC
:10B8C00020180700000000FF0000000000C9FD0074
:10B8D0002030AC6330000202FE0202625AC6000051
:10B8E000226722121240308F80432C102C4380009C
:10B8F000BCB60008C8B88FE8888840300FC8082850
:10B9000018000008180808FF048440300E010E30AB
:10B91000408000C8ED00008060F80780601C1010B7
:10B92000FF1010100000010000FF000202020202DE
:10B93000FF0202020200BCFE0000404244584040A8
:10B940007F40405048C60000000040444444444406
:10B950004444444444FF000000B5B1000808E8290D
:10B960002E28E80808C80C0BE80808000000FF09AA
:10B9700049897F00000F40807F000000C7B00000B1
:10B98000FE20203F2000FC24E4242223E20000804B
:10B990007F0101FF80601F8041261826418000B092
:10B9A000E6000010101010D030FF30D01010101032
:10B9B000000010080402090808FF0808090204082A
:10B9C0001000B1BE00808080BEA2A2A2A2A2A2A24C
:10B9D000BE80808000000000060504040444844406
:10B9E0003C00000000BAC500404042CC0040A09E90
:10B9F0008282829EA02020000000003F9088404369
:10BA00002C10284641808000C9E800809090484C66
:10BA100057242424544C4480808000000000FF49B7
:10BA200049497F494949FF00000000B1B800008042
:10BA300060F807000424242526242424040001009F
:10BA400000FF000000F94949494949F90000D0C503
:10BA500000000000FC54545655545454FC0000009F
:10BA600000403000033941414559414173000830DD
:10BA700000CFA2000000007F494949494949497F58
:10BA8000000000008141211D214181FF89898989B0
:10BA900089818100CAC70000028282422212FA060E
:10BAA00022224242820000010100FC4444444544F9
:10BAB0004444FC00000100B7F10000101090101089
:10BAC0001116101010D01010000040404040435C90
:10BAD0004040504C434040404000C1A20000FE9214
:10BAE000929292FE0000FE020202FE0000003F2041
:10BAF000100A04180000FF000408070000BCB4008E
:10BB0000003E22E2223E0010885724548C000000A0
:10BB1000407E403F22220001FE424242FE010100DF
:10BB2000C2B700001088C43380824222121A262233
:10BB3000408000020100FF00404242427E424242F9
:10BB4000424000BEB6000484E45C44C400F2929219
:10BB5000FE9292F2020002017F10103F808F542467
:10BB60005F4484878000D3B20000FE02FA02FE0028
:10BB700080FF80A090888680008047300F1067008B
:10BB800000FF40230C10204000D5CB00808080BEF9
:10BB9000A2A2A2A2A2A2A2BE8080800000000006F3
:10BBA000050404044484443C00000000BAC50010AD
:10BBB0008C4404E40495A64424148444940C0002A8
:10BBC000027A414143427E42424243F8000000C3B0
:10BBD000DC000484E45C44C40002F2828282FE80C1
:10BBE000800002017F10103F0008080808488840C4
:10BBF0003F00C2EB00C808090EE808405E5050DF65
:10BC000050505E4000206F201C131000FE027F0287
:10BC10007E82FE0000B6CB000000FC040404040495
:10BC200004040404FC00000000007F2020202020E9
:10BC3000202020207F000000BFDA00404424A4948C
:10BC40008C84FF848C94A4244440004040405F4A8C
:10BC50004A4A4A4A4A4A5F40404000B2E9004040EE
:10BC600042CC0020D04C4B48C80808F80000000027
:10BC7000007F20101F1212125F80403F0000D1AFE2
:10BC800000404042CC00202222A262222222200038
:10BC9000000040201F20444E4544444445464C404B
:10BCA00000D4CB00001088C4330040424242C2425C
:10BCB00042424000020100FF0000000040807F007F
:10BCC00000000000D0D000808080BEA2A2A2A2A26C
:10BCD000A2A2BE8080800000000006050404044487
:10BCE00084443C00000000BAC500000000000000D1
:10BCF0000000002F000000000700070000147F1460
:10BD00007F1400242A7F2A1200626408132300365D
:10BD10004955225000000503000000001C2241008C
:10BD2000000041221C000014083E08140008083ED0
:10BD30000808000000A060000008080808080000CB
:10BD400060600000002010080402003E5149453E9A
:10BD50000000427F400000426151494600214145B8
:10BD60004B31001814127F10002745454539003C1F
:10BD70004A494930000171090503003649494936ED
:10BD800000064949291E00003636000000005636DC
:10BD900000000008142241000014141414140000C0
:10BDA0004122140800020151090600324959513E4E
:10BDB000007C1211127C007F49494936003E414106
:10BDC0004122007F4141221C007F49494941007FB7
:10BDD00009090901003E4149497A007F0808087FA6
:10BDE0000000417F4100002040413F01007F0814D6
:10BDF0002241007F40404040007F020C027F007FD4
:10BE00000408107F003E4141413E007F09090906B8
:10BE1000003E4151215E007F0919294600464949EB
:10BE200049310001017F0101003F4040403F001FB8
:10BE30002040201F003F4038403F00631408146337
:10BE400000070870080700615149454300007F4121
:10BE5000410000552A552A55000041417F00000449
:10BE60000201020400404040404000000102040082
:10BE7000002054545478007F4844443800384444E7
:10BE8000442000384444487F003854545418000873
:10BE90007E0901020018A4A4A47C007F0804047891
:10BEA0000000447D4000004080847D00007F102819
:10BEB00044000000417F4000007C04180478007CAE
:10BEC0000804047800384444443800FC242424182E
:10BED0000018242418FC007C08040408004854546A
:10BEE000542000043F444020003C4040207C001C83
:10BEF0002040201C003C4030403C00442810284496
:10BF0000001CA0A0A07C004464544C4414141414DD
:10BF100014140000000000000000000000000000F9
:10BF20000000000000F800000000000000333000B6
:10BF3000000000100C06100C0600000000000000BD
:10BF4000000040C07840C0784000043F04043F0433
:10BF50000400007088FC08300000001820FF211E3B
:10BF60000000F008F000E018000000211C031E2172
:10BF70001E0000F00888700000001E2123241927ED
:10BF8000211010160E00000000000000000000004C
:10BF90000000000000E01804020000000007182064
:10BFA000400000020418E0000000004020180700D4
:10BFB0000000404080F0804040000202010F01027A
:10BFC0000200000000F0000000000101011F01015B
:10BFD0000100000000000000000080B070000000C0
:10BFE000000000000000000000000001010101014C
:10BFF00001010000000000000000003030000000DF
:10C0000000000000000080601804006018060100B5
:10C01000000000E010080810E000000F10202010C1
:10C020000F00001010F8000000000020203F20202A
:10C0300000000070080808887000003028242221C1
:10C040003000003008888848300000182020201177
:10C050000E000000C02010F8000000070424243F58
:10C06000240000F808888808080000192120201101
:10C070000E0000E0108888180000000F1120201129
:10C080000E0000380808C83808000000003F000013
:10C0900000000070880808887000001C22212122FE
:10C0A0001C0000E010080810E000000031222211FE
:10C0B0000F00000000C0C000000000000030300091
:10C0C0000000000000800000000000008060000010
:10C0D0000000000080402010080000010204081049
:10C0E0002000404040404040400004040404040458
:10C0F0000400000810204080000000201008040206
:10C100000100007048080808F00000000030360107
:10C110000000C030C828E810E000071827242314C6
:10C120000B000000C038E0000000203C2302022782
:10C13000382008F8888888700000203F20202011CF
:10C140000E00C0300808080838000718202020100A
:10C15000080008F808080810E000203F2020201000
:10C160000F0008F88888E8081000203F20202320CE
:10C17000180008F88888E8081000203F2000030015
:10C180000000C03008080838000007182020221ED0
:10C19000020008F808000008F808203F21010121EA
:10C1A0003F20000808F8080800000020203F202059
:10C1B000000000000808F8080800C08080807F00A8
:10C1C000000008F888C028180800203F2001263801
:10C1D000200008F8080000000000203F2020202058
:10C1E000300008F8F800F8F80800203F003F003F52
:10C1F000200008F830C00008F808203F2000071889
:10C200003F00E01008080810E0000F102020201068
:10C210000F0008F808080808F000203F210101017C
:10C220000000E01008080810E0000F18242438501F
:10C230004F0008F8888888887000203F2000030C91
:10C24000302000708808080838000038202121229A
:10C250001C00180808F8080818000000203F2000FB
:10C26000000008F808000008F808001F202020201F
:10C270001F000878880000C83808000007380E0141
:10C280000000F80800F80008F800033C0700073C2D
:10C290000300081868808068180820302C03032CDD
:10C2A00030200838C800C83808000000203F2000AF
:10C2B000000010080808C83808002038262120206F
:10C2C0001800000000FE020202000000007F404053
:10C2D0004000000C30C000000000000000010638E3
:10C2E000C00000020202FE000000004040407F004B
:10C2F0000000000004020202040000000000000030
:10C30000000000000000000000008080808080802D
:10C310008080000202040000000000000000000015
:10C32000000000008080808000000019242222226A
:10C330003F2008F8008080000000003F11202011FD
:10C340000E000000008080800000000E11202020E0
:10C350001100000000808088F800000E11202010DD
:10C360003F200000808080800000001F22222222C7
:10C370001300008080F0888888180020203F20204B
:10C3800000000000808080808000006B9494949373
:10C39000600008F8008080800000203F210000201D
:10C3A0003F2000809898000000000020203F2020BF
:10C3B0000000000000809898000000C08080807F0E
:10C3C000000008F8000080808000203F24022D300B
:10C3D0002000000808F8000000000020203F202076
:10C3E00000008080808080808000203F20003F20EF
:10C3F000003F8080008080800000203F21000020DE
:10C400003F200000808080800000001F202020202E
:10C410001F00808000808000000080FFA12020118C
:10C420000E000000008080808000000E112020A0FF
:10C43000FF80808080008080800020203F212000BD
:10C4400001000000808080808000003324242424A8
:10C450001900008080E0808000000000001F202084
:10C4600000008080000000808000001F202020103D
:10C470003F20808080000080808000010E30080610
:10C48000010080800080008080800F300C030C3021
:10C490000F0000808000808080000020312E0E314F
:10C4A0002000808080000080808080818E7018064F
:10C4B000010000808080808080000021302C2221BB
:10C4C000300000000000807C020200000000003FFD
:10C4D000404000000000FF00000000000000FF00DE
:10C4E00000000002027C800000000040403F00008D
:10C4F0000000000601010202040400000000000028
:10C5000000000000600100000100000020000000A9
:10C5100020000000002C0000200000000306010B9A
:10C520000405020925262734350000010001000119
:10C5300000010000004000000000020000000400B4
:10C54000000008000000100044560020445700205E
:10C5500044580020445900200B0000000C0000004B
:10C560000D0000000E0000000F0000001000000091
:10C570001100000038000000390000003A000000FF
:10C580003B0000003B000000000102030405060020
:10C59000040000000800000010000000200000005F
:10C5A00040000000800000000001000001000200C7
:10C5B000040008001000200040008000000100027C
:10C5C0000004000800100020004000800001020369
:10C5D0000405060708090A0B0C0D0E0F01000000E8
:10C5E000020000000400000008000000100000002D
:10C5F000200000004000000080000000000100005A
:10C60000000200000004000000080000001000000C
:10C61000002000000040000000800000060708091C
:10C620000A17171717172828282828280003030691
:10C6300001040602050003051F1C1F1E1F1E1F1FED
:10C640001E1F1E1F000000000000000030313233AA
:10C650003435363738394142434445464030580036
:10C660003031323334353637383961626364656668
:10C6700040307800040000080000000000000002C4
:10C68000000100001000000004FA97999999D93F21
:10C69000AF788E1DC571CC3F9FC678D0099AC33F35
:10C6A000935555555555E53F599322942449D23F0A
:10C6B000DE03CB966446C73F44523EDF12F1C23FD1
:10C6C000000000000000F03F000000000000F83F04
:10C6D00000000000000000000000004003B8E23F3E
:10C6E000000000000000000006D0CF43EBFD4C3EF0
:10C6F000033333333333E33FFFAB6FDBB66DDB3FE5
:10C700004D268F515555D53F01411DA96074D13F2C
:10C7100065DBC9934A86CD3FEF4E454A287ECA3F26
:10C720003E5555555555C53F93BDBE166CC166BFA8
:10C730002CDE25AF6A56113FF16BD2C541BDBBBEA1
:10C74000D0A4BE726937663E000000000000000001
:10C750003031323334353637383961626364656677
:10C76000787000303132333435363738394142430E
:10C77000444546585000000002400000000000A060
:10C780000000000005400000000000C8000000009C
:10C790000C4000000000409C000000001940000018
:10C7A0000020BCBE0000000034400000BFC91B8E4A
:10C7B00000000004B5400000504BCFD06607E2CF28
:10C7C000010000006C4100003E8251AADFEEA73458
:10C7D00001000000D9420000DCB5A0E23A301F970A
:10C7E000FFFFFFFFB4450000FD25A0C8E9A3C14F2E
:10C7F000FFFFFFFFFF3F000000000080000000007F
:10C80000FF3F000000000080000000000D0A2A2AFF
:10C810002A2A2A2A2A2A2A2A2A2A2A2A2A2A2A2A78
:10C820002A2A2A2A2A2A2A2A2A2A2A2A2A2A2A2A68
:10C830002A2A2A2A2A2A2A2A2A2A2A2A2A2A2A2A58
:10C840002A2A2A2A2A2A2A2A2A2A2A2A00000000F0
:10C850000D0AB0E6C8A8B9E9CAF4203A20EACCB378
:10C86000CFBFC6BCBC20323031372F382D323032EA
:10C87000372F38202E0909090909090D0ABCBCCA3D
:10C88000F5D6A7B3D6203A204D722E2057616E6799
:10C8900020203133363335353133363138202E00D0
:10C8A0002A4745542A20496170466C61673A5B25E6
:10C8B000635D21202052756E4170704E756D3A5B3C
:10C8C00041505025635D2120204A756D705265737B
:10C8D000756C743A5B25635D212020426F6F74563E
:10C8E0006572733A5B25735D212020417070566537
:10C8F00072733A5B25735D2120204373713A5B2587
:10C90000735D21202045633230566F6C3A5B25738E
:10C910005D21202053696D49636369643A5B257327
:10C920005D212020467470557365726E616D653AA5
:10C930005B25735D21202046747050617373776F9F
:10C9400072643A5B25735D212020467470466F6CDB
:10C950006465723A5B25735D2120204674704950EE
:10C960003A5B25735D21202054637049503A5B2562
:10C97000735D212020546370506F72743A5B25738D
:10C980005D210000B2CECAFDB2BBBACFB7A821006C
:10C99000C3FCC1EEB8F1CABDB4EDCEF32100000076
:10C9A000C3FCC1EEB2BBD6A7B3D600007175616EF1
:10C9B0002E73756E696E672E636F6D002F676574D9
:10C9C00053797354696D652E646F0000504F535452
:10C9D00020687474703A2F2F25732573204854549F
:10C9E000502F312E310D0A436F6E74656E742D54C5
:10C9F0007970653A6170706C69636174696F6E2FEC
:10CA00006A736F6E3B636861727365743D5554461B
:10CA10002D380D0A486F73743A25730D0A636F6ED3
:10CA200074656E742D6C656E6774683A25640D0AC2
:10CA30000D0A2573000000007B226D6163223A22FB
:10CA40002573227D00000000415445300D0A00008E
:10CA500041542B4342430D0A0000000041542B5126
:10CA6000504F57440D0A000041542B474D520D0AB8
:10CA70000000000041540D0A0000000041542656F9
:10CA80000D0A0000415426570D0A0000453A203097
:10CA900000000000453A2031000000002B434243D3
:10CAA000000000004F4B0000504F574552454420B6
:10CAB000444F574E000000004552524F52000000B4
:10CAC00041542B5149435347503D25642C312C226E
:10CAD0002573222C22222C22222C310D0A00000048
:10CAE00041542B435245473D320D0A0041542B43DC
:10CAF000475245473D320D0A0000000041542B4388
:10CB00005245473F0D0A000041542B4347524547C9
:10CB10003F0D0A0041542B51494143543F0D0A0037
:10CB200041542B51434349440D0A000041542B51B9
:10CB30004E57494E464F0D0A0000000041542B430A
:10CB400053510D0A0000000041542B514944454106
:10CB500043543D25640D0A0041542B51494143542F
:10CB60003D25640D0A0000002B435245473A000062
:10CB70002B43475245473A002B514E57494E464F9B
:10CB80003A0000002B4353513A0000002B51494119
:10CB900043543A002B5143434944000041542B5124
:10CBA00049434C4F53453D25642C31300D0A00005C
:10CBB00041542B51494F50454E3D312C25642C2278
:10CBC000544350222C222573222C25642C25642CBE
:10CBD000310D0A0041542B514953544154453D31C4
:10CBE0002C25640D0A00000041542B514953454E39
:10CBF000443D25642C25640D0A0000002B51495347
:10CC0000544154453A0000002B51494F50454E3A8B
:10CC1000000000003E00000053454E44204F4B00F2
:10CC20002573000041542B51485454504346473D0E
:10CC300022636C6F73657761697474696D65222C0A
:10CC40003130300D0A00000041542B5148545450EB
:10CC500055524C3D25642C36300D0A0041542B5161
:10CC6000485454504346473D22636F6E74656E745A
:10CC700074797065222C310D0A00000041542B514B
:10CC8000485454504346473D22726571756573742C
:10CC9000686561646572222C310D0A0041542B5184
:10CCA000485454504346473D22636F6E7465787410
:10CCB0006964222C320D0A0041542B5148545450BF
:10CCC000504F53543D25642C362C360D0A0000007D
:10CCD00041542B5148545450524541443D360D0A5D
:10CCE000000000002B5148545450504F53543A20E8
:10CCF000302C3230300000002B51485454505245F3
:10CD000041440000434F4E4E4543540058CE040862
:10CD100000000020C40600006CC1030880D1040894
:10CD2000C4060020FCE00000C8C103081001000098
:10CD300043000000F8FFFFFF0040404040404040FB
:10CD400040404141414141404040404040404040DE
:10CD50004040404040404040400502020202020282
:10CD600002020202020202020220202020202020D1
:10CD700020202002020202020202909090909090E5
:10CD800010101010101010101010101010101010A3
:10CD90001010101002020202020288888888888817
:10CDA0000808080808080808080808080808080803
:10CDB000080808080202020240000000000000000B
:10CDC0000000000000000000000000000000000063
:10CDD0000000000000000000000000000000000053
:10CDE0000000000000000000000000000000000043
:10CDF0000000000000000000000000000000000033
:10CE00000000000000000000000000000000000022
:10CE10000000000000000000000000000000000012
:10CE20000000000000000000000000000000000002
:10CE30000000000000000000000000001C000000D6
:10CE400043000000F8FFFFFF0C0000000E00000090
:10CE50000F0000002E000000014832301EA0C9045F
:10CE60000884041A900451320C620117F50D04086D
:10CE70000101100C03020101050946040802011F0B
:10CE80000103020209610C1303011F020403030BD7
:10CE9000B90C1A042418160104040D1147040805DE
:10CEA000010108060505101540040806381E07058F
:10CEB00005116D0C180A0701010608050512C50CBD
:10CEC0001955181F07050808131D41040809010218
:10CED0000A0A090914414204080A010209090A0A56
:10CEE00015910C18160B01030C0C0B0B169D43042B
:10CEF000080C01030B0B0C0C17ED0C18220D010490
:10CF00000F0E0D0D18E94404080E01040D0F0E0E4E
:10CF100019494504080F01040E0D0F0F1AA90C2D15
:10CF200010010510012809793E04081101061101BC
:10CF30001AE10C2D12010712012809493F040813B8
:10CF4000010813011AAD0C2D14010914011A759072
:10CF50002D15010A15011AD90C2D16010B16011AEF
:10CF6000E1902D17010C17011A5D842D18010D1881
:10CF7000011A3D842D19010E19011A910C2D1A0167
:10CF80000F1A01290C412230500D3132312E34312B
:10CF90002E37392E3837180A581B7017CCC9040899
:10CFA000AC041ABC044B38CA2C811A5C10238A02C8
:10CFB0001AA8081AFF011AB8081A041032011A74C4
:10CFC0000C320AAAA41C2203191F111A7C0C190B7B
:10CFD000115A8C1C2A941C193529145A481CB9382A
:10CFE000193532040A15841C32050A15681C3206EC
:10CFF0005A508CDA9C1C412D20CB0408401A94080E
:10D00000A9A829C40A15E054293B5AFC1CAA68386F
:10D01000191929140A19ECC41A0830291CDA7038B5
:10D0200029845A2C1CAA781C198929C45A3C1CDA58
:10D03000843832070A15C07032081A58301ADC5D7D
:10D04000B91C195432091A481C1A900CE91C320AEE
:10D050005A1470DA8C70411AB0142AC8CCCACC3871
:10D060001903111A9C1C0A11648C293B1AD41C291F
:10D07000E8DAFC5429681AE8142A1478D9543204DE
:10D080001A2014291CDA181C411A9C142954E9701E
:10D09000291F0A157C1C298C0A15241C298C0A15A9
:10D0A0005C1C298C1A481C2A580CCACD8C293029A2
:10D0B000A809123832061AB81C323CE9385A073827
:10D0C0003250DAE4E032081AD0143264DAF81C1074
:10D0D0000B3118040809190408402732201468404D
:10D0E000531A2009E268280901020209020A0A0CFF
:10D0F0000A17030A030B0B021438014012441240B2
:10D100001A48041A4C0412501B4004141A04141A2E
:10D1100004141A04141EE1540408ED041AF9042C32
:10D1200005550487198C1C02401C041A30041A444B
:10D13000041A58041A6C041A800419E51B401C04D4
:10D140001A30041A44041A5804111A08681A0C04F4
:10D150001A10041A14041A18041A1C041A200401C0
:10D16000133C0204066819A82A04041506070809D6
:10D170008CA24A04CA5914011B1AAA0101540000C6
:040000050803C131FA
:00000001FF
